:04000003000084BDB8
:020000040000FA
:10800000007F0020BD840000E5840000FD9D00008D
:10801000E9840000EB840000ED840000A04AFCDF4E
:108020008F9E939B2028056E01010000F9840000BB
:10803000F1840000A06301006385000073850000E7
:1080400069960000F7840000C1090100A503010042
:10805000F784000000000000099600000000000006
:10806000F7840000F7840000F7840000F784000024
:10807000F7840000F7840000F7840000F784000014
:10808000F7840000F7840000F7840000F784000004
:10809000F7840000F7840000F7840000F7840000F4
:1080A000F7840000F7840000F7840000000000005F
:1080B00000000000000000000000000000000000C0
:1080C00000000000000000000000000000000000B0
:1080D000000000000000000000000000CD1B0100B7
:1080E0000000000000000000000000000000000090
:1080F0000000000000000000000000000000000080
:10810000000000000000000000000000000000006F
:10811000000000000000000000000000000000005F
:1084000010B5054C237833B9044B13B10448AFF3CE
:1084100000800123237010BDC80C00200000000064
:108420004C7F010008B5034B1BB103490348AFF370
:10843000008008BD00000000CC0C00204C7F010033
:10844000A3F5803A704700BF174B002B08BF134BB2
:108450009D46FFF7F5FF00218B460F461348144A4F
:10846000121A0DF07BFE0E4B002B00D098470D4BDF
:10847000002B00D098470020002104000D000D487B
:10848000002802D00C48AFF3008005F0A2FF2000C6
:10849000290006F02DF90DF015FE00BF00000800C0
:1084A00000000000D1E30000007F0020C80C002085
:1084B0000C4F002000000000000000000649074AA1
:1084C000074B9B1A03DD043BC858D050FBDC08F077
:1084D00005FBFFF7B9FF0000747F010000000020DA
:1084E000C80C0020FEE7FEE7FEE7FEE7FEE7FEE73A
:1084F000FEE7FEE7FEE7FEE71EF0040F0CBFEFF31A
:108500000880EFF30980816911F8021CD9B901B51F
:1085100090E80F10E047BDE800508CE80300194BCD
:1085200093E80600914208BF704719B12CE9F00F9B
:10853000C1F838C01A60906BB0E8F00F80F309887A
:108540006FF0020E7047104A13689942FAD801B5CD
:1085500052F821C00FC8E047BDE80050CCF8000039
:10856000704701B50AF02AFABDE80140EFF3098C23
:10857000D5E701B50AF0EAF9BDE80140EFF3098C4F
:10858000CDE70000900B0020D87B0100034613F8D4
:10859000012B002AFBD1181A0138704700F034BDB6
:1085A000427873B5044680782679130443EA0023A1
:1085B000E0781843637946EA0326A37946EA03463E
:1085C000E37946EA03662378013B0D4636BA0B2B66
:1085D00000F2E280DFE803F03656B0CBCED1D5DB37
:1085E0007C17062606F108039D4240F0D5803146EF
:1085F00004F1080201F081FB0146002840F0CC8024
:108600002A46204627E001F071FB0546002800F0CD
:10861000C38008220021204600F058FE324608217F
:10862000284618E0A37961791B0243EA0143E17906
:10863000194301F06EFB002840F0AE80207800F076
:108640005FFE0AE0012D0DD1284600F059FE01F031
:1086500031FB0B22294600F039FE02B0BDE8704024
:1086600000F022BD0C2D40F09780651C284601F0DB
:10867000E7FA002840F09080207800F041FE0B22BD
:108680000121CDE7012D0BD101F018FB00BA0190BB
:10869000207800F035FE042229460DEB0200DAE7CF
:1086A000052D79D1A378607840EA0320E37840EA89
:1086B0000340237940EA036000BA01F0E3FA00289E
:1086C0006AD114F8010B00F01BFE0422012198E787
:1086D000012D12D101F0FEFA00BA009001F000FB6A
:1086E00000BA0190207800F00BFE0422294668466B
:1086F00000F0ECFD04220521CFE7092D4CD1A37831
:108700006078617940EA0320E37840EA0340237906
:1087100040EA0360A37941EA0321E37941EA034196
:10872000237A41EA036100BA09BA884234D801F0D9
:10873000B9FA2A46002164E7012D0AD1032000F08E
:10874000DFFD01F0C1FA2A468DF80400294601A890
:1087500081E7022D20D1101E18BF012001F09CFAE4
:1087600014F8010B00F0CCFD0122114649E701F09D
:1087700025FA60E701F03AFA5DE71F2363700222F1
:10878000D8E7102300216370A170032239E7034B5F
:1087900001221A70082052E7202050E7E50C002043
:1087A00030B587B00D4604460B22002103A80DF01A
:1087B000D5FCD5B12378132B0ED80F2B05D8A3B138
:1087C00020238DF80C30322361E0113B022B0ED8B0
:1087D000DFE803F0656A0400202BF1D10B220021B1
:1087E00003A800F073FD00F05FFC07B030BD11235B
:1087F0008DF80C3063788DF80D30013B062B49D88D
:10880000DFE803F0040D141A223C41000222524911
:108810008DF80E200DF10F000DF078FCDEE702223E
:10882000ADF808208DF80E2002A9F3E740F20113FD
:10883000ADF808300222F5E701F0E4F847490122DB
:1088400008708DF80E20E5E701F086F84FF47A7491
:108850006043019001F0FEF8082360430290042277
:108860000DEB03010DF10F008DF80E300DF04EFCF5
:1088700004220DEB02010DF11300CDE7012238496E
:108880008DF80E20C6E720238DF80C3036238DF8A6
:108890000D30A3E720238DF80C303423F7E7202395
:1088A0008DF80C303323F2E76378013B092BF1D8C4
:1088B00001A252F823F000BFE1880000E188000027
:1088C000E1880000E1880000E1880000E188000004
:1088D000EB8800001F890000958800003B8900009C
:1088E00020238DF80C303723D1E7A378012B11D149
:1088F000E378082B09D11B4A13701B4B05221A7011
:1089000013238DF80C300723C1E720238DF80C309A
:108910003823BCE720238DF80C303523B7E7A37844
:10892000012BF7D1E378114A003B18BF01231370E4
:1089300013238DF80C300823A9E7A378012BE9D184
:10894000E3780B4A003B18BF0123137013238DF803
:108950000C300A239BE700BFEA070020EB0C002045
:108960008C3B0020EE070020EA0C0020F0070020DE
:10897000E807002000F048BB08B500F097FC702124
:10898000084800F053FC7021074800F061FC722198
:10899000064800F04BFCBDE808400548722100F095
:1089A00057BC00BFA18700009D850000A185000085
:1089B00075890000022808B509D100F05BFC054A62
:1089C00000231370044A01211170044A137000201F
:1089D00008BD00BFEC0C0020F0070020EA0C0020CE
:1089E0002DE9F04100F584708846440201F072F9E7
:1089F000054601F075F9461B06F58023A34214D9FC
:108A0000A4F50437631905EB460607EB050C414650
:108A10000022181ABB189D420BD9A35C0B700132BF
:108A2000B2F5007F01F10101F4D14FF40070BDE80F
:108A3000F0819E4210D90CEB02035B0803F504336E
:108A400012F0010F1B780CBF1B0903F00F03092B59
:108A500094BF30333733E1E7835CDFE710B50020A4
:108A600008F036F900F090FA49F6051398422B49C0
:108A70002B4B3DD049F6061290423BD049F60412EA
:108A8000904239D1274A83F89C21C2F3072483F806
:108A90009D41C2F30744120E83F89E4183F89F2143
:108AA000088000F0E5FC00F02FFF00F0ABFF1E4C4B
:108AB000207000F037FE00F037FE23781B4A022BAF
:108AC0000CBF6423FF2313FB03F05843137000F51E
:108AD000FE404FF60163B0FBF3F0C0B200F038FE89
:108AE00001F05CF8FFF748FFBDE8104000F0A0BAC5
:108AF0000F4AC8E70F4AC6E70F4A83F89C21C2F322
:108B0000072083F89D01C2F30740120E83F89E01EF
:108B100083F89F2149F603130B80C2E7EA07002080
:108B20003808002020630100EB0C0020EF07002034
:108B3000256301002A6301002F63010038B5274B2C
:108B40001B68DB69984750BB254C23788BB108F034
:108B5000DDF8054630BB02200AF044FD214B2570AC
:108B600001221A70204B1B884F2B204B18D807224C
:108B700010E008F0CBF81E4D08B92B7863B1012046
:108B80000AF030FD184A01232370002313802B7054
:108B9000164B09221A7002E02378002BD7D138BD7A
:108BA0000622F7E72378002BF9D008F0AFF8002869
:108BB000F5D00D490D4A0B880A2B04D802201070FD
:108BC00001330B80EBE74F2BF8D9772B01D803202B
:108BD000F5E70420782B1070E1D1F1E74877010028
:108BE000EC0C0020F0070020E80C0020EA0C00202C
:108BF000EE0C00207FB5834D2B78022B42D100F084
:108C0000DBF9814BFF221A70804E814C33782BB1F7
:108C1000062323702B780BB901232B7000F09AFBED
:108C20002B78002B35D17B4B1B78002B31D123784F
:108C3000002B2ED1784B1B78002B4DD000F072FB0F
:108C400038B3764B06221A7005232370744B1B78B9
:108C5000022B07D02B78002B40F0A2806D4B1B78A5
:108C6000002B48D105F01EFD6E4B1A786E4B002A82
:108C700000F09480694A1278082A40F08B80FF2225
:108C80001A7080E0002BBFD100F0AAF95E4B64227D
:108C9000B9E723780A2B2ED801A252F823F000BF9F
:108CA000D98C0000E98D0000E18C00002F8D0000C0
:108CB0003B8D00004D8C0000478D0000D98D0000D9
:108CC000A98D0000CD8C0000D58C0000564BC82229
:108CD0001A7010E0002323704B4B1A78524BF7E7C1
:108CE000524B1B88782253436FF04F0293FBF2F3F1
:108CF0004D4A383B13702378042B7DD04A4B1B78A8
:108D000013FB03F0584300F5FE404FF60163B0FB40
:108D1000F3F0C0B200F01CFD454B1A78002A6ED06B
:108D200000221A7004B0BDE8704003F0B1BE3E4BA3
:108D300050221A703F4B0822CAE73E4A1378002B94
:108D4000D9D0013BD6E700F05FF90B22002101A842
:108D50000DF004FA11238DF80430327809238DF8D0
:108D6000053001238DF8063082B102228DF80720EC
:108D7000002232702B4A13700B22002101A800F050
:108D8000A5FA00F091F900232370B4E703238DF8CE
:108D90000730F1E7062A01D1642271E700226FE76C
:108DA000022BA8D10823EFE71F4A1378092B09D813
:108DB000013313702B78002B9DD1164B1B78002BA1
:108DC000E1D098E70A2B01D1FF23F2E7F52B94BFFE
:108DD000002303F1FF33ECE7174A13783BB1013B63
:108DE000DBB2052B1370EAD10F4B002270E70A2388
:108DF00013700D4BFF226BE70E4B18788AE704B017
:108E000070BD00BF8C3B0020EF070020EF0C00205E
:108E1000EA0C0020ED0C0020E8070020EE070020FF
:108E2000EB0C0020F0070020F1070020E80C0020E8
:108E3000E50C0020E60C0020E40C0020054B1B781C
:108E4000062B02D0082B02D0704700F07BBB00F04D
:108E50006FBB00BFEE070020014B01221A70704764
:108E6000ED0C0020074A08B500231370064A0121C3
:108E70001170064A137000F0FDF9BDE8084000F0DB
:108E8000C3B800BFEC0C0020F0070020EA0C002063
:108E900008B504490B220DF029F908B900F057FF75
:108EA000002008BD3463010070B503F0DBFF70B330
:108EB000224B1A68224BA0F10C01995400F5FA706C
:108EC0001344C0F3072058701E4B186803F0BCF819
:108ED00028B11D494FF4DB72002006F0EBFF1B4B5D
:108EE00017491A68002003F013F938B103F0B2F9FA
:108EF00015494FF4DE72002006F0DCFF03F0AAF9FA
:108F000028B1114940F2C112002006F0D3FF00F051
:108F1000E1FE054600F0E4FE044600F0CFFE064602
:108F200000F0D2FE48B100F0C5FEA3195B1B084952
:108F3000BDE87040002204F0F1BF70BD00000020C9
:108F4000040000204877010040630100E40700208E
:108F5000E18900001FB500230C2201A91030019304
:108F6000029303930DF0C2F8C0B2B0FA80F040094A
:108F700005B05DF804FB0378832B03BF4078B0FA9B
:108F800080F04009002070474FF08053084AD3F822
:108F90000031934208D0074949F6051249F60310FB
:108FA0008B4208BF1046704749F60610704700BF55
:108FB0002028050033280500074B1B681F2B07D806
:108FC0004FF0A04203F5E073032142F823107047ED
:108FD000024A03F01F03F5E7CC3C002000030050D9
:108FE000074B1B681F2B07D84FF0A04203F5E07317
:108FF000022142F823107047024A03F01F03F5E7ED
:10900000CC3C002000030050074B1B681F2B07D8E7
:109010004FF0A04203F5E073022142F8231070479D
:10902000024A03F01F03F5E7F00C00200003005094
:109030004FF08053D3F80021164B9A42164B25D19E
:1090400009221A604FF01022D2F80C32D9071FD52E
:10905000124B0121C3F80415D2F80C1221F00101C2
:10906000C2F80C12D3F80024D207FBD50022C3F8B3
:109070000425BFF34F8F0A490A4BCA6802F4E06225
:109080001343CB60BFF34F8F00BFFDE710221A6080
:10909000FFF7BABF33280500F00C002000E00140C4
:1090A00000ED00E00400FA050A4B1B681F2B0CD8EA
:1090B0004FF0A04203F5E071032042F821000121A6
:1090C00001FA03F3C2F80C357047034A03F01F039B
:1090D000F0E700BFF00C00200003005038B5064D4B
:1090E000064C2A88002120460DF038F800232B80FA
:1090F00043F62013238038BD1015002008110020EE
:1091000008B50346084611460B4A12689A4203D036
:109110000A4A12689A4204D19847BDE80840FFF70E
:10912000DDBF074A1360074B1172506000221A70AE
:10913000BDE8084005F0BEBA14150020181500203F
:10914000F40C0020F207002010F0010F38B5214D7B
:10915000044610D02B6819072AD51F4B5B6A984725
:1091600048B11E490B7833B122041CD51C4BC2B246
:109170001868FFF7C5FF220708D5174B17481B6A69
:109180004FF481619847174B04221A70630708D582
:10919000114B1548DB694FF481619847114B04224C
:1091A0001A702C6038BD6304E5D5104BC2B2DFE7FE
:1091B0005A07E0D5084B5B6A9847230403D50A4950
:1091C0000B4BC2B2D4E76104D5D50749094BC2B2F3
:1091D000CEE700BF2415002018790100000D002003
:1091E0001C15002012150020081100202015002059
:1091F000141500201815002010B5074C23684BB13A
:10920000217A606898470023236063602372034BD0
:1092100001221A7010BD00BFF40C0020F2070020DC
:10922000014BDB68184700BF18790100712905D090
:10923000722905D0702905D1034B186000207047B2
:10924000024BFAE7012070471C1500202015002072
:10925000712905D0722905D0702905D1034B1860FA
:1092600000207047024BFAE70120704714150020D8
:109270001815002008B5FFF731FF4FF48162074849
:1092800000210CF06BFF064A002313605360137239
:10929000044A1370044B01221A7008BD000D00200F
:1092A000F40C002012150020F207002010B5054C28
:1092B000FFF7E0FFA3680448984723690220BDE850
:1092C00010401847187901004991000010B58C181A
:1092D000B4F5816F0B460CD80146064818440CF0D3
:1092E00015FF054B1A88944288BF1C80034B00224F
:1092F0001A7010BD0811002010150020F207002080
:10930000054B1870054B1A880AB901221A80044BC4
:1093100000221A70704700BF0811002010150020AD
:10932000F207002008B5084BDB6A9847074A034656
:10933000107838B103F00100054B1B7803430CBFD4
:109340000120002008BD00BF18790100F2070020AD
:1093500012150020024A13780BB1013B13707047BD
:10936000121500204FF0805330B5D3F800210E4B7A
:109370000E4C0F480F499A420F4A104B0AD11F2535
:1093800025601E2404600620106000220A600B2263
:109390001A6030BD0225256003240460012010609E
:1093A00007220A60F4E700BF3328050028150020D3
:1093B0002C15002038150020301500203415002011
:1093C00010B5044608F026F8FFF70AFE4FF0A04358
:1093D0000222C3F80027C3F804270CB1FFF720FFCF
:1093E0001D4B1E4A1B681E49C3F3801313701D4B8F
:1093F000D3F804230A60D3F80413C3F808131A4BF4
:109400001B681F2B24D84FF0A04101EB830442F0CE
:109410000042D4F8000740F44030C4F800070120AF
:1094200000FA03F3C1F820350E4B0021C3F87C117C
:10943000C3F80423084A402313604FF08043D3F855
:109440000413C3F808138021C3F80413106010BD7F
:10945000064903F01F03D8E700E100E03C150020B7
:109460004015002000600040D03C00200003005068
:1094700008B54FF08043D3F80024D20242BF244AFB
:1094800001211170D3F80034DB0342BF214B0122CC
:109490001A70FFF767FF204B2049D3F804230A60B6
:1094A000D3F80413C3F808131D4B1B681F2B2BD8CC
:1094B0004FF0A04003F5E073002140F82310194B52
:1094C0001B681F2B1CD84FF0A04003F5E07342F03F
:1094D000004240F82310104BC3F87C11C3F804235A
:1094E000114A402313604FF08043D3F80413C3F8AC
:1094F00008134FF4C071C3F804130123136008BDAF
:109500000A4803F01F03E0E7084803F01F03D1E710
:10951000EF0C0020EE0C0020006000404015002001
:10952000D03C00203415002000E100E00003005092
:1095300008B50120FFF744FF4FF080430122C3F834
:10954000002508BD10B50020FFF73AFF30BF4FF0EF
:109550008043D3F80423C3F808234FF4C072C3F840
:109560000423234B01221A602248027832B9402298
:10957000C3F88020BFF34F8FBFF36F8F1E4BD3F81C
:109580000423C3F808231D4B1B681F2B2CD84FF056
:10959000A04202EB8304D4F8001721F44031C4F850
:1095A0000017012101FA03F3C2F82035124B002203
:1095B000C3F87C21124A1268C3F80423037813B15C
:1095C0000B4B40221A604FF0A0430322C3F804273C
:1095D0000222C3F808250122C3F80027BDE8104085
:1095E000C3F8082507F0F4BE064A03F01F03D0E7CE
:1095F00000E100E03C15002000600040D03C00206D
:109600004015002000030050134BD3F87C2110B507
:10961000EAB10022C3F87C21104B1B681F2B17D81E
:109620004FF0A042D2F82005012404FA03F10842C9
:109630000DD002EB8303C2F82015D3F8000720F405
:109640004030C3F80007064BC2F820151C7010BD4F
:10965000044A03F01F03E5E700600040D03C00200F
:10966000EE0C0020000300504FF0804310B5D3F8FB
:109670001C214AB10022C3F81C2100F0C3F90D4B94
:1096800018700D4B01221A704FF08043D3F820213F
:1096900072B10024C3F8204100F0B4F9054B1870F2
:1096A00008F014F90CF06EF8044B1C70044B1C709D
:1096B00010BD00BFEB0C0020EF0C0020ED0C0020D3
:1096C0008C3B0020124B1B78013BDBB2FD2B1DD8DD
:1096D000104B4FF08062C3F88020BFF34F8FBFF371
:1096E0006F8F0D4BD3F80425C3F808250B4A0121D1
:1096F000516011610A490022C1F81025C3F81025F4
:10970000C3F81425C3F81825C3F81C25704700BFFB
:109710004415002000E100E000F0014000A00140FD
:109720000060004070470000074B1B681F2B07D8E4
:109730004FF0A04203F5E073032142F82310704775
:10974000024A03F01F03F5E7C83C00200003005065
:1097500038B53B4C237883420ED070B9FFF7B2FF87
:10976000384B1B681F2B62D84FF0A041012202FA30
:1097700003F3C1F80C35207038BDFF280DD1FFF779
:10978000A1FF304B1B681F2B55D84FF0A041012281
:1097900002FA03F3C1F80835EDE7013BDBB2FD2B1C
:1097A00031D9294A0321C2F808150721C2F810153A
:1097B00000250121C2F80012C2F80455C2F8441570
:1097C00040F6F611C2F840151E4A11681F4A42EAD7
:1097D00001221F49C1F810251E4A01F5A03101F5EB
:1097E000A271C2F81015A1F5A031E439C2F8141520
:1097F00001F5A031E031C2F81815A1F5A031A1F5AD
:109800008871C2F81C15104A00EB80014900FD2B3D
:10981000C2F84415AFD9104B4FF0806119600D4B61
:109820000321C3F804150123D3601360A3E70B4998
:1098300003F01F039AE7094903F01F03A7E700BFDE
:1098400044150020C83C002000A001400300130084
:109850000060004000F0014000E100E00003005023
:109860002DE9F0430646002947D00868254C00231F
:1098700001256560C4F80035C4F80032D4F804232B
:10988000C4F808233F27C4F838354FF0020CC4F859
:1098900008359E46C4F804659846C4F83455DA196C
:1098A000013202EBD272521042EA0229C4F830951A
:1098B000C4F800C5C4F800812560D4F80091B9F15E
:1098C000000FFAD0A560D4F800946560C4F800E5F4
:1098D000B9F1000F13D1571EFA1A002A00F1010046
:1098E000DDDC01B108604FF4966043439809072E10
:1098F00008BF00EB8000BDE8F0830846B6E71346DA
:10990000EAE700BF0030014008B5FFF72BFD0F4B21
:109910001B681F2B16D84FF0A04203F5E0730321FC
:1099200042F823100A4B1B681F2B07D84FF0A042A8
:1099300003F5E073002142F8231008BD054A03F047
:109940001F03F5E7034A03F01F03E6E7281500208D
:109950002C150020000300504FF08053D3F8002155
:10996000044B9A4201D100F07BB8034B00211868E8
:10997000FFF776BF33280500381500202DE9F341A5
:109980001D4E0023019333681F2B00F131004FF06F
:1099900032040D46B0FBF4F42AD84FF0A041012266
:1099A00002FA03F3154FC1F8083540F6B17838686C
:1099B00001A9FFF755FF4FF47A7308FB00F0B0FBE5
:1099C000F3F0019BA34203D2002DF0D0A842EED3C6
:1099D00033681F2B8ABF0A494FF0A04103F01F03D1
:1099E000012202FA03F3C1F80C3502B0BDE8F081A0
:1099F000034903F01F03D2E728150020301500208B
:109A00000003005038B5114B1C681F2C1AD84FF0BA
:109A1000A043D3F8105540F20E6140F6B83025FA55
:109A200004F4FFF7ABFF14F0010F40F20D6304D113
:109A3000984294BF0120032038BD98428CBF022079
:109A40000020F9E7024B04F01F04E2E73415002080
:109A50000003005040F6E44140F6B830FFF78EBFF7
:109A600037B52C4B00200322C3F8000501A9C3F829
:109A7000F0250122C3F8F805C3F8F405C3F8302631
:109A8000C3F82C164FF40031C3F818150D21C3F894
:109A90001015C3F81405110101F1804103EB021404
:109AA00001F5E0410132D3F81855C4F81855082AD9
:109AB000C1F81005C1F81405EDD10122C3F8002545
:109AC0001A60D3F80021002AFBD00022C3F800213D
:109AD00001225A600F4BD3F80421002AFBD0002248
:109AE000C3F8042101229A60D3F81421002AFBD084
:109AF0000022C3F81421BDF8040000B220EAE0708F
:109B0000C0EB0010C0EB0010800A00EB800003B037
:109B100030BD00BF007000400B4B30B521F0030199
:109B20000124C3F804451144801A8A4203D100205D
:109B3000C3F8040530BD841852F8045B2560D3F8DF
:109B40000044E407FBD5F0E700E00140064B0222A9
:109B5000C3F80425C3F80805D3F80024D207FBD5C1
:109B60000020C3F80405704700E0014010B5084C20
:109B7000084B094920460B2240F8043B0CF0C6FA7A
:109B800000234FF4F032E37322616361A36110BDDF
:109B9000F4070020676663732C6401004FF4003102
:109BA000044B0A689A4203D103481C220CF0AEBA57
:109BB000FFF7DCBF67666373F407002008B50A4847
:109BC0001C224FF400310CF091FA50B14FF40030E8
:109BD000FFF7BCFF28B9044A1C214FF40030FFF7FF
:109BE0009BFFC0B208BD00BFF407002010B54FF4C2
:109BF0000030FFF7ABFF044608B9FFF7B7FF204678
:109C000010BD0000F0B50D4D06460FCD87B001AC7C
:109C10000FC42B68236001AF0024083657F8041BDB
:109C2000032230460CF062FA28B10134052CF5D13C
:109C3000002007B0F0BD0120FBE700BFB8610100C4
:109C400038B5054604F0DCF898B12846FFF7DAFF8E
:109C500030B109480B2229460CF058FA002038BDD3
:109C60000822294604480CF051FA0449044803220A
:109C7000F2E70120F3E700BFF80700203464010099
:109C800000080020B0F5F83F9DBF024B186100208E
:109C900001207047F4070020014BD8730020704763
:109CA000F4070020024B586199610020704700BF03
:109CB000F407002000487047F8070020014B18699E
:109CC000704700BFF4070020014BD87B704700BFEE
:109CD000F4070020014B5869704700BFF4070020CB
:109CE000014B9869704700BFF407002000F504306D
:109CF000B0F5802F28BF0020704710F504300B46C8
:109D000005D20344B3F5802F01D8FFF705BF01202A
:109D1000704738B500F5043401F5043544EA05030D
:109D2000C3F30B038BB9AC420FD8B4F5043F0CD38B
:109D3000B5F5802F09D2204604F58054FFF706FFC1
:109D4000A54201D30028F6D038BD0120FCE708B5B4
:109D5000FFF74CFF28B9BDE808404FF4F031FFF79A
:109D6000D8BF08BD08B5EFF3088400F00F030D2B32
:109D700001D1EFF30984E3699A0554BF04F120058A
:109D800004F12405C30658BF483505F077FEEFF30C
:109D9000098005F073FEEFF3088005F06FFEEFF326
:109DA000148005F06BFE284605F068FE606905F03A
:109DB00065FEA06905F062FEE0690E4C05F05EFEEE
:109DC000E06A05F05BFEA06A05F058FE206B05F026
:109DD00055FEE06B05F052FE606B05F04FFEA06B88
:109DE00005F04CFE04494322002006F063F801F020
:109DF00045FCFEE700ED00E0386401007046FFF727
:109E0000B1FF704710B5EFF3108472B60023C16044
:109E100082600360436084F3108810BD38B5044647
:109E2000EFF3108572B64368C268D1544368826804
:109E300001339342436009D30B494FF030020CBF0A
:109E40000120002006F036F800236360D4E9000307
:109E5000C01A05494FF0350218BF012006F02AF854
:109E600085F3108838BD00BF6464010070B50446F6
:109E7000EFF3108672B6D0E90003C01A4FF0420229
:109E800018BF01200C4906F015F82368E268D55C7C
:109E9000A26801339342236009D307494FF0470278
:109EA0000CBF0120002006F005F80023236086F394
:109EB0001088284670BD00BF64640100EFF3108174
:109EC00072B6426803689A423BBF80688018D01A15
:109ED000C01A81F31088704738B5EFF3108572B659
:109EE0008468FFF7EBFF85F31088013C201A38BD2A
:109EF000F8B515460C460646FFF7E0FF854228BF39
:109F000005466719BC4201D12846F8BD3046FFF727
:109F1000ADFF04F8010BF5E7F8B515460C4606460B
:109F2000FFF7DAFF854228BF05466719BC4201D119
:109F30002846F8BD14F8011B3046FFF76FFFF5E720
:109F40000D4B0E4A1B68B0EB930F03D301235370E4
:109F50005360704700EB5303013BB3FBF0F0022862
:109F60004FF0000194BF01200323517088BFB0FB64
:109F7000F3F05060704700BFE4090020481500204E
:109F800070B5064608460D46FEF700FB01303C283A
:109F90000DD82846FEF7FAFA441C224629463046D8
:109FA0000CF0B4F8002386F83B30E0B270BD3C24DE
:109FB000F3E7FF230B704FF0011070472DE9F04FCE
:109FC000047884F080031F2B8BB005468A4604D8A2
:109FD00000F060FD0BB0BDE8F08F04F16003DBB270
:109FE0005E2B02D8FFF7E5FFF4E70B4603F8014BC1
:109FF00005931D2C00F2BC84DFE814F01E009400D1
:10A000009E00B600E901FB01F503BA04A404C400F4
:10A01000D600BA04BA04BA04BA04BA04DB004F0189
:10A0200065017501CD01E301E701BA04BA04BA0480
:10A03000BA04BA04BA0480014378092B01F102057D
:10A040000AD8012B10D9033B062B12D8DFE803F006
:10A05000171B2236474C5000FE2B61D0FF2B59D0E6
:10A06000F02B48D0F12B4BD08AF8014004F10210BC
:10A07000B0E7AB492846FFF783FF0446F4E704F056
:10A0800035F80146F6E7A749062228460CF03EF8C7
:10A090000624E9E7A44B1B69002BE5D093F8A52122
:10A0A00093F8A41141EA022193F8A62193F8A7316D
:10A0B00041EA024151EA0361DCD1D5E79A4B1B69C1
:10A0C000002BD1D093F8A92193F8A81141EA0221DD
:10A0D00093F8AA2193F8AB3141EA0241EAE7924BA7
:10A0E000D96F0029C6D1BFE78F4BD3F88010F8E7AE
:10A0F00004F010F8C5E731238AF802300124B3E7F1
:10A1000000238B70E123CB70F5230B7105234B717A
:10A110000424A9E740238B700023CB700224A3E71B
:10A120000823E9E74378012B3CD9FF237F488AF8CD
:10A13000013000F101104DE74378012B00F2DC8083
:10A140007B4A012313704FF0A0420321C2F8041789
:10A150000221C2F80815C2F80037C2F808358AF89B
:10A1600001304FF00110E4E7714A002313704FF003
:10A17000A0420221C2F800170120C2F804178AF891
:10A180000130D6E7437882786A4943EA02226A4B73
:10A190001B68B3FBF1F303210233B3FBF1F3534329
:10A1A000013BFDD10023C1E700238B704B700220DF
:10A1B000BFE78378C1784278007941EA0021687965
:10A1C00041EA0041A87913F0010541EA00610AD093
:10A1D0004FF0A04012F0010F4FF0020414BFC0F87E
:10A1E0000845C0F80C4513F002060AD04FF0A04015
:10A1F00012F0020F4FF0010414BFC0F80845C0F878
:10A200000C45002939D003F0200001904B488142D1
:10A2100028BF0146642000FB01FC4948D109D0F861
:10A2200004B0029103F004074FEA520E5BB24FEA0A
:10A2300092084FEA52194FF0A0442DB1D4F80415FA
:10A24000C1F340018A4213D12EB1D4F8101501F0A8
:10A2500001018E450CD117B1B8F1000F08D1019959
:10A2600011B1B9F1000F03D1002B06DA029921B127
:10A270004168A1EB0B018C45DFD84FF0A04231487B
:10A28000D2F80435D2F810255200C3F3400302F08F
:10A29000020213438AF801304BE7AB78407840EA7A
:10A2A0000320EB7840EA03402B7950EA036004D1A5
:10A2B000FF2325488AF801303BE71D4B9860FFF7E4
:10A2C0003FFE0023F5E74478002C08BF4FF480746C
:10A2D000811C204600F07EFC0023E01D8AF801303E
:10A2E000C00801305EE04378114903F003020132F7
:10A2F000C3F380030A774B77002330E74FF0000B5E
:10A3000081F801B0012443788F1C2546811C4FF051
:10A31000A048A24603F1FF39C3B944EA054008E763
:10A32000876401008F640100A06301000100020046
:10A330004815002040420F00E4090020C0C62D004F
:10A34000001000E0010006000100040011F8010BFC
:10A3500010F03F0643B208BF4026002BB4BFC8F838
:10A3600000B7C8F818A507363A4602930191F608D7
:10A3700000F072FC0199029BB9F1000F01D1C8F8FD
:10A3800018A5002B05F10105B9BFBF19A41989193A
:10A39000AD194B46BEE7FF234B704278811C01206C
:10A3A000013A03D2000440F00100C2E60B7813F03A
:10A3B0003F0308BF40230733DB0801331944184427
:10A3C000EEE7FF2340784B708BE7FF23C7E6A84BEF
:10A3D00042781A74C178827842EA01229A8202791C
:10A3E000417942EA0122DA820023A2488AF8013048
:10A3F0009FE6431C06939E4B82781B780192012BAB
:10A4000000F1030440F0E081DFF86C924FF00008A7
:10A41000CD1C89F8008046464046CDF80C80019B53
:10A42000FBB9012811D1002E00F0AF81904B924F63
:10A430009E8A09A90E2000F08DFD022840F0988127
:10A440001EB13B78013E002BF3D0039B8AF801300C
:10A45000069B8AF80200E41A059BE81A40EA0440C9
:10A4600067E62346DFF808B213F8017B029317F082
:10A47000020F00F01D81002E4ED007F01103012BBA
:10A48000BBF814B01CD109A9384600F063FD0228BE
:10A4900028D1BBF1000F05D099F800300BF1FF3B3C
:10A4A000002BF0D0029C23789A0740F15F81DF06F1
:10A4B00000F15C810134019B013B0193F3D1B0E7D2
:10A4C00009A90E2000F046FD02280AD1BBF1000FB9
:10A4D00005D099F800300BF1FF3B002BF0D000269F
:10A4E000E0E700260128DDD1099B2B701A0A6A706B
:10A4F0001A0C1B0EAA70EB702A1D002E43D03B06CF
:10A5000040D55B4BDB682B711A0A6A711A0C1B0E63
:10A51000AA71EB7130460835554B17F01002B3F8AD
:10A5200014B007F001015DD0A0786278DB8A049353
:10A5300042EA0022E07842EA0042207942EA0062E0
:10A540000792621D029201BB494CB4F814B009A9EC
:10A55000384600F0FFFC0228014629D1BBF1000F6C
:10A5600005D099F800300BF1FF3B002BEFD0404BAA
:10A570009A69099B1340079A9A422DD041F0100026
:10A58000C0B28FE730461546C6E70021384600F0D6
:10A59000E1FC022809D1BBF1000F83D099F800300B
:10A5A0000BF1FF3B002BF0D07CE70128CCD079E702
:10A5B000A269099B012803EA0203D8D1079A9A42AB
:10A5C000D5D0049B002BD2D0049A99F80030013AE0
:10A5D0000492002BB9D0CAE701287FF463AF4FF093
:10A5E000000826E091B3002EF9D10021384600F092
:10A5F000B1FC02281E4B0AD1BBF1000F3FF46FAF34
:10A6000099F800200BF1FF3B002AEED04AE7012821
:10A610007FF448AF3E0640F1A380DB682B701A0A36
:10A620006A701A0C1B0EAA70EB704FF000080646F9
:10A630000435039B99F8002001330393019B013BF0
:10A64000002A7FF42FAF029C0193E8E609A938465F
:10A6500000F080FC0228064B10D1BBF1000F3FF444
:10A6600021AF99F800200BF1FF3B002AEED019E74B
:10A6700048150020010005006815002001287FF41E
:10A6800011AF3C060AD5DB682A46190A02F8043BDA
:10A690006970190C1B0EA970EB701546099B2B7085
:10A6A0001A0A6A701A0C1B0EAA70EB70043596E732
:10A6B000F6B1BBF81430049309A90E2000F04AFC4F
:10A6C000022809D1049B002B3FF4ECAE99F800203E
:10A6D000013B002AEFD0E5E601287FF4E3AE099BB9
:10A6E0002B701A0A6A701A0C1B0EAA70EB700435D4
:10A6F000A278637843EA0223E27843EA02432279AC
:10A7000017F0200F43EA026304F105020292099355
:10A710009A4A03D09361002601208AE7968A09A904
:10A72000384600F017FC022808D1002E3FF4BAAEDC
:10A7300099F80030013E002BF1D0D0E601287FF4DB
:10A74000CEAE390610D5DBF80C302B701A0A6A70C1
:10A750001A0C1B0EAA70EB7080460435002668E7C1
:10A760004FF00008064664E78046F7E70534A2E6A6
:10A7700001287FF46AAE099B2B701A0A6A701A0CC2
:10A780001B0EAA70EB7004355FE6B8F1000F3FF4C2
:10A790005CAE7A4B7A4F9E8A00210E2000F0DAFBE5
:10A7A00002287FF452AE002E3FF44FAE3B78013EBC
:10A7B000002BF1D049E62378990712D5DA0610D498
:10A7C0000134019B013B0193019B002BF3D18AF8DB
:10A7D00001308AF80230069BE01A000440F00200C3
:10A7E000A7E40534EDE7DFF894B19BF80030012BC6
:10A7F0004FF0000340F0A180614C90F8028023707C
:10A80000C3780A1D58EA0328019200F09480077962
:10A8100017F0020611D1431DB045BBF8149069D161
:10A8200000210E2000F096FB022839D1B9F1010970
:10A8300036D32378002BF3D032E017F0010010D08C
:10A84000BBF814600021384600F084FB022806D1D2
:10A8500036B32378013E002BF4D0002620E00128F7
:10A86000FBD1DDF804904346A8EB0306CDF8049035
:10A870005A1EABB11AB917F0010F18BF0E27BBF85B
:10A880001430039209A93846029300F063FB0228B2
:10A89000039A1DD1029B1BB12178013B0029F0D006
:10A8A000019B059A8AF80160360A8AF803008AF843
:10A8B0000260981A2B799B075FBFAC78ED7844EA69
:10A8C000052401344CBF40F4802040EA844030E449
:10A8D000012809F10409E3D1099B09F8043C190A8C
:10A8E00009F8031C190C1B0E09F8013C09F8021C9D
:10A8F0001346B9E759781A7842EA0122997842EA70
:10A900000142D97842EA01620992043309A9384622
:10A91000029300F01FFB0228029B08D1B9F1000F3F
:10A92000BED0227809F1FF39002AEFD0B8E701281C
:10A93000B6D1013670E740468FE74B708B70CB7015
:10A940000320B7E70D4B1B78012B0FD1C27883781A
:10A9500043EA0223027943EA0243427909A943EA1E
:10A9600002630020099300F0F5FA3DE5FF233CE582
:10A97000FF230B704FF00110FFF72CBB4815002090
:10A9800068150020F8B505787F2D15D10C46871C79
:10A9900004F8025B45784D704FF002160DB9304651
:10A9A000F8BD21463846FFF709FB013D064407EB99
:10A9B000104714FA80F4F1E7BDE8F840FFF7FEBA5B
:10A9C000064B0748986000221A701A7464219A6135
:10A9D000012259619A83FFF7B3BA00BF48150020DE
:10A9E00000127A0000230822C0F81832C0F81C3286
:10A9F000C0F81022C0F8143270470346D0F8140291
:10AA000010B5B8B10138C3F81402D3F81C0203EB37
:10AA100080140C6000F58071013033F81110116062
:10AA2000D3F8102200F007000132C3F81C02C3F86B
:10AA30001022012010BD70B50446D0F810020E4659
:10AA40001D4630B30138C4F81002D4F81802412A68
:10AA500028BF402204EB80100BF058FBD4F81812EA
:10AA6000304604EB8111FFF78DFFD4F8182202F570
:10AA7000807324F8130004EB82132B60D4F8143293
:10AA8000013202F007020133C4F81822C4F814326C
:10AA9000012070BD7FB503780B70803B06460D46E4
:10AAA0000D2B00F28E80DFE803F007172239448C6B
:10AAB0008C8C54626C71758303F018FB0646FDF7AD
:10AAC00065FDC4B2687022463146A81C0BF01EFB1F
:10AAD00004F58030023008E002A805F0E9F807220A
:10AAE00002A9681C0BF012FB374804B070BD02A825
:10AAF00005F0DEF80422711C0DEB02000024019425
:10AB00000BF004FB019B029302A805F0B7F8204666
:10AB100005F0E2F801232D486B70E6E73E21A81C02
:10AB200006F050FD044610B1012003F0A7FD6C7043
:10AB3000CEE744780230214606F010FD012003F0F4
:10AB40009DFD0123E01800046B70184300F1011013
:10AB5000CBE701234B70407820B903F0BBFD4FF0E9
:10AB60000210C2E70128F8D000234B70F7E7012359
:10AB70004B7005F057F810B9022008F033FD144867
:10AB8000B3E7407800F0E0FE6870E8E700F048FFC7
:10AB90006870F4E74478012003F07AFD2146B01C88
:10ABA00000F008FF6870601C000440F00100CDE771
:10ABB00000234B70407810B901F096FBCFE70120DD
:10ABC000FAE74FF0011090E70900010002000500CC
:10ABD0000200010000283BD01E4B2DE9F04100246B
:10ABE000421E4FF0A04C58684FF001082346022542
:10ABF00015E013F0010F04F1FF34074606461BD0A1
:10AC0000CCF80885CCF80C55013FFDD1CCF808559F
:10AC1000013EFDD1013A561C4FEA530316D08E4631
:10AC2000002CE6D11EF8013B13F0010F4FF0070492
:10AC3000714607460646E3D1CCF80C85CCF80C5596
:10AC4000013EFDD1CCF808550646E1E7BDE8F081AC
:10AC5000704700BF4815002010F03F0C08BF4FF0B0
:10AC6000400C0306F0B540F1AD80554D14464FF051
:10AC7000A04302206968C3F80C050A46013AFDD1D9
:10AC8000D3F81025C3F808050E46013EFDD14FEA62
:10AC9000C21EBCF1010F0F465FFA8EF600F0408134
:10ACA000C3F80C05013FFDD1D3F81025C3F8080502
:10ACB0000F46013FFDD14FEAC21E5FFA8EFEBCF186
:10ACC000020F0A464EEA560E00F02F81C3F80C051B
:10ACD000013AFDD1D3F81025C3F808050E46013E10
:10ACE000FDD1D201D2B2BCF1030F0E4642EA5E0E94
:10ACF00000F01E81C3F80C05013EFDD1D3F81025EC
:10AD0000C3F808050E46013EFDD1D201D2B2BCF116
:10AD1000040F0E4642EA5E0E00F00D81C3F80C05EA
:10AD2000013EFDD1D3F81025C3F808050E46013EBB
:10AD3000FDD1D201D2B2BCF1050F0E4642EA5E0E41
:10AD400000F0FC80C3F80C05013EFDD1D3F81025BE
:10AD5000C3F808050E46013EFDD1D201D2B2BCF1C6
:10AD6000060F0E4642EA5E0E00F0EB80C3F80C05BB
:10AD7000013EFDD1D3F81025C3F808050E46013E6B
:10AD8000FDD1D201D2B2BCF1070F0E4642EA5E0EEF
:10AD900000F0DA80C3F80C05013EFDD1D3F8102590
:10ADA000C3F808050139FDD1D201D2B242EA5E0EE4
:10ADB000BCF1080C04F801EB7FF45CAFF0BD00BF00
:10ADC00048150020624A52680E464FF0A043012405
:10ADD000022016F801EB1EF0010F0CBFC3F80C4562
:10ADE000C3F808451546C3F80C05013DFDD1C3F86D
:10ADF00008051546013DFDD1BCF1010FDED01EF066
:10AE0000020F0CBFC3F80C45C3F808451146C3F840
:10AE10000C050139FDD1C3F8080511460139FDD1F2
:10AE2000BCF1020FCAD01EF0040F0CBFC3F80C45D2
:10AE3000C3F808451146C3F80C050139FDD1C3F824
:10AE4000080511460139FDD1BCF1030FB6D01EF043
:10AE5000080F0CBFC3F80C45C3F808451146C3F8EA
:10AE60000C050139FDD1C3F8080511460139FDD1A2
:10AE7000BCF1040FA2D01EF0100F0CBFC3F80C459C
:10AE8000C3F808451146C3F80C050139FDD1C3F8D4
:10AE9000080511460139FDD1BCF1050F8ED01EF019
:10AEA000200F0CBFC3F80C45C3F808451146C3F882
:10AEB0000C050139FDD1C3F8080511460139FDD152
:10AEC000BCF1060F3FF47AAF1EF0400F0CBFC3F881
:10AED0000C45C3F808451146C3F80C050139FDD1EE
:10AEE000C3F8080511460139FDD1BCF1070F4FEA3F
:10AEF000DE113FF463AF81B9C3F80C451146C3F8C6
:10AF00000C050139FDD1C3F8080511460139FDD101
:10AF1000BCF1080C7FF45DAFF0BDC3F80845EDE768
:10AF20004FEAD61E84F800E0F0BD4FEA9E1EF9E716
:10AF30004FEA5E1EF6E74FEA1E1EF3E74FEADE0E0B
:10AF4000F0E74FEA9E0EEDE74FEA5E0EEAE700BF3C
:10AF5000481500202DE9F0475A4E737886468A46F8
:10AF6000002B00F0B1804FF0A043012202201EF020
:10AF7000010FC3F80825C3F80C05C3F8080514BF72
:10AF8000C3F80825C3F80C254FF0A0420223012086
:10AF90001EF0020FC2F80C35C2F8083514BFC2F813
:10AFA0000805C2F80C054FF0A0420220C2F80C05BB
:10AFB0001EF0040FC2F808054FF0010014BFC2F8DC
:10AFC0000805C2F80C054FEA5E034FF0A0420220CC
:10AFD00003EB9E03C2F80C050124C2F808051EF01D
:10AFE000080F4FEADE00734414BFC2F80845C2F8E8
:10AFF0000C4503444FF0A042022013F0010F4FF024
:10B000000103C2F80C05C2F8080514BFC2F80835E0
:10B01000C2F80C354FF0A0430220C3F80C05C3F86A
:10B020000805327F0124C3F80C45C3F80C05C3F8AA
:10B030000805C3F808450024C3F80C05C3F8080543
:10B04000C3F8004714462AB1013CC3F80C05C3F805
:10B050000805F9D14FF0A0430225C3F80C55D3F8E9
:10B060001075C3F80855C3F80C55D3F81005C3F88C
:10B070000855C3F80C55D3F81045C3F808554000DF
:10B0800004FA05FC28400CF0040C07F0010740EA24
:10B090000C003843012800F08181022800F0C881AB
:10B0A000042800F0C5812132013AC3F80C55C3F8D9
:10B0B0000855F9D10122C3F81825C0B2C3F80825F4
:10B0C000BDE8F087481500204FF0A0420120C2F8EB
:10B0D000080573680224C2F80C451D46013DFDD1E8
:10B0E000C2F808451C46013CFDD11EF0010F14BFFB
:10B0F000C2F80805C2F80C054FF0A0400222C0F8C3
:10B100000C251C46013CFDD1C0F808251A46013A21
:10B11000FDD101241EF0020F14BFC0F80845C0F88D
:10B120000C454FF0A04002244FEA5E02C0F80C45E7
:10B130001D46013DFDD1C0F808451C46013CFDD12E
:10B1400001241EF0040F14BFC0F80845C0F80C45D8
:10B150004FF0A040022402EB9E02C0F80C451D46B1
:10B16000013DFDD1C0F808451C46013CFDD101243C
:10B170001EF0080F14BFC0F80845C0F80C454FF08A
:10B18000A040022472444FEADE07C0F80C451D4679
:10B19000013DFDD1C0F808451C46013CFDD13A44B3
:10B1A00012F0010F4FF0010214BFC0F80825C0F8DB
:10B1B0000C254FF0A0420227C2F80C751846013842
:10B1C000FDD1C2F8087518460138FDD10120C2F83A
:10B1D0000C051C46C2F80C75013CFDD1C2F808757F
:10B1E0001C46013CFDD1C2F80805C2F80C75184692
:10B1F0000138FDD1C2F8087518460138FDD1347FF9
:10B200000020C2F80007A44664B1C2F80C751846C5
:10B210000138FDD1C2F808751D46013DFDD1BCF1D4
:10B22000010CF2D14FF0A0420225C2F80C5518468D
:10B230000138FDD1D2F81085C2F8085518460138FA
:10B24000FDD1C2F80C5518460138FDD1D2F8107561
:10B25000C2F8085518460138FDD1C2F80C551846F9
:10B260000138FDD1D2F81005C2F808551946013948
:10B27000FDD14FEA470CA8400CEA050C00F0040091
:10B280004CEA000C08F001084CEA080CBCF1010F74
:10B290001DD0BCF1020F00F0FA80BCF1040F00F0E9
:10B2A000F6802134C2F80C5519460139FDD1C2F897
:10B2B000085519460139FDD1013CF3D10123C2F8EB
:10B2C00018355FFA8CF0C2F80835BDE8F0871EF03B
:10B2D000020740F028815CB1C2F80C5518460138CD
:10B2E000FDD1C2F8085518460138FDD1013CF3D113
:10B2F0004FF0A0404FF00108C0F81885DAF80020A0
:10B300002021022412F0010F14BFC0F80885C0F8F4
:10B310000C851D46C0F80C45013DFDD1C0F808451F
:10B320001D46013DFDD1013917444FEA5202E9D1D2
:10B330004FF0A042F8074FF001014CBFC2F80815CA
:10B34000C2F80C154FF0A0420221C2F80C151846A5
:10B350000138FDD1C2F80815013BFDD101201EF0D6
:10B36000800F1EBF934B5B68F360337C93B14FF04B
:10B37000A04101227468C1F80C250225C1F80C55C2
:10B380002246013AFDD1C1F808552246013AFDD1C5
:10B39000013BF3D14FF0A04301228FE61EF00200E3
:10B3A00040F00A812AB1013AC3F80C55C3F8085598
:10B3B000F9D14FF0A0420125C2F81855DAF8003053
:10B3C00020210224DF074CBFC2F80855C2F80C55F3
:10B3D00001391844C2F80C454FEA5303C2F8084536
:10B3E000F0D14FF0A0430122C4074CBFC3F8082599
:10B3F000C3F80C254FF0A0430222C3F80C2501200E
:10B40000C3F808251EF0800F1EBF6A4B5B68F3600F
:10B41000337C002BBED04FF0A0420121C2F80C15A6
:10B420000221013BC2F80C15C2F80815F9D1B1E7A9
:10B43000757F002D6FD01EF0020640F00281002AB9
:10B4400000F013814FF0A0430221013AC3F80C151C
:10B45000C3F80815F9D10122C3F818257DB10EF003
:10B46000020666B94FF0A0420123C2F80C35022152
:10B470002123013BC2F80C15C2F80815F9D14FF091
:10B48000A0430122C3F80825C0B2BDE8F087767F4B
:10B49000002E38D01EF0020740F0C280002C00F0D1
:10B4A000DB804FF0A0410220C1F80C051A46013A9A
:10B4B000FDD1C1F808051A46013AFDD1013CF3D18E
:10B4C0000122C1F81825AEB10EF0020797B94FF06E
:10B4D000A0400122C0F80C2502242122C0F80C450E
:10B4E00019460139FDD1C0F8084519460139FDD189
:10B4F000013AF3D14FF0A0430122C3F808255FFAC7
:10B500008CF0BDE8F087002CCBD14FF0A043012296
:10B51000C3F81825EEE7002A94D14FF0A04301228A
:10B52000C3F81825ABE74FF000092027C846C2F83A
:10B530000C5518460138FDD1D2F81005C2F808554F
:10B5400000F0010019460139FDD18044013F4FEA66
:10B55000C07040EA5909EAD1C2F80C5518460138C2
:10B56000FDD1D2F81005C2F80855013BFDD188EA9B
:10B57000000818F0010F0CBF01200820BAF1000FDD
:10B5800001D0CAF800907CB172684FF0A04102254A
:10B59000C1F80C551346013BFDD1C1F808551346BF
:10B5A000013BFDD1013CF3D14FF0A0430122C3F890
:10B5B0001825D4E6001000E04FF00008202447468C
:10B5C000C3F80C55D3F81005C3F8085500F0010076
:10B5D0000744013C4FEAC07040EA5808F0D1C3F874
:10B5E0000C55D3F81005C3F80855474017F0010F64
:10B5F0000CBF01200820BAF1000F01D0CAF800806A
:10B6000042B14FF0A0430221013AC3F80C15C3F830
:10B610000815F9D14FF0A0430122C3F81825F1E62F
:10B6200021224FF0A0400225C0F80C5519460139DF
:10B63000FDD1C0F8085519460139FDD1013AF3D1C1
:10B640002CE721234FF0A0410224013BC1F80C4517
:10B65000C1F80845F9D1F2E64FF0A0420121C2F845
:10B660001815002F7FF446AF31E74FF0A0430122B9
:10B67000C3F81825002E7FF402AFF3E6BFF34F8F17
:10B680000549064BCA6802F4E0621343CB60BFF37E
:10B690004F8F00BFFDE700BF00ED00E00400FA059A
:10B6A000DFF854C0F0B54FF0FF33002401278C427F
:10B6B00003DB93FAA3F0C043F0BD065D072200252B
:10B6C00016F0010F1CBF07FA02FE45EA0E05013A0B
:10B6D0004FEA5606F4D283EA05630822002B02F1F2
:10B6E000FF324FEA4303B8BF83EA0C0312F0FF02B4
:10B6F000F4D10134DBE700BFB71DC104DFF854C04B
:10B70000F0B500240127C04390FAA0F0944203DB77
:10B7100090FAA0F0C043F0BD0E5D0723002516F09F
:10B72000010F1CBF07FA03FE45EA0E05013B4FEA75
:10B730005606F4D280EA05600823002803F1FF339F
:10B740004FEA4000B8BF80EA0C0013F0FF03F4D1C9
:10B750000134DBE7B71DC10400F09EBBF0B5002348
:10B7600089B0CDE906330D4616460593441C06AF55
:10B7700005AB01934FF4807300930297234607AA09
:10B780003146284600F0D4FF38B9069A1AB1059818
:10B79000214600F081FA09B0F0BD02280CD1069ACA
:10B7A0001AB9079BF61A1D44E2E70598214600F0F6
:10B7B00073FA0028F5D0EEE7012809D1069A2AB1DC
:10B7C0000598214600F068FA0028E4D11320E2E74A
:10B7D00004280DD0431FDBB2012BC9D8053818BF90
:10B7E000012004494FF4B07204F064FB1620D2E744
:10B7F0001520D0E79564010010B540F2011204460F
:10B8000000210AF0ABFC00F06DFF00232370BDE8BF
:10B81000104000F00FBA00F00DBA08B504F0E2FBDA
:10B82000431E5842584108BD08B500231A4600F08F
:10B8300013F9003818BF012008BDF0B5044690F890
:10B8400030002F2885B00F4615462DD8C0F13006A0
:10B85000964228BF1646324620440AF057FC94F818
:10B8600030103144C9B22F2984F8301027D9002371
:10B870001A46204600F0F0F820B303AB00220093F4
:10B88000114602AB00F028F9D0B9029894F83020A4
:10B890006063214600F000FA90B9636B94F83020A1
:10B8A00013443744AD1B6363606B2A46394600F08E
:10B8B000F3F928B9626B2A446263142000E0002087
:10B8C00005B0F0BD1C20FBE708B507F05BFC054B9D
:10B8D00005491B681B1A584258416222BDE80840BE
:10B8E00004F0E8BA781600209564010000F0D4BA9C
:10B8F00070B5084E336804460D46984740B9336921
:10B9000029462046984700280CBF0320012070BD1F
:10B910000020FCE71008002010B500F10804032205
:10B92000074821460AF031FC40B10648032221466F
:10B930000AF02BFC00280CBF0120032010BD00BF23
:10B9400034640100C764010070B5144D2E780446BC
:10B9500036B185220020124904F0ACFA022070BDF5
:10B96000012801D98B22F5E707F00CFC0D4B4FF4B1
:10B970008272186031460C480AF0F0FB01232B70EC
:10B980000A4B094803EB0414094B1C606368984791
:10B990000028E4D003232B70E1E700BF74160020D9
:10B9A0009564010078160020701500201008002012
:10B9B0006C15002070B5164D2B78012B04460E46F1
:10B9C00007D01449A422002004F074FA022420466F
:10B9D00070BDFFF779FF104B10481B6821469B682C
:10B9E000324698471328044602D102232B70EEE713
:10B9F000142800D048B928780649431E58424FF011
:10BA0000B202584104F056FAE1E70323EEE700BF23
:10BA100074160020956401006C150020701500203C
:10BA200010B5094C207828B90849C02204F042FA20
:10BA3000022010BDFFF748FF054B06481B68DB6876
:10BA4000984700232370F4E77416002095640100E2
:10BA50006C1500207015002030B5054608462F28CB
:10BA600085B094BF00200120184947221C4604F0ED
:10BA700021FA0C2205F1200101A80AF047FB0CB9BC
:10BA8000134B1C70134B029A9A420ED103F136539A
:10BA9000019803F5672303F26F63984213D0FC3BD0
:10BAA000C31A5842584105B030BD284604F086FA02
:10BAB00028B114B9064B01221A700320F3E7002CB9
:10BAC00018BF0320EFE70220EDE700BFCB640100C1
:10BAD000B61600202028056E2DE9F047DDF82080FD
:10BAE00006460D4691461F4613B1B8F1000F09D125
:10BAF00071224049002004F0DDF94FF00209484668
:10BB0000BDE8F0874FF0000AC3F800A0C8F800A015
:10BB100002F03EFC044600B3022E0CD1B9F1000F36
:10BB200002D0B5F5004F55D1334B1C684FF400459A
:10BB30004FF0000905E0032EF0D0002425464FF019
:10BB40001C0904F077F808B9012E50D0B9F1000FA4
:10BB5000D5D1002C47D1B822CBE702F01BFC00283E
:10BB6000EBD0012E08D1B9F1000F01D0002D36D154
:10BB7000214B00251C68DBE7032EDED11F4B1A6921
:10BB8000002ADAD00C325378157845EA03259378E9
:10BB900045EA0345D37855EA03650DD15179137908
:10BBA00043EA0123917943EA0143D17953EA0163DE
:10BBB00002D1134B1C68BBE7517A137A43EA012385
:10BBC000917A43EA0143D17A43EA0163012BF0D031
:10BBD0001432D8E7544655464FF01B09B1E72546C5
:10BBE0004FF01A09ADE73D60C8F8004087E74FF015
:10BBF0001C0984E7CB6401008C650100A06301008F
:10BC00004877010070B506460C46154602F0C2FBA7
:10BC100048B1032E07D1064B1B6923B129462046A4
:10BC2000FDF798F908B9002070BD1D20FCE700BFA2
:10BC3000A063010038B50F4D2C783CB10E49DA22D3
:10BC4000002004F037F90224204638BD0B4830228A
:10BC5000FF210AF083FA01232B70094B1C70094B5A
:10BC60001C60094B1C60094B1C60094B1C70094B84
:10BC70001C70E9E7BD160020CB640100801600208F
:10BC8000B5160020B0160020B81600207C16002043
:10BC9000B4160020BC1600202DE9F04F734E154657
:10BCA0003278012A85B004460F4608D0002070493A
:10BCB000EF2204F0FFF8022005B0BDE8F08F6D4BD5
:10BCC000197821B96C491A7008606C490860DFF86E
:10BCD000B08198F80030002B70D1684A1368591968
:10BCE000A342116048D1DFF89CA1DFF89CB1DAF8DB
:10BCF0000000C0F13009A94528BFA94639464A4687
:10BD000058440AF003FADAF8000048442F28CAF829
:10BD100000004F44A5EB09054C444BD9A0F130037A
:10BD200058425841524940F2111204F0C3F8524AA5
:10BD3000DAF80010126801235846FFF78DFE534BC6
:10BD4000187002ABDFF844914B490093096899F8E9
:10BD5000000003AB0122FFF7BFFE50B903F07AFFEA
:10BD600070B1484B48491A6899F80000FFF74AFF3C
:10BD700030B1032333709FE7444B03221A70E0E78E
:10BD800098F800003A4980F001004FF49A7204F0EC
:10BD900091F8029800F058F90028EAD1012388F8B8
:10BDA0000030384B38491A68334B186800F0B0F946
:10BDB00020B1DEE798F80030002BF2D198F800307F
:10BDC00033B12A463946204600F0A2F90028D0D1E6
:10BDD0002E4B1B78022B43D0032B03D0012B42D0D8
:10BDE000002069E72A4B187800283FF465AF294BFB
:10BDF000186900283FF460AF00F10C025178137805
:10BE000043EA0123917843EA0143D17853EA01637D
:10BE10000BD15079137943EA0023907943EA004328
:10BE2000D07953EA006002D146E79C420CD35379A3
:10BE3000107940EA0320937940EA0340D37940EA3D
:10BE400003608442034601D91432D7E700283FF447
:10BE500033AF2C449C42C3D30223337013202BE70F
:10BE60004FF4F833F5E74FF40043F2E7BD16002036
:10BE7000CB640100BC160020B81600207C16002000
:10BE8000B4160020B016002080160020B516002041
:10BE9000B6160020A063010010B50E4B1C783CB90B
:10BEA00020460D4940F26B1204F004F8022010BD48
:10BEB00000221A70094B187808B100F0CBF9022C57
:10BEC000F5D0074B1B78032BF1D0002808BF2520A5
:10BED000EDE700BFBD160020CB640100B4160020C2
:10BEE000B51600202DE9F041DFF84480114E98F896
:10BEF0000030114F0446CBB9104B32681B68104913
:10BF00009B68386898470123054688F800303268F6
:10BF10000B48FF210AF022F93368B4FBF3F003FB6E
:10BF20001040241A3C602846BDE8F0810025EEE769
:10BF3000C01A0020D41A0020D01A0020D81A0020DD
:10BF4000C0160020F8B5384F3B685B690546984736
:10BF50003B6806469B6928469847044606B140B9A7
:10BF6000324940F23512002003F0A4FF022420469B
:10BF7000F8BDB6F5806F8CBF002001202B494FF42F
:10BF80009D7203F097FF4FF48060B0FBF6F07043B2
:10BF9000A0F5806358425841244940F23B1203F017
:10BFA00089FFA6428CBF0020012020494FF49E72D9
:10BFB00003F080FFB4FBF6F006FB1040B0FA80F00F
:10BFC00040091A491A4E40F23D1203F073FFB5FBC7
:10BFD000F4F0184B04FB10501C60174B281A186023
:10BFE0003B68164D1B6A3060B4F5806F28BF4FF474
:10BFF00080642C6033B19847044618B13B685B6895
:10C000009847B4E70E4B1B7833B13B683068DB6868
:10C01000984704460028F1D12A680A48FF210AF00F
:10C020009DF80024A3E700BFD81A0020FF64010098
:10C03000C41A0020C81A0020D01A0020D41A0020E8
:10C04000E01A0020C0160020F8B5254F3D780446C0
:10C0500035B147222349002003F02CFF02242AE0B7
:10C0600000282AD0436843B3836833B3C36823B33B
:10C07000036913B3436903B38369F3B1C369E3B1DC
:10C080004FF48062FF211848184E0AF067F8184BE9
:10C09000346001221A70174B1D70174B1D60174B2F
:10C0A0001D60174B1D60174B1D60174B1D602368EB
:10C0B0009847044618B12046F8BD4D22CAE7134BF5
:10C0C0001B784BB933681B699847054620B1336824
:10C0D0005B6898472C46EEE701233B70EBE700BF17
:10C0E000E11A0020FF640100C0160020D81A0020C9
:10C0F000C01A0020CC1A0020D01A0020D41A002028
:10C10000C41A0020C81A0020DC1A0020E01A0020FF
:10C110002DE9F74F454D95F80080B8F1010F8346A2
:10C120000E46144608D0002041497B2203F0C2FE8F
:10C13000022003B0BDE8F08F3E4F3A7852B9FFF7C6
:10C1400001FF10B102232B70F3E73B4A87F8008010
:10C15000C2F800B0DFF8E480374FD8F800003A6842
:10C16000BBFBF0F1B2FBF0FC00FB11B100FB1C20AB
:10C17000ABEB0101121A914204D05846FFF7B2FE10
:10C180000028DFD1DFF8B8A03A68DAF80000BBFB7E
:10C19000F0F1B2FBF0FC00FB11B100FB1C20ABEB9B
:10C1A0000101121A914236D1DFF89890D9F8002097
:10C1B000D8F800100A445A4504D85846FFF792FEB2
:10C1C0000028BFD16CB3204BDAF800101A680A447B
:10C1D0005A4504D85846FFF7B5FE0028B2D1D9F821
:10C1E0000000D8F80020194B0244A2EB0B02A24237
:10C1F000ABEB000028BF224631461844019209F0FB
:10C2000085FF019A1248B2FA82F1490901709344FC
:10C210001644A41ACAE75846FFF794FE0028C3D074
:10C2200090E7C7F800B0204683E700BFE11A00207E
:10C23000FF640100CC1A0020DC1A0020D41A002070
:10C24000C81A0020D01A0020C41A0020C0160020EE
:10C25000C01A002070B5194E307830B91849CC2278
:10C2600003F028FE0224204670BD012823D10020BF
:10C27000FFF738FE0546134B1B685B6898474FF481
:10C2800080620446FF21104809F068FF0F4B01222D
:10C290001A700F4A002313700E4A337013600E4A4F
:10C2A00013600E4A13600E4A13600E4A9C4208BF88
:10C2B0002C461360D7E70025DDE700BFE11A002018
:10C2C000FF640100D81A0020C0160020C01A002008
:10C2D000CC1A0020D01A0020D41A0020C41A002042
:10C2E000C81A0020DC1A002010B5044603F0F8FB41
:10C2F000014B1C7010BD00BFE01A00204FF480708D
:10C3000070474FF480507047024B1878431E5842D4
:10C3100058417047012B002008B50D4B187828B9FB
:10C320000C49832203F0C6FD022008BD00201870CE
:10C3300004F062FC50B9084B1B780BB10020F4E705
:10C3400002F026F80028F9D12520EEE71F20ECE7BF
:10C35000012B002033650100022B002038B5174D5A
:10C360002C783CB116496222002003F0A3FD022480
:10C37000204638BD22462146204604F03BFCD0B979
:10C38000104B11481C70114B1C70114B1C70114B41
:10C390001C60114B1C60114B1C70114B1C60114B2D
:10C3A0001C60114B4FF4805221461C6009F0D6FEF0
:10C3B00001232B70DCE71E24DAE700BF012B0020ED
:10C3C00033650100022B0020011B0020001B002010
:10C3D000F81A0020F41A0020FC1A0020EC1A0020A1
:10C3E000E81A0020F01A0020E41A002038B52C4D7D
:10C3F0002B78012B044606D000202A49FF2203F0A7
:10C4000059FD022038BDC0F30B0040B1254940F270
:10C410000712002003F04EFD02202870F2E7224AA6
:10C42000137853B1214B22491B6809680B449C4285
:10C4300003D01C494FF48772ECE7A4F50043B3F531
:10C44000B83F03D202232B702120DBE701231370B6
:10C45000164B1C60164B4FF48052B4F5004F1A6017
:10C4600016D201F097FF68B164B9204601F01EFEB4
:10C4700090B94FF400424FF4807101F020FE68B98A
:10C480000020BFE7204601F011FE0028F8D0D9E7D0
:10C49000232002232B70B5E71020FAE72020F8E7CD
:10C4A000012B002033650100F81A0020F41A002047
:10C4B000FC1A002070B5144D2B78012B07D00020FA
:10C4C000124940F2371203F0F5FC022070BD104E05
:10C4D000347844B100200D4940F23D1203F0EAFCEB
:10C4E00002202870F2E72046FFF780FF18B10223F0
:10C4F0002B702220EAE704F58054B4F5004FF2D106
:10C5000001233370E2E700BF012B002033650100F7
:10C51000001B00202DE9F843664D2B78012B0646C1
:10C520000C46174608D06449A222002003F0C2FC42
:10C5300002242046BDE8F883C3B21BB1AB225E499A
:10C5400000200EE0FF2A02D912F0FF0001D0B22233
:10C55000F5E7C6F30B031344B3F5805F06D9B922A0
:10C560005549022403F0A6FC2C70E2E7534B1B78DC
:10C570007BB9534B187808B9C122F1E7514B1B68BE
:10C580009E4204D3504A126813449E4201D3C722EC
:10C59000D5E74E4A137843B14D4B4E491B680968A5
:10C5A0000B449E4201D0CF22C9E7B6F5F83F07D22F
:10C5B000F319B3F5004F03D902232B702024B8E7F9
:10C5C00001231370424B1E60424BB6F5004F1F60B3
:10C5D00057D201F0DFFE002859D0C6F5FF48DFF83A
:10C5E000F89008F17C0847453A46D9F8000028BF82
:10C5F00042462146FFF782F8B6F5805FC9F8000091
:10C6000007D236483A462146304409F07FFD0024DF
:10C610008FE7F319B3F5004F39D1C6F5FF43C6F5DF
:10C62000FF427D337E32E15CA35C14F808201B04DA
:10C6300043EA01231343C6F5FF427F32A25C43EA7B
:10C64000026398421FD122463946304601F037FD39
:10C65000D8B901F02BFD90B9204A4FF4805101F078
:10C660002EFD00280CBF0024202401F081FD1C4B6E
:10C6700001221A70002CCAD002232B7059E7102413
:10C68000F3E72324F8E72724F6E72024F4E72246FB
:10C690003946304601F013FD044600288CD13E4453
:10C6A000B6F5004FB3D301F063FD0D4B01221A70B4
:10C6B0003FE700BF012B002033650100001B002075
:10C6C000F81A0020F41A0020FC1A0020EC1A0020AE
:10C6D000E81A0020F01A0020E41A0020011B0020B4
:10C6E000022B002008B525220948002109F036FD5B
:10C6F000084A00231360084A1370084A1370084A56
:10C700001370084A1370084A1380084A137008BD52
:10C71000072B0020302B00202D2B0020062B002083
:10C72000342B00202C2B0020042B0020352B002044
:10C730002DE9F74F9246964A0E9F89464518117883
:10C740009846002306463B6021B101783A2940F023
:10C75000D68013708F4B1A78C2B18F4C21460022BD
:10C760001A70404611F8042B09F0D0FC22783B687F
:10C770008A49607813443B600B68A4781B0C1B0447
:10C7800040EA04200343134490440B60824C01961A
:10C79000019EAE4200F0B380019B13F8012B019380
:10C7A0000D2AF5D03A2A1DD00A2AF1D07C497D4BBA
:10C7B00009781B78002900F0DC80D00602F00F0118
:10C7C00058BF0931E25C774801F00F011143E15491
:10C7D00022780133DBB2111D9942037040DA002345
:10C7E000184610E025220021204609F0B7FC6C4ACB
:10C7F000002313706B4A13706B4A1370C8E714F868
:10C800000CC06044C0B25FFA83FC614503F10103D0
:10C81000F5DA002840F0B880634B197801BB01219C
:10C8200019706378A17894F803B043EA01235BBAE6
:10C8300098B26370C3F30723A370BBF10D0F0FD839
:10C84000DFE80BF0142F600E7C0E0E0E0E0E070E9E
:10C850000E146279237943EA0223544A5BBA1380A7
:10C860004F4A1378B3FA83F35B09C6E74F4B1B8833
:10C870003BB14F490988994203D04E4909889942F2
:10C880003AD1DFF818B14C4BDBF800C00CEA0301D9
:10C8900001438C453F4917D001230B701E444FF0D4
:10C8A000020B0C9B3A68FF219A1A404609F056FC8D
:10C8B0003A4B3A681B68AD1B9B1A0D9AA9EB05050C
:10C8C0001360CAF8005035E0002008703B4940462C
:10C8D00009F01CFC21783A68374B0A443A60DBF8CF
:10C8E0000020A0781340627842EA002213430B44F0
:10C8F0008844CBF80030B3E7254B01221A704FF083
:10C90000000BCEE70C9B3A68FF219A1A404609F0CB
:10C9100025FC224A396813685B1A0D990B6063790C
:10C920002179AD1B1B01A9EB050543EA0133CAF8C8
:10C9300000501360584603B0BDE8F08F0C9B3A6876
:10C94000FF219A1A404609F009FC144A3968136815
:10C950005B1A0D990B6063792179AD1B1B04A9EB60
:10C96000050543EA0163CAF8005013604FF0020B5B
:10C97000E0E7242B3FF674AF02F00F01D20658BF58
:10C9800009310901E1546BE74FF0040B89E700BF5F
:10C99000352B00202C2B0020072B0020302B0020D3
:10C9A0002D2B0020062B0020342B0020042B0020F0
:10C9B000EC070020EA0700200000FFFF0B2B0020FF
:10C9C000024B0021186805F08BBF00BF602B0020D0
:10C9D000014B186805F098BF602B002008B506F0E1
:10C9E000D1FB064B06491B681B1A5842584140F2BE
:10C9F0006912BDE8084003F05DBA00BF642B002057
:10CA00009065010038B5104D104C0FCD0FC40FCDFF
:10CA10000FC495E8030084E8030000F033FB0C48E2
:10CA200001F086F901F022F90A4B18600A4B4FF425
:10CA300000721A60094B01221A60094B094A400A28
:10CA40001860094B1A6038BDC4650100382B0020FE
:10CA500059CC0000E04E0020A84E0020A44E00203B
:10CA6000A04E00206C2B00209C4E002010B50446E8
:10CA7000FFF7A6FF054B3CB11A780AB902221A70DB
:10CA8000BDE81040FFF7A4BF1C70F9E76D2D002032
:10CA900008B5FFF795FF074B1978074B1A788A42BC
:10CAA00003D1022A04BF01221A70BDE80840FFF733
:10CAB0008FBF00BF6C2D00206D2D00202DE9F843A5
:10CAC000064613380128454C454994BF00200120F3
:10CAD0004FF43A7203F0EEF994F82030032B07D1AB
:10CAE000BDE8F8433E494FF43B72002003F0E2B941
:10CAF0002368002B50D0A569E269AA424CD325B126
:10CB00006568A268AA1A5542554105F0010294F8D9
:10CB1000269084F82520002B40D194F82770033FFD
:10CB200018BF0127002D3BD094F8248094F82330BF
:10CB3000002B236908BF0025013333D060682849E2
:10CB4000013040F20A3218BF012003F0B3F96268E5
:10CB500023699B1A6269B2EB432F8CBF0123002328
:10CB600016B3032384F8203094F82030032B0CD123
:10CB700094F821303BB1FEF753FF002384F82130B5
:10CB80009E4208BF0646174B1E70B9F1000F23D115
:10CB9000BDE8F843FFF77CBF0025B6E70127C1E7F2
:10CBA000A846C3E70023DBE7B9F1000F09D033B98A
:10CBB000002FD6D0B8F1000F08BF0426D1E7062613
:10CBC000CFE7002DCDD1B8F1000F01D00223C9E786
:10CBD000002FC9D00123C5E7BDE8F883382B00201A
:10CBE00090650100362B002030B4194C94F8205089
:10CBF000032D06D130BC174940F23522002003F046
:10CC000059B9256805B92060A068013094F827005B
:10CC100008BFA1600328A06908BF84F827309042AC
:10CC200007D9E069904204D91AB1032030BCFFF75C
:10CC300045BF481C02D0A0688842F6D1032B03D020
:10CC400094F827109942F0D1A2610020EEE700BFCE
:10CC5000382B0020906501002DE9F041354C1D4630
:10CC600007468846164600F08FFA94F82030032BCA
:10CC70001FD0B8F1020F16D1D4F80080B04518D1FA
:10CC8000284601F047F80646284601F01FF80446FA
:10CC90003846FEF741FE3246034621464046BDE88F
:10CCA000F041FFF7A1BFB8F1000F04D0B8F1010FB8
:10CCB0001BD0BDE8F0813846FEF72EFE0328F8D0E1
:10CCC000284601F032F88307F3D43846FEF724FEF5
:10CCD0000746284601F01EF80446284600F0F6FFF5
:10CCE0003B46014622463046D9E72368B342E0D1AD
:10CCF00094F8223033B100234FF0FF322360A2605A
:10CD0000A361D6E70C4D0FCD0FC40FCD0FC495E82E
:10CD1000030084E80300FFF753FE084B1A78012A4A
:10CD200004D1074A1278022A08BF1A70BDE8F04100
:10CD3000FFF74EBE382B0020C46501006D2D00208A
:10CD40006C2D0020F8B5414E414C0546FFF746FEDC
:10CD5000FFF736FE327823789A4203D1BDE8F840D7
:10CD6000FFF736BE3B4940F2F912012003F0A2F86A
:10CD70003378022B11D1384B93F82030012B55D04A
:10CD800008D9023B012B05D9324940F20B22002081
:10CD900003F090F84FF4FA7304E0002B37D12278B7
:10CDA000022A3BD12D4A11684EF65F20814203D8FA
:10CDB0000D4499421560D1D9257837783570012D09
:10CDC00008BF02234FF0000608BF23701660FFF76C
:10CDD000FFFD022F16D1204C94F82030032B05D0F4
:10CDE0000123304684F82630FFF768FE94F82000CF
:10CDF0001849C31E584240F21112584103F05AF824
:10CE000000F064FA012D17D9022D19D0F8BD012BBD
:10CE100004D12378022B0CD0002BC3D00D4940F253
:10CE20001B22002003F046F80023BBE744F62063F2
:10CE3000B8E740F6C413B5E7094B00221A60E5E7EE
:10CE4000FFF7E0FD064B0122F8E700BF6C2D002044
:10CE50006D2D002090650100382B0020682B0020EC
:10CE6000D84E002008B5FFF7B9FD014B187808BD72
:10CE7000362B002008B506F085F9094B1860002014
:10CE800005F01CFD074B1860FFF7BCFD064A0023A8
:10CE90001370064A1370064A1360064A136008BDF1
:10CEA000642B0020602B00206C2D00206D2D0020B5
:10CEB000682B0020D84E002070B504460D4616465B
:10CEC000FFF78CFD064B1B684BB1012001F0E0FB26
:10CED000324629462046BDE8704000F02FBF70BDA5
:10CEE000D84E00202DE9F041054688461646FFF74A
:10CEF00075FD534B1B68CBB1524B534C00221A604B
:10CF000094F82030032B11D0012001F0C1FB3246F0
:10CF10004146284600F03EFF94F82030032B05D010
:10CF200094F8223023B163689D423ED2BDE8F0817F
:10CF300071024046FEF7DCFC0328074620D094F837
:10CF40002100424940F2852280F0010002F0B2FF48
:10CF5000681C18BF01203D4940F2862202F0AAFF5A
:10CF60006368013394F8273008BF6560032B63685A
:10CF700008BF84F827709D4207D00320FFF79EFD6D
:10CF800094F82230002BD1D0CDE794F82730BB4263
:10CF9000F3D13846FEF7D8FC0028EFD10123E56035
:10CFA00084F8213084F82230E8E7E3689D420AD013
:10CFB000BCD22369013308BF25612369AB4294BF0A
:10CFC00023612561B2E7E369354403EB4623770229
:10CFD00094F82360E361E56026B10020BDE8F041EC
:10CFE000FFF76CBD19494FF43172012002F062FF66
:10CFF000164994F8210040F2C52202F05BFF394641
:10D000004046FEF7D7FC1328054610D1FEF708FD71
:10D010000123054684F8216084F8233084F8243005
:10D02000FBF720FF63693B4463612846D6E7142879
:10D0300003BF012384F82430354684F82460F1E7E7
:10D04000D84E0020682B0020382B0020906501006E
:10D0500000220346114610461847000070B50646E8
:10D0600007480D46FBF792FA04462DB136B9024641
:10D070000349284609F04AF8204670BD0024FBE722
:10D08000EC65010037B5304C304A23464FF08061E3
:10D0900013F81F0F002814BF1846104600F0FCFCC0
:10D0A0002B48FFF7D5FF14F8145F29490346294898
:10D0B0000022954218BF204600F030FF2648FFF7B7
:10D0C000C7FF254903460022244800F027FFFFF749
:10D0D000C9FE40B12248FFF7BBFF214903460022A9
:10D0E000204800F01BFF204B204A2148412102F03C
:10D0F00085FC58B11F48FFF7ABFF1E4903460022CD
:10D100001D4800F00BFF002100F0DEFD002300931E
:10D110004FF40043019301F03DF980B1009801996B
:10D120004FF4807208F0E2FF044640B91348FFF75D
:10D130008FFF124903462246114800F0EFFEFBF72D
:10D14000B3FE03B030BD00BFA0630100586601000C
:10D1500069D4000064660100DDD70000706601003C
:10D160002DD500007C660100B22D0020B02D0020DE
:10D170006E2D002065D60000C46A01005DD000005D
:10D180008866010000207047F7B507460C46FFF798
:10D19000F9FF20B903F0B8FD18B1022C0AD103B091
:10D1A000F0BD03F0B3FD0028F7D102F043FD0028E5
:10D1B000F3D1F4E7002C6FD101230DF107013846BC
:10D1C0008DF80730FBF764FE10BB3C4E4FF0FF3587
:10D1D00031680B22384608F089FF00B935790134EF
:10D1E000102C06F10806F3D16B1C1DD00F2D4CD866
:10D1F000DFE805F008150E1E272B2D313337393D9A
:10D200003F43454901F0C6F810B1012002F0A6FBEA
:10D210009DF80730002BC2D0FFF73AFCBFE7284942
:10D22000E222002002F046FE00238DF80730EFE7EF
:10D23000244B1C682368984723699847636898477C
:10D24000E6E7012002F0D6FCE2E70020FAE7012041
:10D2500002F0D6FCDCE70020FAE7012002F0D6FC61
:10D26000D6E70020FAE7002002F02EFCD0E70120EC
:10D27000FAE7012002F0D0FCCAE70020FAE701201B
:10D2800002F02EFCC4E70020FAE70D494FF4887243
:10D29000002002F00FFEBBE7012C80D10A490B22CF
:10D2A000384608F023FF00287FF479AF02F01EFE15
:10D2B00003B0BDE8F040FFF7EBBB00BFE46A01003C
:10D2C0009466010048770100C46A010008B501F0C6
:10D2D0005FF820B1FFF7C6FD08B9FEF7CFF901F0FE
:10D2E00059F820B102F082FB30B1FEF7C7F9054AC8
:10D2F00013680133136008BD02F0ECFB0128F6D17E
:10D30000F3E700BFB42D00202DE9F04FA5B004AE27
:10D310002E9C0746884691460021802230469A4638
:10D3200008F01CFF631E31467E3413F8012F1AB13A
:10D330009C4201F8012BF8D1DFF81CB135462B785F
:10D34000402B0ED05BB9AD1B0195009653464A4663
:10D350004146384602F079FD25B0BDE8F08F013531
:10D36000EDE76B78562B33D8412B01D83B4C37E097
:10D37000423B142BFAD801A252F823F025D4000026
:10D380006DD3000037D400006DD300006DD30000D2
:10D390006DD300002BD400006DD300006DD30000CE
:10D3A0006DD300006DD30000DBD300006DD300000F
:10D3B0006DD300006DD300006DD3000043D4000096
:10D3C0006DD3000031D400001FD400003DD4000014
:10D3D000623BDAB2142ACCD9C8E700F09FFE0446BB
:10D3E0002846FBF7D3F803902046FBF7CFF8039AC3
:10D3F000111802390346294424A8884229D9023A3F
:10D40000A91CE818039308F08FFE039B21461A46D7
:10D41000284608F07BFE2B78002B90D193E700F094
:10D4200065FEDCE700F066FED9E700F067FED6E7B0
:10D4300000F068FED3E700F069FED0E700F06AFE76
:10D44000CDE79BF82A30064C064A002B08BF14464D
:10D45000C6E7154477E700BFA0630100C36601007B
:10D46000CA630100C9660100F7B50F4600B1F1B902
:10D47000450256020F4B00932A4600233146384698
:10D4800002F001FD0C4B0093044603462A46314648
:10D490003846FFF739FF094B0093044423462A46D8
:10D4A0003146384602F0EFFC204403B0F0BD0020C6
:10D4B000FBE700BF02670100D2670100D5670100EA
:10D4C0002DE9F7430A9C0094984605460E461746F8
:10D4D00002F0D9FC4FF00209124B00933A4608EBD8
:10D4E000000331460446CDF80490284602F0ADFC16
:10D4F0000B9B0093044408EB04033A46314628464C
:10D5000002F0C1FC084B00930444CDF8049008EBF2
:10D5100004033A463146284602F097FC204403B003
:10D52000BDE8F08302680100926801002DE9F74F21
:10D530000D4692460446FFF795FC064600F09AFD1C
:10D540000746304600F0AAFD06460CB1002D4BD12F
:10D550004FEA442B254B01974FEA4A2A00935A463B
:10D56000002351462846FFF7ABFF214B00930446AA
:10D5700003465A465146284602F085FC1D4F044496
:10D5800007F114094FF001086EB9022301931A4BF9
:10D5900000935A4623465146284602F056FC204442
:10D5A00003B0BDE8F08F4F45EFD0B8F1000F0AD1BE
:10D5B00002230193114B00935A46234651462846B5
:10D5C00002F043FC0444F3070AD53B6800935A4633
:10D5D00023465146284602F056FC4FF0000804440A
:10D5E000C6F347060437CFE70020D9E7F867010004
:10D5F000FE670100D06A0100926801000568010021
:10D6000070B4049E044D054C002E08BF2C460494B3
:10D6100070BCFFF755BF00BF08680100C979010061
:10D620002DE9F04186B00DF10C0804460D46404648
:10D630000D991F46164602F0CEFB00F118030DEBC4
:10D640000300002300F80C3C0C9B0093CDF80480F1
:10D650003B46324629462046FFF732FF06B0BDE87A
:10D66000F08100002DE9F04F87B000230E460293B1
:10D6700008B1002975D13C4B1B78012B6ED0022BD1
:10D680003A4B14BF4FF00008984644025502384BFD
:10D690000093224600232946304602F0F4FB354B26
:10D6A0000193354B009307460346224629463046F0
:10D6B000FFF706FF314B1B8801930744304B009363
:10D6C00022463B4629463046FFF7AAFF07EB000AF1
:10D6D000B8F1000F0AD02B4A00925346CDF80480CF
:10D6E000224629463046FFF7EBFE824402A802F0AC
:10D6F000E1F9804670B3029A62B3234A009253461E
:10D7000022462946304602F0BEFBDFF880B0824454
:10D7100000270DF10C090AF10A02B2F5007F19D2B7
:10D720000A225946484608F0F1FC029A484652F847
:10D73000271002F037FB0A23019322465346CDF807
:10D7400000902946304602F080FB0137FAB290453E
:10D750008244E0D8504607B0BDE8F08FDFF8308053
:10D7600093E79A46F6E700BFB22D00201568010046
:10D77000216801006E2D00202A680100B02D0020D4
:10D780002F680100346801003B680100CC61010092
:10D790000A6801002DE9F04186B0002405460E46D6
:10D7A00098460D99049447F630030DF10E00174684
:10D7B0000393ADF814408DF8164002F0F3FA03AB72
:10D7C00001930C9B00933A464346314628468DF818
:10D7D0001640FFF775FE06B0BDE8F0812DE9F04375
:10D7E00085B00D4656024702644B00933A4600232B
:10D7F0003146284602F047FB614B0093044603463E
:10D800003A4631462846FFF77FFD5E4B00930444BD
:10D8100023463A4631462846FFF776FD044402F097
:10D8200001FA594B01903A46314600932846234667
:10D83000FFF7E6FE044402F0FDF9544B01903A462E
:10D840003146009328462346FFF7DAFE044402F0EF
:10D85000F9F94F4B01903A4631460093284623464A
:10D86000FFF7CEFE044402F0F5F94A4B01903A4628
:10D870003146009328462346FFF7C2FE044402F0D7
:10D8800035F9454B019000933A46234631462846E8
:10D89000FFF7B6FE414B0093044423463A46314617
:10D8A000284602F0F0FA3E4B0093044423463A46E1
:10D8B00031462846FFF728FD044400F037FC08B342
:10D8C0000DF108084FF0060936494A46404608F06F
:10D8D0001DFC354B00933A4623463146284602F05C
:10D8E000D2FA044400F04CFD04220146404602F006
:10D8F00096FA2346CDE900893A463146284602F099
:10D90000A4FA0444294B00933A462346314628465C
:10D9100002F0B9FA044400F009FC58B100F01CFC14
:10D92000234B019000933A46234631462846FFF7A1
:10D9300031FF044400F016FC1E4B019000933A4660
:10D94000234631462846FFF725FF1B4B1B680193F2
:10D9500004441A4B00933A46234631462846FFF7C3
:10D960005FFE174B0093044423463A46314628464F
:10D97000FFF7CAFC204405B0BDE8F083466801000B
:10D9800095680100A5680100B2680100BD6801004A
:10D99000D0680100E3680100006901000D69010021
:10D9A00027690100D66101003F6901005469010047
:10D9B000BE690100CD690100B42D0020DB690100C2
:10D9C000E96901007047704710B5540208462246C5
:10D9D000002108F0C3FB204610BD000008B5034637
:10D9E00008463BB904494FF4007208F08FFB4FF42E
:10D9F000007008BD0020FCE7C031002008B50346D8
:10DA000008463BB904494FF4007208F07FFB4FF41D
:10DA1000007008BD0020FCE7C933002083185B02BA
:10DA2000B3F5806F70B506460D46144607D9002041
:10DA30000B4940F2632202F03DFA002070BD4FF422
:10DA400000720021284608F089FB36B9054B0649CB
:10DA50001A682846520108F059FB6002EEE700BF41
:10DA6000646B0100BC310020BC2D00204300013359
:10DA7000B3F5007F05D3064940F23912002002F0C9
:10DA800019BA044A02F81010090AD154704700BFAD
:10DA9000646B0100C03100202DE9F84FDFF8909150
:10DAA000644D654CDFF89481654F8A464FF40072EF
:10DAB0000021064648464FF0000B08F04FFB4FF49C
:10DAC000007200215F4808F049FBC02259465E48B9
:10DAD000C5F800B008F042FB4FF4806259465B483D
:10DAE00008F03CFB5A4B5B4A83F800B05A4B5B4949
:10DAF0001A6048464FF40072C4F800B0C8F800B08D
:10DB0000C7F800B008F002FB99F80C3099F80B2028
:10DB10000AF5803A42EA0322BAFBF2F399F80D20A3
:10DB200041F25A0A0AFB02F199426AD94FF4AB72E8
:10DB30004B49584602F0BEF999F80D300AFB03F341
:10DB4000B3F5803F4FF0000264D389F8132089F8C1
:10DB50001420C3F3072289F82120C3F3074289F870
:10DB6000222089F820301A0E89F8232099F80D20F8
:10DB7000B3FBF2F35B00DFF8D0A03A4903F2FF13E6
:10DB8000C3F3472289F81620C3F347433022504697
:10DB900089F8173008F0BAFA99F8172099F8163072
:10DBA00043EA02230422C8F80020DAF808205B02C6
:10DBB000CAF81430CAF8203002EB4302DAF82C30ED
:10DBC0001A44204B3A60F8221A70FF225A70012042
:10DBD0004FF6FF712860FFF749FF2B6822491B4869
:10DBE00001332B6020220023236008F08FFA1748AE
:10DBF0000B22314608F08AFA236801332360BDE81E
:10DC0000F88F4FF6917A0AFB02F29A4298D240F2CC
:10DC100059128DE7C3F3072189F8133089F81410DE
:10DC200089F8202089F8212089F822209CE700BF6C
:10DC3000C9330020C0330020BC3100208C360020C6
:10DC4000B82D0020C0310020CC350020BC2D002094
:10DC5000C8330020C7D90000C4330020C66B0100C0
:10DC6000646B0100E86D0100C66D010010B5144B36
:10DC7000DC7C187D54EA002006D0DC7A1B7B44EA69
:10DC800003244443204610BD93F8210093F820401C
:10DC900044EA002493F8220044EA004493F8230065
:10DCA00054EA006405D0DA7A1B7B42EA03235C4322
:10DCB000E8E7044940F28912204602F0FBF8E1E768
:10DCC000C9330020646B0100C1727047427F037F3B
:10DCD00043EA0223827F43EA0243C27F53EA02639C
:10DCE00011D0837EC07E094A43EA0020517B831E07
:10DCF000D07A127B40EA022205480068B0FBF2F0BD
:10DD000001FB030070474FF0FF307047C93300201C
:10DD1000B82D0020427F037F43EA0223827FC07F29
:10DD200043EA024343EA00607047C07A704700004C
:10DD3000014B1860704700BFC43300202DE9F04745
:10DD4000894604461546002152024846104E08F006
:10DD500005FA06F1C00A00273846B368844207EB8B
:10DD600053270ED3A7420CD9A7EB0408A84528BF18
:10DD7000A846201A33684246494698474444A5EBD2
:10DD8000080515B10C365645E6D1BDE8F08700BF51
:10DD9000CC3500202DE9F74F4FF00008DFF8589000
:10DDA000DFF858A00446154640464FF00C0BD9F852
:10DDB00000205FFA88F39A4202D803B0BDE8F08FE2
:10DDC0000BFB03A384429E6800EB56260DD3B4429E
:10DDD0000BD2371BAF4228BF2F46201A5B68019138
:10DDE0003A46984701993C44ED1B08F10108002D83
:10DDF000E3D03046DBE700BF8C360020CC35002076
:10DE0000F0B503460078E52885B011D088B1202808
:10DE10000ED0114F5E1E03F10A0416F8015F1022A6
:10DE20003946684608F072F9A5F16103192B02D84A
:10DE3000002005B0F0BD1F2D01D8052DF8D16A4690
:10DE4000002312F8011B8D42F2D00133102BF8D1C0
:10DE5000B442E2D10120ECE7956B010083185B022C
:10DE6000B3F5806F2DE9F74F884608D928494FF45C
:10DE70001F72002003B0BDE8F04F02F01BB8254B25
:10DE8000DFF89490B0FA80F46409560203EB402A5C
:10DE9000770901EB441B0AEB4415BC4207D3324619
:10DEA0004146504603B0BDE8F04F08F02FB920229C
:10DEB0005946284608F01AF9B8B10B2259462846A7
:10DEC00008F014F92A460190D9F800C05B460221F7
:10DED0005846E0479BF80020E52A0BD15B462A46CE
:10DEE00001212846D9F800C0E04701340BF1200B8E
:10DEF0002035D2E7019B002BF7D05846FFF780FF73
:10DF00000028F2D05B462A4600215846EAE700BFC7
:10DF1000646B0100BC2D0020C43300202DE9F74FB5
:10DF2000DFF824811C468A4691468346FFF768FF46
:10DF300040F29512454901F0BDFF98F80C2098F881
:10DF40000B7047EA022798F80D207A43531E2344AA
:10DF5000B3FBF2F74CB33E4D2E6800237A1E9A4273
:10DF6000286815D84FF6FF71FFF780FD2B68013345
:10DF70002B60384A13681F2B19D94FF4D5723349D7
:10DF8000002001F097FF0025284603B0BDE8F08F80
:10DF9000411C89B201920093FFF768FD2968009B3C
:10DFA000019A013129600133D9E72646E1E72A4D7C
:10DFB0002A4905EB4315013313602846202208F057
:10DFC000A5F80B225946284608F0A0F8C6F30741E9
:10DFD00023482975310E697501682C77C4F307222F
:10DFE0006A77AE76C4F30742C6F30726240E0F29DC
:10DFF000AA77EC77EE7602D94FF4DC72BFE7194BC3
:10E00000194E1A4A0C244C4303EB040CBAF1000FCE
:10E0100018BF5646B9F1000F1E5118BF4A46CCF83A
:10E02000042098F80C4098F80B30114A43EA042376
:10E0300098F80D4063437B43CCF8083013780131E6
:10E040000133016013709FE7C9330020646B010046
:10E05000C0330020BC310020BC2D0020A66B010085
:10E060008C360020CC350020C9D90000C5D900006D
:10E07000C8330020272808B503D8054B53F82000E3
:10E0800028B900200349F72201F014FF024808BD17
:10E09000AC750100186E01009468010027289ABF32
:10E0A000014B185C012070474C76010010B5EFF36E
:10E0B000108472B602F0A2FD84F3108810BD10B572
:10E0C000EFF3108472B602F0A9FD84F3108810BD3E
:10E0D000B0F5003F07D201390844B0F5003F2CBF2E
:10E0E0000020012070470020704700000048704762
:10E0F0000E37002000487047AC36002000487047BB
:10E10000BF36002000487047ED36002000487047B9
:10E11000B6360020004870473F370020004870475F
:10E12000E0360020004870475437002008B50C2125
:10E130002020FFF7CDFF48B10020054B026A9A422C
:10E1400004D1406A034BC31A5842584108BD00BF6E
:10E15000939D939B2028056E014B1868704700BF64
:10E1600090360020014B1868704700BF9836002099
:10E17000F8B50024164F174E174D3C6047F6FC715A
:10E18000204634602C60FFF7A3FF28B147F6FC71EE
:10E190002046FDF785FA386010494FF40040FFF73C
:10E1A00097FF28B10D494FF40040FDF779FA306030
:10E1B0004FF480514FF4F830FFF78AFF30B14FF43D
:10E1C00080514FF4F830FDF76BFA2860F8BD00BFBE
:10E1D000903600209836002094360020FC6F010015
:10E1E0002DE9F041FFF7C4FF5A48DFF868815A4F24
:10E1F00003F03AF805F0A2F9052200210446574839
:10E2000007F0ACFF21220021534807F0A7FF21228D
:10E210000021534807F0A2FF09220021514807F0CE
:10E220009DFF4E480522002107F098FF0425002697
:10E23000B81958F8041B01F0B5FD013D064415F06E
:10E24000FF05F6B2F4D1BD55DFF81C81444F04261A
:10E25000781958F8041B01F0A5FD013E054416F09D
:10E26000FF06EDB2F4D17E553E4D4049284601F0FF
:10E2700099FDC0B22E5405F02FF9384D0146042205
:10E28000284607F043FFC4F30F32092AC4F30733CB
:10E290002E7188BF5733364E98BF3033DBB23370A0
:10E2A000C4F30323092B8CBF57333033737001F051
:10E2B00011FC0128C4F3031540D145F008052D4B8E
:10E2C0002D4804F00F04092D4FF030021A708CBF56
:10E2D000573530353222092C8CBF573430345A70C0
:10E2E00035229A70F47037220024DA701C713122C2
:10E2F000B5702146347107F031FF18491E4807F008
:10E3000035FF1B491C4807F031FF13491A4807F035
:10E310002DFF1449184807F029FF1748FAF736F976
:10E32000C0B2164B421C52001A7003225A70124A95
:10E330002546E1B2884206D8BDE8F08105F022F911
:10E340000028BAD0BBE712F8011B9970DD700134C8
:10E350000233EEE79C360020BF360020AC360020AA
:10E36000ED360020B6360020443700202028056E08
:10E37000B13600203F3700200E37002054370020F0
:10E3800008B5FFF7D3FE08B10023986A08BD7047AF
:10E39000002070470120704710B50A4C0221206808
:10E3A00004F004FF084A1368591C1160074A5343DC
:10E3B000B3F1553F05D820680121BDE8104004F0B5
:10E3C000F5BE10BDC0370020BC370020ABAAAAAAFA
:10E3D000704770472DE9F84F01F052FA02F038FC0F
:10E3E000012002F075FC8F4C012002F089FC012015
:10E3F00002F088FCFCF7E4FA20888B49461E704244
:10E400004FF49572704101F055FDE36E03B19847EA
:10E4100005F0C8F8854B1B6813B1DB6803B198475A
:10E42000E468A50702D5012000F098F9E40702D5B9
:10E430000120FDF759FFFFF7D3FEFFF7A8FF07F014
:10E4400091F901F047FBB0FA80F04009FEF70EFBAE
:10E4500001240020764EDFF8DCB107F091F9764B0D
:10E46000764834700022214604F0C2FF032104F0F4
:10E47000D3FF16254FF00B0AA046A1464FF0FF32FE
:10E48000002140F63F2004F0C1FE87B2800507D589
:10E490006B4B1B7813B1012003F04AFC03F0A2FB85
:10E4A000790702D5022005F09DF8FA0613D503205E
:10E4B00005F098F8002002F03DFC002007F060F91C
:10E4C000002002F005FC002002F01AFC002002F0FF
:10E4D00019FCFAF7B3FCBB0602D5032005F082F85D
:10E4E000380501D501F01FFC390701D5FAF784FE84
:10E4F000FA0711D55A20FEF725FC3378052B0BD8E7
:10E50000DFE803F0462546340A030020307002F0AD
:10E5100011FC002007F034F9BB07AFD5FAF70EFB6A
:10E52000FAF768FB474B1B78002B43D0464A137819
:10E53000591E012935D8B9F1000F36D1012B03D16D
:10E5400040480021017011704FF001092FE0BAF12D
:10E55000000F02D0BAF1010ADED1012007F010F954
:10E560000323337016254FF0000AD5E707F02AF988
:10E5700028B1012002F0DEFB02233370CCE70DB19D
:10E58000013DC9D10120002502F0D4FB3570C3E75D
:10E5900007F018F90028EFD1307016254FF00B0A5C
:10E5A000BAE7284A00231370CEE74FF00009484627
:10E5B00002F08EFB9BF80030ABB1244A1378591E51
:10E5C000012908D85CB9012B03D100218BF8001078
:10E5D0001170012404E000238BF80030F9E70024D7
:10E5E000204602F08FFB1A4B1A78002A3FF446AF00
:10E5F00018490A78501E01280AD8B8F1000F0AD12C
:10E60000012A02D10020187008704FF0010804E0C0
:10E6100000221A70F9E74FF00008404602F070FB44
:10E620002CE700BFA06301007F760100CC490020E9
:10E630008C3B0020C4370020E076010099E3000005
:10E640008D3B0020B937002031080020320800201F
:10E65000B837002030080020024B0421186804F06D
:10E66000A5BD00BFC0370020024B01221A70024B2B
:10E6700018707047B937002031080020024B012282
:10E680001A70024B18707047B8370020300800200D
:10E69000024B01221A70024B18707047C4370020D9
:10E6A00032080020024B1021186804F07FBD00BF23
:10E6B000C0370020024B0821186804F077BD00BF66
:10E6C000C0370020024B4FF40061186804F06EBDA3
:10E6D000C0370020014B1870704700BF8D3B0020F1
:10E6E000024B4FF40071186804F060BDC037002081
:10E6F00008B5094B4FF400429A6002F0C1FD03F0E7
:10E7000031FC064A0648002104F02AFD054B18603A
:10E7100003F03CFCFEE700BF00ED00E0BC7601002A
:10E72000D5E30000C037002007B5FF23694633203A
:10E730008DF800308DF801308DF802308DF80330FF
:10E740008DF804308DF805308DF806308DF80730DF
:10E75000FCF740FA012003B05DF804FB014B187090
:10E76000704700BF983B002010B50023DCB2A242E6
:10E7700000D810BDDC0021FA04F4C4540133F5E7DD
:10E7800070B505460E46642431462846FCF7E2FB88
:10E79000022803D1013C14F0FF04F5D170BD13B57C
:10E7A00004220C4601466846FFF7DEFF01460520BD
:10E7B000FFF7E6FF012810D101A90F20FFF7E0FFC6
:10E7C00001280AD101A90E20FFF7DAFF019B23607F
:10E7D000431E5842584102B010BD0020FBE713B55C
:10E7E00004220C4601460DEB0200FFF7BDFF014677
:10E7F0000520FFF7C5FF012802D0002002B010BDA0
:10E8000004220DEB02002146FFF7AEFF01460D206A
:10E81000FFF7B6FF0128F0D100210E20FFF7B0FF6F
:10E82000431E58425841E9E7014B1860704700BF4A
:10E830003408002008B5FCF7C3F84FF0A0430322CA
:10E84000C3F8042701200222C3F80825C3F80007F3
:10E85000C3F8080508BD4FF0A0430222C3F8002703
:10E860000120C3F80427704713B500F00C000C46D4
:10E8700040F0020001A9FFF783FF019B2360431EC4
:10E880005842584102B010BD082837B505460C461D
:10E8900003D10E4B1B688B4215D004220DEB0200F6
:10E8A0002146FFF761FF014605F00C00FFF768FF06
:10E8B000012803D1082D04BF044B1C60431E58429D
:10E8C000584103B030BD0120FBE700BF903B002062
:10E8D00008B51E210020FFF7D7FF003818BF012020
:10E8E00008BD37B504460D4604F0B4FE08B904F07F
:10E8F0007F4004F0F00101430820FFF7C5FF80B11D
:10E9000004F00C0444F0030401A92046FFF738FF8B
:10E9100001A92046FFF734FF019B2B60431E58429C
:10E92000584103B030BD000037B504460D4604F031
:10E9300091FE08B904F07F4004F0F0010143082083
:10E94000FFF7A2FFD8B124B9104B5A68AA421AD0D7
:10E950005D6004220DEB0200294604F00C04FFF771
:10E9600003FF014644F00100FFF70AFF012808D128
:10E9700000210E20FFF704FF431E5842584103B008
:10E9800030BD0020FBE70120F9E700BF903B0020ED
:10E9900038B504460D4600200549FFF7C5FF30B1E4
:10E9A00029462046FFF7FBFE003818BF012038BD7E
:10E9B0005200002338B504460D4600200549FFF7F4
:10E9C000B3FF30B129462046FFF709FF003818BFD2
:10E9D000012038BD5200002337B504460D46002003
:10E9E0000949FFF7A1FF60B101A92046FFF7D7FE53
:10E9F00038B1019BE40004F0180423FA04F42C70ED
:10EA0000012003B030BD00BF5000002338B50446DC
:10EA10000D4600200749FFF787FF50B1E30003F0E0
:10EA2000180305FA03F12046FFF7D9FE003818BF96
:10EA3000012038BD500000232DE9F74F14468E18F1
:10EA400000EB0209A6EB0408A9EB040564B9012058
:10EA500003B0BDE8F08F41462846FFF7BDFF08B977
:10EA60000020F5E7013CEDE715F00307F3D1DFF8EF
:10EA700098A0032C0BD8BC4208EB070105EB07005C
:10EA8000E5D0FFF7A9FF01370028F4D1E8E7C5F387
:10EA90000906C6F58066B44251464FF0000038BF03
:10EAA00024F00306FFF740FF0028D9D004220DEB25
:10EAB00002002946FFF758FE01460520FFF760FED9
:10EAC0000128CDD100210F20FFF75AFE0128C7D120
:10EAD0004FEA96094FF0000B09F1FF39CB4508EBDF
:10EAE0008B0108D30E20FFF74BFE0128B8D1354427
:10EAF000B044A41BBDE70F20FFF742FE0128AFD1B1
:10EB00000BF1010BEAE700BF520000232DE9F347A8
:10EB100015460F46A0EB01083C4608EB07066DB909
:10EB2000012002B0BDE8F087217830460137FFF7B9
:10EB30006DFF08B90020F4E7013DEDE7B307F3D11D
:10EB4000DFF888A0032D0CD82544361BA54206EB20
:10EB50000400E5D014F8011BFFF758FF0028F5D199
:10EB6000E8E7C6F30907C7F58067BD4251464FF095
:10EB7000000038BF25F00307FFF7D6FE0028D9D0E4
:10EB800004220DEB02003146FFF7EEFD01460520A1
:10EB9000FFF7F6FD0128CDD127F00309A144A046D7
:10EBA000C84509D100210E20FFF7EAFD0128C1D197
:10EBB0003E443C44ED1BC5E741460D20FFF7E0FD18
:10EBC0000128B7D108F10408EAE700BF520000238A
:10EBD00070B50C4601460D48FFF7ECFE58B10C4EDF
:10EBE000642521463046FFF7D3FE20B12368DB03BE
:10EBF00003D4013DF5D1002070BD06482146FFF742
:10EC0000C7FE003818BF0120F6E700BFF4ED00E0B2
:10EC1000F0ED00E0F8ED00E037B504460D48019155
:10EC2000FFF7C8FE88B10C4844F48031FFF7C2FEFC
:10EC300058B10A4D642401A92846FFF7A9FE20B166
:10EC4000019BDB0304D4013CF5D1002003B030BDAF
:10EC50000120FBE7F8ED00E0F4ED00E0F0ED00E06E
:10EC60002DE9F04192B0044688461746002124223F
:10EC700005A81E4607F072FA189B0393199B01978B
:10EC80000296049362792379257843EA0223A279D4
:10EC900043EA0243E27943EA02630A93627A237AFF
:10ECA00043EA0223A27A43EA0243E27ACDF84080A3
:10ECB00043EA02630E93637845EA0325A378E47878
:10ECC00045EA034545EA04644FF0807300210820BB
:10ECD0000F941193FFF7D8FD08B9002060E001AD53
:10ECE0000024A84655F8041B2046FFF795FF00288E
:10ECF000F3D00134042CF5D10A990920FFF78CFFD9
:10ED00000028EAD00D2458F824102046FFF784FF8D
:10ED10000028E2D00134102CF5D111992046FFF7DC
:10ED20007BFF0028D9D020492048FFF743FE002868
:10ED3000D3D01F491D48FFF73DFE0028CDD06946BE
:10ED40000420FFF791FD0028C7D0009B13F0A00F0F
:10ED5000C3D1184C154D69462846FFF719FE002807
:10ED6000BBD0009B9A0306D4013CF4D1B5E7B0FABE
:10ED700080F0400914E041460020FFF729FF0028F9
:10ED8000ABD00D490948FFF715FE0028A5D09DF826
:10ED900068300198012BEAD13E44331A5842584159
:10EDA00012B0BDE8F08100BF0B005FA0F0ED00E005
:10EDB00009005FA040420F0003005FA013B5FFF7FA
:10EDC000B3FC10B9002002B010BD9E238DF80430B2
:10EDD00001A9E72310208DF80530FBF7FBFEFFF7B4
:10EDE000A3FC0028EED00024694608208DF80040DE
:10EDF000FBF7F0FE01A92046FFF736FD012818BFFA
:10EE00002046E0E7F7B5002301932F4B2F4E304FFC
:10EE10004FF0FF321A605A600424FFF70BFD33688D
:10EE200013B19B6803B19847FFF7C8FF30B9013CA5
:10EE300014F0FF0423D1204603B0F0BDFFF748FDD6
:10EE40000028F4D000210820FFF71EFD0028EED096
:10EE50004FF0A0410420FFF717FD0028E7D06425FC
:10EE600001A90420FFF700FD0028E0D0019B03F07A
:10EE70002043B3F1204F13D0013DF1D1D7E7012159
:10EE80000020FFF701FD012004F0DAFB022002F070
:10EE90004FFF002004F0D4FB022002F049FFBCE742
:10EEA00039460420FFF7F0FC0028C0D0336813B1C6
:10EEB0001B6903B1984700210820FFF7E5FC0028F3
:10EEC000B5D00124B7E700BF903B0020CC4900201B
:10EED000000F0050062837B5044600F09F80FFF76A
:10EEE000A9FC072C21D8DFE804F0041D096A6D8411
:10EEF0002007012004F0A4FB01205EE0012004F0C3
:10EF00009FFB022002F014FF002004F099FB022076
:10EF100002F00EFF4FF0A0430222C3F80027C3F80F
:10EF20000427E9E7FFF76EFF08B9002045E03F4DF1
:10EF30002878012804D104F083FB022002F0F8FEB7
:10EF40003B493C48FFF736FD044688B9012004F0F0
:10EF500077FB022002F0ECFE204604F071FB022059
:10EF600002F0E6FE32493348FFF724FD0028DCD0EA
:10EF700031480121FFF71EFD0028D6D02B782BB990
:10EF8000012004F05DFB022002F0D2FE002004F01C
:10EF900057FB022002F0CCFE264C01A92046FFF7C9
:10EFA000F7FC0028C1D0019B9A03F6D52248002126
:10EFB000FFF700FD003818BF012003B030BD1F4926
:10EFC0001C48F5E7FFF7FAFE0028AED0FFF780FCFB
:10EFD0000028AAD000210820FFF756FC0028A4D062
:10EFE0004FF0A0410420FFF74FFC00289DD01049AE
:10EFF000E6E7FFF707FF002897D011490D48FFF714
:10F00000D9FC002891D00B4C01A92046FFF7C0FC89
:10F0100000288AD0019B9B03F6D56DE70749054878
:10F02000FFF7C8FC002880D074E700BF983B0020A1
:10F0300001005FA0F0ED00E0FCED00E000005FA04B
:10F0400003005FA0062813B5044600F0DC80FFF73C
:10F05000F1FB072C1AD8DFE804F0044A0AA0A3BE8B
:10F060001907012004F0ECFA012002B010BD0120C4
:10F0700004F0E6FA022002F05BFE002004F0E0FA61
:10F08000022002F055FEFFF7BDFE08B90020ECE7B4
:10F0900001A90420FFF7E8FB0028F7D0019904201C
:10F0A00021F08041FFF7F0FB0028EFD001A90420F8
:10F0B000FFF7DAFB0028E9D001990029F6DB21F0FF
:10F0C00080510420FFF7E0FB0028DFD001A90420D5
:10F0D000FFF7CAFB0028D9D0019B9800F6D44FF067
:10F0E000A0430222C3F80027C3F80427BCE7FFF7B8
:10F0F00089FE0028CAD048494848FFF75BFC04460F
:10F1000088B9012004F09CFA022002F011FE20468A
:10F1100004F096FA022002F00BFE3F493F48FFF749
:10F1200049FC0028B2D03D4C01A92046FFF730FC35
:10F130000028ABD0019B9903F6D539480121FFF790
:10F1400039FC0028A2D0374801A9FFF721FC00288C
:10F150009CD0354B01991B68324801F4E06119439A
:10F1600041F0BF6141F40031FFF724FC00288DD04D
:10F17000022002F0DDFD294C01A92046FFF708FC22
:10F18000002883D0019B9A03F6D525480021FFF77C
:10F1900011FC003818BF012067E724491F48F6E733
:10F1A000FFF70CFE00283FF471AFFFF791FB00283A
:10F1B0003FF46CAF00210820FFF766FB00283FF406
:10F1C00065AF4FF0A0410420FFF75EFB00283FF43D
:10F1D0005DAF1749E2E7FFF715FE00283FF456AF91
:10F1E0000D490E48FFF7E6FB00283FF44FAF0B4CEC
:10F1F00001A92046FFF7CCFB00283FF447AF019B55
:10F200009B03F5D530E709490448FFF7D3FB0028F5
:10F210003FF43CAF63E700BF03005FA0F0ED00E008
:10F22000FCED00E00CED00E03408002000005FA0E1
:10F2300001005FA0024B1878431E584258417047A6
:10F24000A93B00207FB5234E32788242054628D064
:10F25000214B1C68E2B91DB394F838309B071CD4CD
:10F2600063782178E0781D4A41EA0321A37800956C
:10F2700041EA034100230293019341EA00611268CD
:10F2800004F11800FFF7ECFC50B90B2004B070BD7E
:10F2900094F83830990706D528B13378002BDFD0A1
:10F2A00035700020F2E763792179E07941EA0321A2
:10F2B000A37941EA0341002341EA006102930193EB
:10F2C000009304F11800FFF7CBFC0028C3D10C20F9
:10F2D000DCE700BFA83B00209C3B0020A43B0020B3
:10F2E0002DE9F04F6A4B1B6989B007468946904665
:10F2F000002B00F0C380674B1C68002C00F0C0801E
:10F30000654B1B686BB90220FFF79CFF064620B9CE
:10F3100004F1180AB8F1000F0BD1304609B0BDE86E
:10F32000F08F5B69002BEED098470128EBD10D26BA
:10F33000F3E794F8353094F8345094F8250045EA12
:10F34000032594F8363045EA034594F8373045EA0A
:10F35000036594F8243043EA002394F826004545D9
:10F3600043EA004394F8270028BF45462A46494609
:10F3700043EA0060FFF7CAFB002800F08380637C4B
:10F38000217CE07C41EA0321A37C41EA0341002384
:10F390000293019394F8252094F8243043EA022341
:10F3A00094F8262043EA024394F8272043EA0263B4
:10F3B000009341EA00612B463A465046FFF750FC65
:10F3C000002861D000F036FC002852D0627D237DF9
:10F3D00043EA0223A27D43EA0243E27D53EA026349
:10F3E00044D00320FFF72EFF00284FD1637D217DFD
:10F3F00094F817C041EA0321A37D41EA034194F840
:10F400003830019003F00103029394F8252094F81A
:10F41000243043EA022394F8262043EA024394F876
:10F42000272043EA026300933A462B4641EA0C61E7
:10F430005046FFF715FCE0B912266EE7102DAB46DB
:10F4400028BF4FF0100B5A4604A93846FFF7F4FACC
:10F45000C0B15A4604A9484606F048FE0028EBD140
:10F460005F44D944A8EB0B08A5EB0B05002DE5D1B3
:10F4700050E72F44A944A8EB05084BE701264CE7C9
:10F4800002264AE70A2648E7112646E7064644E7E9
:10F49000A06301009C3B0020CC490020194B10B513
:10F4A0001C695CB3184A00231370184A01201360CA
:10F4B00004F098F820B30C346178227842EA0122F3
:10F4C000A17842EA0142E17852EA01630AD1617906
:10F4D000227942EA0122A17942EA0142E17952EA23
:10F4E000016304D0227AD30706D5094A1460094B78
:10F4F00001221A70002010BD1434DDE70120FAE764
:10F500000720F8E7A0630100A83B00209C3B0020F7
:10F51000A03B0020A93B0020284B10B51B690C33F1
:10F5200059781A7842EA0122997842EA0142D97858
:10F5300052EA016225D15C79197941EA04219C796A
:10F5400041EA0441DC7951EA04611CD11C4B186882
:10F55000002830D04278037843EA0223827843EAD5
:10F560000243C27843EA0263164A1360427C037C7A
:10F5700043EA0223827CC07C43EA024343EA006000
:10F5800019E0824218D85C79197941EA04219C7902
:10F5900041EA0441DC7941EA046181420CD3094922
:10F5A0000A605A7C187C40EA02209A7CDB7C40EAA4
:10F5B000024040EA036010BD1433B1E7A0630100CC
:10F5C000A03B0020A43B0020F8B5FFF7A5FF0446B0
:10F5D000C0B31F4E3368834236D00020FFF732FE9F
:10F5E000054668BB94F82D3094F82C2094F8301020
:10F5F00094F8290094F82FC094F8337042EA03225B
:10F6000094F82E3042EA034294F8313041EA032163
:10F6100094F8323041EA034194F8283043EA002359
:10F6200094F82A0043EA004394F82B0042EA0C6263
:10F6300041EA076143EA0060FFF768FA30B13460DD
:10F640002846F8BD0925FBE70025F9E70825F7E777
:10F650009C3B0020F0B52E4B1D6985B0002D54D089
:10F660002C4E05F10C046378207840EA0320A3783F
:10F6700040EA0340E37850EA036013D162792379CA
:10F6800043EA0223A27943EA0243E27953EA02639E
:10F6900008D195F8A201002838D005B0BDE8F040A7
:10F6A000FFF7FCBEFFF738FF28B190F838305B0752
:10F6B00001D51434D7E76078237843EA0023A07893
:10F6C00043EA0043E07843EA0060FFF77DFFE8B9D2
:10F6D0000120FFF7B7FDC8B937687B7A397A97F808
:10F6E0000BC041EA0321BB7A029041EA0341019039
:10F6F00000900346024641EA0C6107F11800FFF74B
:10F70000AFFA0028D5D1102000E0012005B0F0BDEF
:10F71000A06301009C3B002038B51F4B04461869CC
:10F72000002838D0427A037A43EA0223827A43EAF5
:10F730000243C27A53EA026302D0013B002B07DA8C
:10F74000002016494FF4C67200F0B4FB002022E0FE
:10F750004179027942EA0122817942EA0142C17982
:10F7600042EA016202EBC30112F833204D7842EA0B
:10F7700005228D7842EA0542CD7842EA0562A2422E
:10F78000DBD84B79087940EA03208B7940EA0340C3
:10F79000CB7940EA036038BDA0630100F076010038
:10F7A0007FB5194B1B6906464BB3184B1D6845B313
:10F7B000FFF7B2FFB6FBF0F303FB106018B10F24A4
:10F7C000204604B070BD0120FFF73CFD0446002830
:10F7D000F6D16B7B297BE87B41EA0321AB7B02946A
:10F7E00041EA034141EA0061019400942346324614
:10F7F00005F11800FFF734FA0028E1D1DFE7012412
:10F80000DEE70224DCE700BFA06301009C3B002090
:10F81000094B1B6910B5044643B1FFF77DFFFF2874
:10F8200006D82046BDE81040FFF776BF184610BD49
:10F830004FF48070FBE700BFA06301000E4B1B6913
:10F8400010B5B3B10020FFF7FDFC044668B900F025
:10F85000E9F960B1022003F0C5FE072003F0C2FE03
:10F86000064B00221A70FEF7F6FF204610BD01205D
:10F87000F1E70124F9E700BFA0630100A93B0020E4
:10F8800070B52F4D2F4C8E220021284606F066FCC5
:10F890006278237843EA0223A27843EA0243E278BB
:10F8A00043EA0263284A934247D16379227942EAC4
:10F8B00003228E2A164638BF8E268E2A28BF8E2215
:10F8C0002146284606F022FC002385F847308E2288
:10F8D00000211C4806F042FC642323706C236370F3
:10F8E0007623A37026716B2318491948E370360AF2
:10F8F0004122667106F00AFC95F8483095F84B20D5
:10F9000084F8483095F8493084F8493084F84B2021
:10F9100095F84A300F49104884F84A30920006F0B2
:10F92000F5FB95F88C3084F88C3095F88D3084F8A0
:10F930008D30BDE8704000F0FFB88E26C7E700BFED
:10F94000AA3B0020007F0020646C766BB13B002056
:10F95000077F0020F63B00204C7F0020014B987170
:10F96000704700BF007F0020F8B50D460646F8F747
:10F970000DFE41220446471C0021114806F0EEFB13
:10F98000412F84BF403C36190E4C88BF41273A4670
:10F990003146E01D06F0BAFB84F848502D0A84F881
:10F9A0004950FEF7F5FC18B1012384F84A30F8BD40
:10F9B000FEF7F0FC08B10223F7E784F84A00F6E707
:10F9C000077F0020007F002010B5074C4122002156
:10F9D000E01D06F0C3FB002384F8483084F849306A
:10F9E00084F84B3010BD00BF007F0020024B987997
:10F9F000003818BF01207047007F00202DE9F84330
:10FA000006461C48884617461D46F8F7BFFD0446C3
:10FA100026B142460021304606F0A0FB0FB100237C
:10FA20003B800DB100232B70DFF84C9099F8070054
:10FA3000E8B1621C90453FBFC8F1070189184944ED
:10FA4000424628BF09F1070156B199F8483099F8A4
:10FA5000490043EA00233B80304606F057FB01E0B3
:10FA6000002FF9D115B199F84A302B700120BDE86B
:10FA7000F88300BF077F0020007F00200C4B93F825
:10FA80004B100F29024610D8481CC0B2123183F81F
:10FA90004B0003EB8103C2F307211A715971C2F3C2
:10FAA0000741120E9971DA7170470020704700BF4C
:10FAB000007F0020034B024693F84B0008B14C3303
:10FAC00013607047007F0020014B83F88C00704763
:10FAD000007F0020014B93F88C007047007F0020CE
:10FAE000014B83F88D007047007F0020034B93F893
:10FAF0008D00003818BF0120704700BF007F002034
:10FB00001FB50B48FEF7D2FA70B91022FF216846E4
:10FB100006F024FB07490A22684606F0F7FA044873
:10FB20006A461021FEF7CBFA05B05DF804FB00BF72
:10FB300000F00100383C0020002210B511461046AC
:10FB4000284C01F057F8284928480A2206F0DEFA26
:10FB50000A212046FEF7BCFAD8B12378627843EA3E
:10FB60000223A27843EA0243E27843EA0263204A8E
:10FB700093420ED1237962791A491C4843EA022341
:10FB8000092B9BBF227963790A2242EA032206F0FD
:10FB9000BDFA164B134864221A706C225A707622F2
:10FBA0009A706B22DA700A21002219715A71FEF7DD
:10FBB0008FFA90B12378627843EA0223A27843EA6D
:10FBC0000243E27843EA0263094A934205D123796A
:10FBD000627943EA0223092B03D8BDE81040FFF7FE
:10FBE0008FBF10BD00F001004C770100383C0020B1
:10FBF000646C766B014B9871FFF782BF383C002034
:10FC0000014BD871FFF77CBF383C0020014B1872C4
:10FC1000FFF776BF383C0020014B5872FFF770BFEA
:10FC2000383C0020024B9879003818BF01207047FB
:10FC3000383C0020024BD879003818BF01207047AB
:10FC4000383C0020024B187A003818BF012070475A
:10FC5000383C0020024B587A003818BF012070470A
:10FC6000383C002008B501F0B3FBFEF72BFD012066
:10FC700008BD08B501F0E8FB012008BD03460B48AC
:10FC800059781A7842EA0122997842EA0142D978F1
:10FC900042EA016202609A7902715A7942711B79D3
:10FCA00083710023C37101F0DFBB00BF443C00201F
:10FCB000084B1A7802705A7842709A788270DA7813
:10FCC000C2701A7982715A7942719B79037101204D
:10FCD000704700BF443C00200E4B1B6870B5DB69C9
:10FCE00004469847054638B90B4E3CB102F060F91E
:10FCF0003060284603F076FC012070BD02F058F910
:10FD00003368C01AB0F5967F2CBF01202046FEF75D
:10FD1000A3FCF1E7487701004C3C002008B501F056
:10FD20000BFC012008BD00B591B003F0C1FE4028D6
:10FD30000BD858B901F00CFC4028014616D8B0B9D0
:10FD4000FEF7C0FC11B05DF804FB402081B26846AC
:10FD500001F038FC01460028ECD0684603F0B8FEFC
:10FD60000028E7D00120FEF789FCE3E74021684640
:10FD700003F0F8FE0028E3D081B2684601F0EEFB04
:10FD80000028DDD00120FEF779FCD9E7044B0A09F1
:10FD900001F00F019A5C5B5C0270437002207047B7
:10FDA0005677010070B50D46090E0646FFF7EEFFC7
:10FDB000C5F3074104463018FFF7E8FF0444C5F3D4
:10FDC00007213019FFF7E2FF0444E9B23019FFF7C9
:10FDD000DDFF204470BDF0B5054600200A4603460D
:10FDE0000A24B2B950EA030404BF012013462C18B8
:10FDF0000A260027B1FBF6F206FB1211303104F897
:10FE0000011D11462A1B0244824277EB0302F1D303
:10FE1000F0BD013043F10003B2FBF4F2E1E7F8B5C5
:10FE2000154606460F46FFF7D6FF854204460AD917
:10FE30002A4630212C1B304606F090F930193946FD
:10FE4000FFF7C9FF2C462046F8BD70B5059DC0B12F
:10FE50005E19964215D354189C4212D393423BBF6D
:10FE6000D11AAA1A9B1AD2182ABF2A4600230021A7
:10FE7000A64284BFA41B1219049C1844214406F016
:10FE800045F9284670BD2DE9F341DDF82080044690
:10FE900040460D4616461F46F8F778FBCDF8008021
:10FEA00001903B46324629462046FFF7CEFF02B07E
:10FEB000BDE8F081F8B503460D461646A8B9EFF344
:10FEC000108772B602460146FFF798FD044618B93E
:10FED00031462846FFF748FD87F310882CB9EFF329
:10FEE0000383DB0601D1FCF7D3FDF8BD10B5EFF3BA
:10FEF000108472B6FFF768FD84F3108810BD00000F
:10FF00002D4BF7B51C6905460CB3042200230146AE
:10FF10000DEB0200019306F0F9F8019804F1D40307
:10FF20005A7819785E7941EA02219A7841EA0241C9
:10FF3000DA7841EA02611A7942EA06229E7942EAB7
:10FF40000642DE7942EA066251EA020602D1002048
:10FF500003B0F0BD884201D3904201D91433DFE7EA
:10FF600004260422A9190DEB020006F0CFF801982F
:10FF700004F10C035A7819785F7941EA02219A78E2
:10FF800041EA0241DA7841EA02611A7942EA07223B
:10FF90009F7942EA0742DF7942EA076251EA0207A3
:10FFA000D5D0884201D3904201D91433E2E7043618
:10FFB000102ED6D10120CBE7A0630100084A1268B9
:10FFC00008B503460AB1126A22B91846BDE80840CE
:10FFD000FFF796BF9047003818BF012008BD00BF4B
:10FFE000CC4900200B4A1268034612B1526A02B192
:10FFF00010471A783A2A08D1187A302807D03238B0
:020000040001F9
:1000000003288CBF0020012070470020704701208A
:10001000704700BFCC49002037B5194D0446E8B100
:10002000FEF7F0FE17486946FEF75BFC009BB3F154
:10003000227F0AD101214FF08070FEF775FC2B6FF3
:100040000BB12046984703B030BD04220E4B0F4839
:1000500001930DEB0201FEF759FDF0E7094801A9F4
:10006000FEF73FFC019BB3F1227F04D121464FF004
:100070008070FEF759FC2B6F002BE4D00020E1E7E5
:10008000A0630100FC0000010400FA050CED00E093
:1000900007B5042208490DEB020006F037F8BDF859
:1000A0000430002063F30F00BDF8063063F31F40F7
:1000B00003B05DF804FB00BF147901000020704715
:1000C0006FF0030070476FF00300704707B504221C
:1000D00000210DEB020006F041F8104801F0A8F8ED
:1000E00028B19DF8043043F001038DF804300C4A28
:1000F00092F8253092F824205B01920002F004026D
:1001000003F0200313439DF8042022F0240213433C
:100110008DF80430019803B05DF804FB48790100C4
:10012000503C002070B5114DAB699B0706460C464C
:1001300002D44FF0FF3070BD0128FAD10C4800F016
:10014000F7FF0B4800F090FF6C600A4A0848002453
:10015000291DAC6000F002FF074B9842E9D104482A
:10016000AE6100F0B1FF2046E5E700BF503C002043
:10017000487901008D0201000000AD0B054B93F89A
:100180002420054B12B9D3F84C057047D3F83C0531
:10019000704700BF503C00200030004070B50D4655
:1001A000014688B185B10B4E0B4800242A4686F8DB
:1001B000254001F011F8094B984208D1012386F837
:1001C00024303562204670BD6FF00400FBE74FF02D
:1001D000FF30F8E7503C0020487901000000AD0BEB
:1001E00070B50D46014680B17DB10B4E0B48002421
:1001F0002A4686F8254000F0C3FF094B984207D1F4
:1002000086F82440F561204670BD6FF00400FBE7DE
:100210004FF0FF30F8E700BF503C00204879010064
:100220000000AD0B70B5134C054628220021204676
:1002300005F094FFA069256010F0010615D1702328
:1002400063607223A3600C4B0C4A1B68E3600C4B89
:100250000C481B6823610125211DA682A57500F0AD
:100260007DFE094B984202D1A561002070BD4FF080
:10027000FF30FBE7503C0020C03C00208D02010015
:10028000C43C0020487901000000AD0B10B5037894
:10029000204C062B35D8DFE803F0041C2C16272C45
:1002A0002C000379002B0CBF0020042022687AB3B5
:1002B000194BD3F8D43413F0FF0324D140F4004099
:1002C000BDE8104010470379002B0CBF0020082028
:1002D000ECE7114BE069D3F84C35984234BF02206B
:1002E000002040F00100E1E70B4B206AD3F83C35D9
:1002F000F3E70123094884F8253000F02DFF802022
:10030000D4E70020D2E7012B08BF40F48040D7E7B4
:1003100010BD00BF503C0020003000404879010073
:1003200038B5124D0446A869C3071CD544B1022C48
:100330000FD0012C14BF6FF004006FF0030038BD24
:100340000B4800F0F5FEAB6923F00203AB6100201F
:10035000F5E710F00204FAD1054800F0B5FEAB69EC
:1003600043F00203F2E74FF0FF30E8E7503C002093
:100370004879010010B5094CA36903F00303032B6E
:1003800006D1074800F0D4FEA36923F00203A3615D
:10039000034800F069FE002010BD00BF503C002063
:1003A0004879010000F054BF07B5042208490DEB5D
:1003B000020005F0ABFEBDF80430002063F30F002F
:1003C000BDF8063063F31F4003B05DF804FB00BFC7
:1003D0009079010040F2016070470000044B186002
:1003E000044B1A68D2075CBF01221A6000207047D4
:1003F0007C3C0020783C00200C4B10B51C68024669
:10040000C4F34000A4070ED41C6844F002041C602E
:10041000074BC3F834250122C3F838151A6010229F
:10042000C3F8042310BD6FF00100FBE7B03C0020CF
:10043000002000404FF0FF3070470000014B18686B
:10044000704700BFA83C0020034B186810B1034B55
:10045000D3F83C05704700BF843C002000200040DA
:100460000346DAB2013A0846192A00F2D080DFE8E2
:1004700012F01D0066016601660166016601CE008C
:10048000CE00CE00CE00CE00CE00CE00CE00CE00FC
:100490001A001A001A001A001A00F90014011A00B2
:1004A000320148011A006FF00300704713F4E06F47
:1004B00040F0488103F44052B2F5805F15D0B2F5A8
:1004C000005F20D0002A40F04081A149D1F86C257E
:1004D00022F00E02C1F86C2513F4404219D0B2F597
:1004E000804F26D06FF00A007047994AD2F86C15F9
:1004F00021F48071C2F86C15D2F86C1521F00E0150
:10050000C2F86C15E8E7924AD2F86C1541F4807194
:10051000F0E78F49D1F86C2522F0100213F4403334
:10052000C1F86C250BD0B3F5403F25D06FF00B0020
:1005300070478749D1F86C2542F01002EEE7844AF3
:10054000D2F86C3523F00103C2F86C354DF6C023A8
:1005500098426FD031D8B0F5615F61D018D8B0F54E
:10056000965F5AD00ED8B0F5966F4BD0B0F5166F97
:100570004FD06FF007007047754AD2F86C3543F0E2
:100580000103E1E7B0F5165FF3D1714B714A3CE02E
:1005900047F61223984249D008D8B0F5964F42D07A
:1005A000B0F5E14FE5D16A4B6B4A2EE0B0F5164F3E
:1005B000DFD1674B4FF41D0227E0684B984245D0CE
:1005C00013D8B0F5E13F3DD008D8B0F5614F35D034
:1005D000B0F5963FCDD15E4B614A16E0B0F5613F74
:1005E000C7D15B4B4FF06C720FE0B0F5612F31D08B
:1005F0005C4B984232D0B0F5E12FBAD1544B4FF05A
:10060000E86202E0524B4FF49E22C3F824250020FA
:1006100070474F4B4FF41D22F7E74D4B524AF4E71A
:100620004B4B524AF1E74A4B514AEEE7484B4FF4E5
:100630000002EAE7464B4FF46502E6E7444B4FF40D
:100640006B02E2E7424B4FF0EB72DEE7404B4FF0BC
:100650008062DAE73E4B4FF07062D6E73C4B4FF0DA
:100660008052D2E720B101280AD06FF00400704711
:10067000404B374A1B6843F00043C2F80C357047C3
:100680003C4B1B684FF0A04203F5E0710F2042F88D
:1006900021002F4AC2F80C35B9E788B10128E4D10E
:1006A000354B1A684FF0A04302F5E0710C2043F877
:1006B0002100274BC3F81425304AC3F80423A6E7CA
:1006C0002D4B234A1B6843F00043C2F814352B4BD3
:1006D000C2F8083370471E4A294BC2F80833012379
:1006E000D360284BD2F85811012905D1264B1A683E
:1006F0006FF300021A608AE7013BF3D16FF002004A
:100700007047134B214AC3F8082301225A601D4A3F
:10071000D3F8441101290FD11B4A10686FF341002F
:100720001060D9620A4A174BD2F8101101293FF420
:100730006EAF013BF8D1E1E7013AE9D1DEE76FF0B6
:10074000060070476FF0080070476FF009007047AF
:10075000002000400050270000C0750090D003002A
:1007600000903A0140420F0000B0130000F03A0040
:1007700000A04E00D83C0020D43C00200002020023
:100780000001400000710200B03C00201000020097
:10079000014B1868704700BFB03C002082B0019B3D
:1007A0006FF300030193019B6FF341030193019BDE
:1007B0006FF382030193019B6FF3C3030193019BCA
:1007C0006FF31F130193019802B07047144B70B57B
:1007D0001C6814F0010420D11A68124E42F0010284
:1007E0001A60114B1860114B20290D46196028BF63
:1007F00020250F4B2A46014630461C6005F086FC3A
:100800000C4B0122C3F84465C3F848559A604FF475
:100810008072C3F80423204670BD6FF00100FBE72F
:10082000B03C0020883C0020803C0020AC3C0020F4
:10083000A83C002000200040012807D902380128E8
:1008400094BF6FF003006FF0040070474FF0FF306B
:100850007047000070B5394D2C68E607014669D530
:1008600040B1022840D0012814BF6FF004006FF09F
:10087000030070BD324C2368DA0702D51820FFF759
:10088000EFFD23689B0703D500211920FFF7E8FD42
:100890002C4B0024C3F800452B4B0426C3F8806082
:1008A000BFF34F8FBFF36F8F18202146FFF7D8FD9E
:1008B00021461920FFF7D4FD32462146204805F095
:1008C0004DFC224B22481C60224B1C60224B1C60BA
:1008D000224B202221461C6005F040FC2B6823F0AF
:1008E00002032B600020C4E714F00204FAD1214671
:1008F0000422134805F032FC144B15481C60154BBC
:100900001C60154B1C60154B202221461C6005F015
:1009100025FC0C4B0822C3F800252B6843F002038A
:100920002B60094B602283F802230422C3F8802144
:100930001A60D7E74FF0FF309BE700BF783C0020FC
:10094000B03C00200020004000E100E0803C00209E
:10095000883C0020AC3C0020843C0020A83C0020C7
:1009600038B5124C23689B0702D50020FFF772FFB1
:100970000F4B10481B6843F00042C0F80C2503F5EC
:10098000E0734FF0A042022142F823100A4B1B688B
:1009900043F0004503F5E073C0F8145542F8231006
:1009A000064B00202060186038BD00BF783C002056
:1009B000D83C002000200040D43C00207C3C00209B
:1009C0002DE9F041374DD5F8200120B3364B0024F6
:1009D000C5F820411E68D5F84C0582191A60334BC2
:1009E000196801441960324B1E68B2424DD2B61AE2
:1009F000304F202E28BF20263246384605F086FB91
:100A00000123C5F84475C5F84865AB604FF48073A1
:100A1000C5F804332046234BD3F8102162B10021DE
:100A20001022C3F81011C3F80823234B1A6861F38E
:100A300041021A6040F002001A4BD3F8442122B15F
:100A40000022C3F8442140F04000D3F82421B2B181
:100A5000D3F88024C3F88024150748BF40F08000F5
:100A60000021540748BF40F48070C3F82411910757
:100A700048BF40F40070D30748BF40F020000F4B40
:100A80001B686BB1BDE8F04118474FF48073C5F89F
:100A90000833094B1A6864F300021A600920BAE7A8
:100AA000BDE8F08100200040A83C0020803C0020F0
:100AB000AC3C0020883C0020B03C00207C3C002066
:100AC0004FF08053D3F830010D2804D0A0F110036B
:100AD00058425841704701207047000008B5FFF7A1
:100AE000EFFF40B14FF080430022C3F80C21C3F860
:100AF0001021C3F83825FFF7E3FF002846D04FF058
:100B00008052374BD2F80414C3F82015D2F80814D9
:100B1000C3F82415D2F80C14C3F82815D2F8101411
:100B2000C3F82C15D2F81414C3F83015D2F81814E1
:100B3000C3F83415D2F81C14C3F84015D2F82014A9
:100B4000C3F84415D2F82414C3F84815D2F8281471
:100B5000C3F84C15D2F82C14C3F85015D2F8301441
:100B6000C3F85415D2F83414C3F86015D2F8381409
:100B7000C3F86415D2F83C14C3F86815D2F84014D1
:100B8000C3F86C15D2F84424C3F87025FFF798FF1A
:100B900048B14FF08043D3F80024D20744BF6FF030
:100BA0000102C3F800244FF08053D3E94C230D2AEF
:100BB00010D1022B02D80B4AD35C3BB14FF010236B
:100BC000D3F808224FF08043C3F85825064B074A54
:100BD0001A6008BD102AF9D1032BEFD8044AEBE7BD
:100BE00000C0004094790100E40900200090D00387
:100BF000977901000020704700207047064B0222C1
:100C0000C3F80425C3F80805D3F80024D207FBD5A0
:100C10000020C3F80405704700E001400B4B30B5DD
:100C200021F003010124C3F804451144801A8A42CB
:100C300003D10020C3F8040530BD841852F8045BCA
:100C40002560D3F80044E407FBD5F0E700E001405D
:100C50001B4B1B681F2B2ED84FF0A04203F5E071F1
:100C6000032042F82100012101FA03F3C2F80C35F8
:100C7000144B1A681F2A1AD84FF0A04303EB8203C3
:100C80000322C3F80027C3F80027C3F800270E4B40
:100C90001B681F2B07D84FF0A04203F5E0730C210F
:100CA00042F823107047094A03F01F03F5E7074B8A
:100CB00002F01F02E2E7054A03F01F03CEE700BF80
:100CC000C83C0020CC3C0020D03C00200003005059
:100CD000094B1B681F2B0BD84FF0A041012202FAD1
:100CE00003F310B9C1F80C357047C1F808357047E7
:100CF000024903F01F03F1E7CC3C00200003005041
:100D0000FFF7E6BFFFF7E4BF00207047074B1B6803
:100D10001F2B8ABF064A4FF0A04203F01F03D2F8F0
:100D20001005D840C04300F001007047D03C0020BF
:100D300000030050704710B101280CD070474FF0ED
:100D40008043C3F80401D3F804210222C3F804232A
:100D500001229A6070474FF080430022C3F80021BF
:100D6000D3F80021C3F804031860704700280DDB96
:100D70004309012200F01F0002FA00F02033044A68
:100D800042F82300BFF34F8FBFF36F8F704700BF50
:100D900000E100E04358002B1EBF002242504258A1
:100DA000A1F5807114BF01230023890803FA01F023
:100DB000704703680BB108461847704707B5002A0B
:100DC0008DF80010416808BF4FF4807201920A4309
:100DD00042606946FFF7EDFF03B05DF804FB0000D9
:100DE0002DE9F74301238B724D7ADFF83881DFF864
:100DF00038910E464FF482710746FFF7CBFF4FF450
:100E0000927104463846FFF7C5FF4FF4A6710443BC
:100E10003846FFF7BFFF4FF4A87104433846FFF789
:100E2000B9FF4FF4B27104433846FFF7B3FF4FF4F4
:100E3000B47104433846FFF7ADFFEDB20443002C14
:100E400035D0042D55D8DFE805F0033845565D0050
:100E500014F0020302D024F00204F0E7610110D57F
:100E6000E20258BF01258DF800304CBF02252B4609
:100E7000694630468DF8043024F0C364FFF799FFCB
:100E8000DDE7A3010BD503238DF8003004F4002324
:100E9000002B0BBF0123002303250425E8E7D7F827
:100EA000D024C7F8D02406213046FFF787FF00235F
:100EB0007572B37203B0BDE8F0831C4D254003D0BA
:100EC00024F480140225BAE7D7F8D024C7F8D02438
:100ED0000221E9E714EA0805F6D001238DF8003075
:100EE000D7F84C35019369463046FFF762FF24F08E
:100EF00002040025A3E714EA09050CD024F4002419
:100F000004259CE714EA080505D004238DF8003079
:100F1000D7F83C35E6E7D7F8D024C7F8D024052128
:100F2000C2E700BF02000006020008060200100629
:100F300010B4037908490C225A438C188A584AB9CC
:100F4000A27A3AB903EB4303006810BC01EB8301BA
:100F5000FFF746BF10BC7047B43C00202DE9F047B6
:100F6000DFF8F08007790C2303FB078391461B7A97
:100F7000002B6DD104684FF0FF3644F3073AC4F8F4
:100F800000355046C4F80865C4F80C65FFF7EEFE5E
:100F90008B68C4F808630E7C03F01F0340F2026202
:100FA0004FF0A04003F5E07342EA860640F8236064
:100FB000CB684E7C03F01F0303F5E07342EA860220
:100FC00040F823200E684B6856EA03024FEA1435B6
:100FD00037D0003E18BF01260BB146F00206EBB237
:100FE0008D7CBAF1000F4FEA4515EDB22BDB1A48A4
:100FF00000EB0A0282F8005301224FEA5A1A03F06A
:101000001F0302FA03F340F82A308A68CB68C4F859
:101010000825C4F80C350B78C4F888350B79C4F86A
:101020008C350C235F4308EB07030022C4F894655A
:1010300048F807909A7209485A7201221A72BDE85C
:10104000F0870126CBE7064A03F00F03D554DCE70F
:101050000448F4E7B43C002000E100E00000AD0BE0
:1010600014ED00E00500AD0B2DE9F04101680679B3
:10107000D1F80855D1F80C4500274FF0FF38C1F8DA
:10108000007541F30730C1F8088505F01F05C1F868
:101090000C8504F01F04FFF769FE05F5E0754FF0BD
:1010A000A04304F5E0740222C1F8088343F8252028
:1010B00043F82420034A0C237343D118D7500F72EE
:1010C000BDE8F081B43C0020036800790022C3F839
:1010D0000421D3F80411C3F82421D3F82411C3F850
:1010E0004C21D3F84C11C3F85021D3F85011C3F858
:1010F0006421D3F86411C3F868210C21D3F8682166
:10110000094A4143515811B10849C3F80413092150
:10111000C3F800150C2303FB0023022100225A60B0
:1011200019725A72704700BFB43C002002021806C0
:101130000268074B0179C2F808330023C2F8003572
:10114000044B0C2202FB013301221A72704700BFCC
:1011500002021806B43C002010B50446FFF7E8FE72
:101160002279064B0C2101FB02330433002253E8A1
:10117000000F43E800219142F9D110BDB43C00209A
:1011800030B5104B04790C2505FB04331B7A022B78
:1011900011D101F06043B3F1005F0ED1C2F30E0430
:1011A00094420CD103680848C3F844150122C3F8DF
:1011B00048455A6330BD0548FCE70548FAE705484D
:1011C000F8E700BFB43C00200000AD0B0500AD0BFC
:1011D0000A00AD0B0600AD0B30B5104B04790C25A1
:1011E00005FB04331B7A022B11D101F06043B3F1EC
:1011F000005F0ED1C2F30E0494420CD1036808487C
:10120000C3F834150122C3F838451A6330BD0548C8
:10121000FCE70548FAE70548F8E700BFB43C0020C2
:101220000000AD0B0500AD0B0A00AD0B0600AD0BC9
:1012300010B50446FFF77CFE2279044B0C2101FB1C
:101240000233587A003818BF012010BDB43C00208A
:1012500003498B7A13B90348FFF7C2BD704700BF3B
:10126000B43C0020003000404FF08053D3F8002100
:1012700002601A6E42605B6E83600023C360704739
:101280004FF08053F0B4D3F800211B4B1B4E1C4D84
:101290001C4C1D481D499A421D4A1E4B1BD1292733
:1012A00037600F262E60112525600224046003207C
:1012B00008601D2111601C221A604FF08043D3F892
:1012C0000C24D3F80C34D90301D5D30711D4F0BCC6
:1012D0000120FFF730BD062737600E262E600F2550
:1012E00025601D240460082008601C2111601E2256
:1012F000E2E7F0BC704700BF33280500D03C002077
:10130000CC3C0020C83C0020D83C0020D43C00202D
:10131000C03C0020C43C002008B5074907484FF4F2
:101320000072F8F76FFDBDE80840054905484FF425
:101330000072F8F767BD00BF103F0020003F00209B
:10134000003D0020F03C002037B5820704460FD551
:101350001948F8F7C1FD132805461FD9174B164841
:101360001979F8F75BFD164B16489B6901219847E0
:10137000E3071FD51448114CF8F7A0FDC8B1124877
:10138000F8F774FD03462046012100F8053F0C4B99
:101390005B69019303B0BDE830401847E3D1FEF725
:1013A00051FC0028DFD0094903482A46F8F7B4FD6C
:1013B000D9E7206003B030BDF03C0020DC3C0020C9
:1013C00058790100E03C0020003F00209B7901009B
:1013D00038B5FFF7A1FF094D094B0A4800241C60EE
:1013E000AB6898472B6902209847074B1C80074B36
:1013F0001C60074B01201C6038BD00BF58790100FC
:10140000DC3C002049130100EC3C0020E83C0020BB
:10141000E43C002038B50A4C0021A56A1620A847F4
:1014200000211920A847236900209847E3689847BE
:10143000FFF772FF034B00221A60012038BD00BF86
:1014400058790100DC3C002038B5064C0425C4F86E
:101450008050BFF34F8FBFF36F8FFFF75DFF2560A5
:10146000012038BD00E100E02DE9F8430479631F55
:10147000022B43799ABF240201340124012B064632
:1014800045D0022B01D144F48054B379012B41D0D3
:10149000022B42D0F37923493268012B0B6808BF35
:1014A00044F44034A342204B02D1186890422BD020
:1014B0001E4F0C604FF004081A60C7F88080BFF31D
:1014C0004F8FBFF36F8FDFF86890FFF725FFD9F8D4
:1014D000285000211620A84700211920A84731686C
:1014E0002046A847E0B901211520A8470121162070
:1014F000A847D9F818300F4801219847C7F88081CC
:10150000C7F80080FFF7A0FF0120BDE8F88344F48E
:101510000054BAE744F40044BCE744F48044B9E71B
:101520000020F2E7E83C0020E43C002000E100E07D
:1015300058790100E03C002038B5044D2B888342E7
:10154000044602D0FFF780FF2C8038BDEC3C002021
:101550000148F8F7C1BC00BF003F002038B50A467B
:1015600029B3144B0421C3F88010BFF34F8FBFF38E
:101570006F8F114D01461148F8F7CEFC2B680446D9
:1015800083B90E48F8F79AFC60B10C48F8F76EFC86
:1015900003462846012100F8053F094B5B6998473F
:1015A00001232B60034B04221A60204638BD0846F5
:1015B000FCE700BF00E100E0DC3C0020003F002031
:1015C000587901000A4601460148F8F791BC00BF6E
:1015D000F03C002002F07ABE08B502F0DDFABDE86A
:1015E000084004F031B808B502F0B0FE02F0D8FAB5
:1015F000F7F732FC08BD70472DE9F0434C4C4D49DC
:1016000093B0092201A804F081FD092201A9204616
:1016100004F07CFDFEF75EFA012871D1464A13887A
:10162000013B9BB21380454A23716FF07403A37092
:1016300013880025173BE57084F88B50138009262A
:101640003F4B40491D70404BA71905F1010842224C
:1016500001A883F8008004F059FD01A94222384610
:1016600004F054FDBD70BD7287F8225087F82380C6
:1016700087F82D8002F02AF906F14207334B3449EE
:1016800005F102092744202201A883F8009004F004
:101690003DFD01A92022384604F038FD87F802906C
:1016A00002F084FF06F162072A4B2B4905F103087B
:1016B0002744092201A883F8008004F027FD01A92E
:1016C0000922384604F022FD87F80280234F244B7C
:1016D000244987F80E806B3604353444172201A85C
:1016E0001D7004F013FD172201A9204604F00EFD21
:1016F000A57087F8AE5013B0BDE8F04301F0B2BF5B
:1017000001F040FF002889D0174B18490025172207
:1017100001A81D7004F0FAFC172201A904F10900C8
:1017200004F0F4FCE572FBF7A5FB2026012587E712
:10173000D6410020DC610100740B0020E809002084
:10174000A9430020FC610100AA430020AB43002014
:101750003E620100AD4300205E620100290A0020C4
:10176000A843002067620100AC430020E56101004E
:101770004FF08053D3F830010D2804D0A0F11003AE
:1017800058425841704701207047000008B5FFF7E4
:10179000EFFF48B1144B49F275320321C3F8002C16
:1017A000C3F8141DC3F8002C104B0122C3F8002508
:1017B0000F4AD3F80014090501D4013AF9D1D3F83E
:1017C000002422F40062C3F80024FFF7D1FF48B1DF
:1017D000054B49F275320021C3F8002CC3F8141DE3
:1017E000C3F8002C08BD00BF00E0064000700240B6
:1017F0000071020010F0780F70B5C4B224D104F06B
:101800007F04C0F3C0101A4B04EBC00592B233F84A
:101810001550954228BF1546164A142623B206FBDA
:10182000042290B19B0003F1804303F51C33C2F8FE
:101830000016C2F8045601225A60D3F80821002A83
:10184000FBD00022C3F8082170BD9B0003F1804348
:1018500003F51C33C2F80017C2F8045701229A623C
:10186000D3F83021002AFBD00022C3F83021EBE767
:10187000BC4700200070024010B5FFF779FF0A4C0A
:1018800020B1FFF783FF0023C4F80035FFF77EFF88
:101890000123C4F80433054B402283F82723802218
:1018A000C3F884215A6010BD0070024000E100E0DE
:1018B000054BD3F8042520B142F00102C3F80425FA
:1018C000704722F00102F9E70070024038B50B4D75
:1018D0000B4C4FF0FF33C5F808330A4B0021196059
:1018E000094B01221A602046202204F037FC4023D5
:1018F00023802382054BC5F8043338BD00700240B5
:10190000BC470020DC470020B04300200104A001B8
:101910007047704770470000837813F0780F13D139
:10192000C27802F00302012A0ED04179027942EA1C
:101930000122D90903F07F0303EBC103402A0349C5
:1019400028BF402221F81320704700BFBC47002069
:101950000038024B18BF012018607047B0430020C8
:1019600010F0780FC2B214D102F07F0310F0800F94
:101970004FF0010202FA03F2064B05D0D3F810151E
:101980000A43C3F810257047D3F814150A43C3F867
:10199000142570470070024010F0780FC2B212D1C7
:1019A00002F07F030421012299409A40064BC3F8BC
:1019B0000813D3F81015D2430A4010F0800FC3F873
:1019C000102500D0704770470070024010F0780F6B
:1019D000C3B21ED113F07F03C0F3C01017D00D4A5D
:1019E00040B143F0800143F4C073C2F80C15C2F853
:1019F0000C35704743F48071C2F80C35C2F80C15F1
:101A0000044A03F59473002142F8231001E00028F2
:101A1000F6D070470070024010F0780FC3B20ED1BC
:101A200013F07F03064A02D1012353657047010674
:101A30004CBF43F4C07343F48073C2F81835704749
:101A40000070024010F0780FC3B20BD103F07F0397
:101A5000054A10F0800F18BF43F08003C2F8183514
:101A6000FFF7B4BF704700BF007002402DE9F0419E
:101A700000F078030D46C0F3C0110B43C4B25AD135
:101A800014F07F0438D12D4B1E682EB92C4B1B68E7
:101A90007BB33046BDE8F0811C602A4BD3F880242C
:101AA0002A70D3F884246A70D3F88824AA70D3F8F3
:101AB0008C24EA70D3F890242A71D3F894246A71A4
:101AC000D3F89824D2B2AA71D3F89C14E97142EAEF
:101AD000012212B21C4952B901220A601A65082675
:101AE000184B04F59474002243F82420D1E70C60CD
:101AF000F5E7154B1B68E3B904F59473DFF84480F0
:101B000058F82370B9B2914288BF1746BEB20F4948
:101B1000F21C22F0030201EB8411FFF76BFE324648
:101B2000284604F0F3FA002CDAD10123C8F850302B
:101B3000D6E72646D4E70026ABE700BFDC47002007
:101B4000B043002000700240B4430020BC4300209A
:101B500010F0780F70B5C3B2054629D1C0F3C01498
:101B6000280623D513F07F0305D11348006808BB6E
:101B700012480468D4B1124C03F1080034F8106024
:101B800094B2B44228BF344623B9B4423EBF0D4B91
:101B900001221A600C4E06EB80162246304604F0F5
:101BA000B5FA224631462846FFF724FE204670BD8E
:101BB0000024FBE71C46F9E7B4430020B0430020B3
:101BC000BC470020B8430020BC430020044B8022C7
:101BD000C3F88420BFF34F8FBFF36F8FFCF780BD36
:101BE00000E100E0F8B5434BD3F8002152B10022E8
:101BF000C3F80021FFF76AFE03F0C4FD3E4B1B68EB
:101C000003B198473B4BD3F8582192B1D3F8004425
:101C10000022C3F80024C3F85821E20503D5374B4E
:101C20001B6803B19847A30503D5354B1B6803B167
:101C30009847304CD4F8543133B10023C4F85431B0
:101C4000304B1B6803B19847D4F85C3163B12E4B1D
:101C500001221A602D4A00231360C4F85C312C4B1A
:101C60001B680BB102209847224BD3F8282182B180
:101C7000264A14680022C3F82821254B1B6823B18B
:101C8000244A12689AB30820984714B1194B0122CC
:101C90001A65184BD3F860212AB3D3F86C541C4F43
:101CA00000220124C3F860212646C3F86C5406FACA
:101CB00004F32B4204D057F824300BB10820984786
:101CC0000134082CF3D1124F01244FF4803606FA68
:101CD00004F32B4204D057F824300BB1042098476A
:101CE0000134082CF3D10C4B80225A60F8BD04203B
:101CF000CAE700BF007002408C7A0100987A0100A8
:101D0000907A0100947A0100DC470020B84300205B
:101D1000447A0100B043002000E100E0FEE7FEE766
:101D200008B5014610B1132001F064F9002008BD88
:101D3000EFF305834BB9EFF3108333B9EFF311835E
:101D40001BB9DFF80CC000DF70476FF0050070476B
:101D5000211D0100EFF310832BB9EFF31180003840
:101D600018BF0120704701207047000070B5474C34
:101D7000217A012900F08580002940F08480444DBB
:101D80009C2204F1080004F0E9F9EB68EE6AE365CF
:101D90002B8AA4F85430296BAB682364304600F0DA
:101DA00019F908B1C4F880606E69A969304600F07D
:101DB00011F908B9D4F880606667EE69296A30467F
:101DC00000F008F908B9D4F88060A6676E6AA96ABD
:101DD000304600F0FFF808B9D4F88060E6676E6B13
:101DE0003EB1F368B2683168304600F05DF9C4F87E
:101DF0008460AE6B3EB1F368B2683168304600F083
:101E000053F9C4F88860EE6B3EB1F368B26831688C
:101E1000304600F049F9C4F88C602E6C3EB1F3688E
:101E2000B2683168304600F03FF9C4F890606E6CDB
:101E30003EB1F368B2683168304600F035F9C4F855
:101E40009460AE6C3EB1F368B2683168304600F021
:101E50002BF9C4F89860EE6C3EB1F368B268316853
:101E6000304600F021F9C4F89C602D6D3DB1EB685F
:101E7000AA682968284600F017F9C4F8A050012381
:101E80002372002070BD4FF0FF30FBE77C0B002079
:101E9000B862010070B5234D2B7A012B03D04FF0AF
:101EA000FF34204670BD01F03BF90028F7D01E4AF0
:101EB0001E4E1F497068FF2382F8223092F82230AC
:101EC000D26863F0FF03DB4314BFB3FA83F320232C
:101ED000C3F12003C2F30222934298BF531CFE2297
:101EE00002FA03F3104ADBB2D37701F0A9FA0446F1
:101EF0000028D4D101F0DCFA286101F0C1FA0D48C4
:101F000000F09AFE00F00CFF336813F0010F4FF061
:101F1000020303D083F314882B72C2E7032282F3F7
:101F20001488F9E77C0B002000ED00E0B8620100A6
:101F300073850000980B002038B5084BDD6801F070
:101F4000BFFA044601F0C2FA18B101F0B9FA01353E
:101F5000044601F0B0FA05FB004038BD7C0B0020C0
:101F60007047000008B5FFF7FBFFEFF3058313B1DF
:101F70006FF0050008BDFFF7EDFE0028F8D1DFF88F
:101F800008C000DFF6E700BF6D1D010008B5EFF3E4
:101F9000058313B16FF0050008BDFFF7DBFE0028D5
:101FA000F8D1DFF808C000DFF6E700BF951E01009A
:101FB00008B5EFF305831BB1BDE80840FFF7BCBFD0
:101FC000FFF7C8FE0028F7D1DFF804C000DF08BD26
:101FD000391F010010B5034688B1084310F007000F
:101FE0000DD117290AD9196008391022CC189C6024
:101FF0005A60C85099684A60D860012010BD00201E
:10200000FCE7F0B5034670B369B332F003002AD1A0
:102010000F3121F0070103F1080634463668656880
:10202000301B25F00305401B814203D9306800288E
:10203000F3D1F0BD5F681D680F445F602B44083B1F
:102040005868874288BF5F6063680A431BB9626053
:1020500004F10800EDE723F00303E018E6504260C6
:1020600020600830E5E70020E3E710B5034678B1CB
:10207000C1B1083900F1080200248A4209D151682F
:1020800021F003005968091A596044B954600120CD
:1020900010BD106814460028FAD00246EDE7136818
:1020A0002360F4E70846F3E730B5C0B189B1C2B1A7
:1020B000CBB10024446002FB01F41D190160826071
:1020C000C360436105611846013904D1A21A9950D1
:1020D0000121084630BD851805602846F4E7014611
:1020E000F7E71146F5E71946F3E710B50346A8B13F
:1020F00000F1140252E8000F10B9BFF32F8F04E073
:10210000016842E8001404B1F4E738B1043353E83D
:10211000002F511C43E8001404B1F8E710BD30B59E
:10212000F0B1C3688B421BD803698B4218D900F108
:1021300014031A680A60BFF35F8F53E8002F0C681E
:102140009442F6D143E8001505B1F2E7043050E8B7
:10215000003F5A1E40E8002101B1F8E7002030BDE1
:102160006FF00300FBE7EFF310832BB9EFF311805F
:10217000003818BF01207047012070474B688A68FB
:1021800023B19A608A681AB153607047C262F9E756
:10219000036370472DE9F84F8846074618B90026B3
:1021A0003046BDE8F88F0029F9D0CE1C26F0030692
:1021B0000C36B0FA80F304D0B6FA86F10B441F2B2C
:1021C000EDDD06FB07F9E2B194688CB1A307E6D117
:1021D000D368332BE3D91569D2F800A053695DB1F8
:1021E00015F0030BDBD19945D9D8002C3DD10AE07D
:1021F000D368002BEFD0D2E7002BD0D11CB19B4687
:102200000DE092461546254BD3F8A000D8B1FFF754
:102210006CFF04460028C2D04FF0010B2DBB1F4BB2
:102220000022D86F4946FFF7ECFE0546B8B9BBF16E
:10223000000FB4D0194BD3F8A060214656B13046F8
:10224000FFF76DFFABE7D3F8800001223421FFF7E1
:10225000D8FEDEE7D3F88000FFF707FFA0E74A4685
:10226000002103F07BFF4BF0020BFA2323700023C5
:102270003246A360A362E362236384F802B02B4674
:10228000C4F804A0C4F82480394604F10C00FFF718
:102290000BFF024B024A1A67264681E77C0B00209F
:1022A0003123010010B500F1280353E8002F12B9C3
:1022B000BFF32F8F04E0511E43E8001404B1F4E78C
:1022C0000AB9002010BDC06A01220028F9D0811C83
:1022D000D1E84F3FC1E8442F04B1F9E7DBB2002B4E
:1022E000F0D08068F1E7036B30B5E3B1CD7800241E
:1022F000DA78AA420FD31A464A608C608AB191609C
:10230000A4B16160283050E8003F5A1C40E8002129
:1023100001B1F8E730BD5A681C46002AECD01346DC
:10232000E6E7C162ECE74B608B60C1620163E9E7FD
:10233000F8B5877804468FB3C5680146002728465C
:10234000FFF71CFF277005F10C042046FFF7E7FE9E
:10235000AB68002B48D02046FFF7C7FE0446002894
:1023600042D0284600F068FC3A460646394600F05E
:102370000DFD304600F0BCFC6A6A8168064604F137
:102380000C0003F0C3FEF9232370A770F368E37019
:1023900021462846BDE8F840FFF7A5BF8568AB6831
:1023A000002BF5D05B78832BF2D1284600F044FC5B
:1023B0003A460646394600F0E9FC304600F098FC03
:1023C00006466A6A806804F10C0103F09FFEF36818
:1023D0000BB1E2781A7000232370214605F10C003E
:1023E000BDE8F840FFF79BBEF8BD00002DE9F041C5
:1023F0000C46174698460546002848D00378FA2B25
:1024000045D1002943D08368C3B15B78832B15D1B4
:1024100000F012FC01220646002100F0B7FC304615
:1024200000F066FC06466A6A8068214603F06EFE8C
:10243000F06808B107700020BDE8F08105F10C00DC
:10244000FFF753FE064670B121466A6A0C3003F06E
:102450005DFE0024F9233370B470F77031462846CE
:10246000FFF741FFE7E7B8F1000F13D04146932093
:1024700000F0C0FD40B1094B2846596900F0CAFB85
:10248000EFF309839C60DF606FF00100D4E76FF029
:102490000300D1E76FF00200CEE700BF7C0B002005
:1024A0002DE9F0410F46144698460546002859D0BC
:1024B0000378FA2B56D1002954D0FFF7F3FE0646D5
:1024C00000283BD001462846FFF758FE6A6A06F10D
:1024D0000C01384603F01AFE0CB1F3782370002487
:1024E00005F10C07347031463846FFF718FEAB682B
:1024F00013B90020BDE8F0813846FFF7F6FD064627
:102500000028F6D0284600F097FB21460746012216
:1025100000F03CFC384600F0EBFB6A6A8168074635
:1025200006F10C0003F0F2FDF9233370B470FB6880
:10253000F37031462846FFF7D6FEDAE7B8F1000F10
:1025400013D04146832000F055FD40B1084B28468A
:10255000596900F05FFBEFF309839F60DC606FF067
:102560000100C7E76FF00300C4E76FF00200C1E7A6
:102570007C0B002010B50446EFF305830BB100205F
:1025800010BDFFF7F0FD0028F9D1DFF808C02046A4
:1025900000DFF5E7952101002DE9F04106460F46E1
:1025A00090461C46EFF305831BB166B96FF003003C
:1025B00026E0FFF7D8FD0028F7D1DFF850C03046FD
:1025C000234600DF1CE03378FA2BEFD1002FEDD04B
:1025D000002CEBD106F10C00FFF787FD054688B112
:1025E000726A39460C3003F091FDF92328462B70AE
:1025F000AC7085F803806F60AE6000F027FA20466B
:10260000BDE8F0816FF00200FAE700BFED230100A2
:10261000F8B504460F4616461D46EFF305831BB179
:1026200064B96FF0030023E0FFF79DFD0028F7D1A8
:10263000DFF844C020462B4600DF19E02378FA2B50
:10264000EFD1002FEDD0002DEBD12046FFF72AFE71
:10265000054670B100F10C01626A384603F056FD80
:102660000EB1EB7833702846EC6000F0EFF90020F3
:10267000F8BD6FF00200FBE7A1240100EFF3108327
:102680002BB9EFF31180003818BF012070470120EB
:102690007047000038B5034660B3D0E90045806854
:1026A000A0B110F0030201D0002038BDDB681B2B65
:1026B000FAD91346F522837000230270C570446076
:1026C0008360C360036143610376EEE7DB68002B40
:1026D000EAD10A4BD3F8940030B9D3F88000012234
:1026E0001C21FFF78EFC01E0FFF7FFFC0028DBD088
:1026F0000123DFE704460546EBE700BF7C0B002023
:10270000224B70B55D6904460E46002D35D0002879
:1027100036D00378F52B33D1037E53B90361EB6ACE
:10272000C560436103B11861EC6201232376002088
:1027300070BDC278D10706D5C168A94203D1FF2B6D
:1027400021D00133F2E7F6B193070AD5E06895F995
:10275000203090F920209A4203DA80F8203000F0EF
:102760007DFA3146532000F045FC18B12946204639
:1027700000F050FA6FF00100DAE74FF0FF30D7E7D2
:102780006FF00300D4E76FF00200D1E77C0B00206C
:1027900038B5284B5A690446002A42D0002843D055
:1027A0000378F52B40D1037E002B40D0C1689142C5
:1027B0003DD1013BDBB2037633BB43690BB1016909
:1027C0001961216911B34B61E3789B0705D592F933
:1027D0002110D36AE3B982F82010A3688BB1204698
:1027E00000F02AFA00220546114600F0CFFA002335
:1027F0002361EB6AE560636103B11C610123EC6254
:102800002376002000F096FA00200CE0D362DBE78C
:10281000986820B190F920008142B8BF01465B69F9
:10282000D8E74FF0FF3038BD6FF00300FBE76FF0E3
:102830000200F8E77C0B00202DE9F0410446002659
:1028400001270CB9BDE8F081E378D4F814801B07A8
:1028500012D5A36826767BB1204600F0EDF9002260
:102860000546114600F092FAEB6AE5602661636165
:1028700003B11C61EC6227764446E2E710B4C378EA
:102880009B0719D5C06890F92130C26A94688C42C0
:1028900008BF8C6824B194F92040A342B8BF2346F6
:1028A0005269002AF2D190F920209A4204D080F88F
:1028B000203010BC00F0D2B910BC704708B50246F9
:1028C000EFF305830BB1002008BDFFF7D7FE00280A
:1028D000F9D1DFF808C0104600DFF5E795260100C2
:1028E00008B50246EFF3058313B16FF0050008BD8C
:1028F000FFF7C4FE0028F8D1DFF808C0104600DF5B
:10290000F5E700BF0127010008B50246EFF3058394
:1029100013B16FF0050008BDFFF7B0FE0028F8D135
:10292000DFF808C0104600DFF5E700BF912701007F
:1029300010B5D0E85F3F5A1C914200D80022C0E891
:10294000542F04B1F5E798B210BD000038B51A4C09
:1029500000F0AAFDE3680133E360236D03B19847FB
:1029600000F096F9002000F0E5F9236C1BB3A26B90
:10297000A1698A4202D0A163E3631CE0E36BB3B9AF
:10298000237A022B17D1656AADB195F9201092F91F
:10299000203099420FD1284600F057F9A06B00F083
:1029A0006FF9284600F0BCF9236CA563E4E7013B0E
:1029B000E363002BE4D038BD7C0B002070B5224CC3
:1029C00004F1560504F15A06B4F85410D5E85F3FF7
:1029D00013B9BFF32F8F04E05A1EC5E8502F00B182
:1029E000F4E79BB25BB33046FFF7A2FFE36D53F809
:1029F000200020B30378F13B082BE5D801A252F860
:102A000023F000BF292A0100C92901002F2A010053
:102A1000C9290100C9290100332A0100372A010010
:102A2000C92901003B2A0100236E9847CCE7636E59
:102A3000FBE7A36EF9E7E36EF7E7236FF5E7BDE881
:102A40007040002000F076B97C0B002070B5164C69
:102A50000546B4F8541004F15602D2E85F3F99429B
:102A600002D8BFF32F8F04E0581CC2E8560F06B1FE
:102A7000F3E79BB2994205D829460220BDE8704091
:102A8000FFF74DB904F15800FFF752FFE36D43F82B
:102A90002050637A23B9054B4FF080525A6070BDC5
:102AA0000123A372FBE700BF7C0B002000ED00E0D8
:102AB000EFF310832BB9EFF31180003818BF01201A
:102AC0007047012070470378F12B00D07047C06831
:102AD000F9E7000010B50A4A90F92010012343706D
:102AE000536A1C321BB193F920408C4205DCC26052
:102AF0008360906003B1D86010BD1A469B68F1E70F
:102B00007C0B0020014B5869704700BF7C0B0020F4
:102B1000DFF804C000DFFEE7C130010010B500237C
:102B2000038083789A07044608D513F0100F016BD1
:102B30000E4B0FD0D3F88400FFF7F1FAA378DB0730
:102B400012D50A4BD3F88800214638B1BDE81040B1
:102B5000FFF7E5BA586FFFF788FAEFE7BDE81040D6
:102B6000D3F88000FFF781BA10BD00BF7C0B0020B6
:102B700010B5C46903694169621C0AD103B1596186
:102B800042691AB113610023436101E0064A1363ED
:102B900010BD1BB1DA6959612244DA614269002A29
:102BA000F0D1014AD362F3E77C0B0020930710B504
:102BB00002F0010422D400F1280384B153E8000F8D
:102BC00000EA01028A4203D0BFF32F8F002005E004
:102BD00020EA010243E8002404B1EFE710BD53E806
:102BE000000F084203D1BFF32F8F002005E020EA39
:102BF000010243E8002404B1F1E7EFE7806A01EA4B
:102C000000031CB18B4218BF0020E7E7002B08BF70
:102C10000020E3E710B591F9202083681BB193F9F8
:102C20002040944205DAC8608B60816003B1D960AE
:102C300010BD18469B68F1E70346806882689A6079
:102C400002B1D3600023C3607047C2682AB18368B1
:102C5000936003B1DA600023C360704710B5044687
:102C600064B12378F12B07D0FFF7EFFF0146204630
:102C7000BDE81040FFF7CEBFE468F1E710BD0000EB
:102C80000123014643700148FFF7C4BF980B0020A1
:102C900038B5164DEC6A44B3E369013BE36123BBED
:102CA0006378732B06D009D8532B0BD003F0DF03C6
:102CB000432B0DD12046FFF706FF09E003F0EF0399
:102CC000832BF6E72046FFF7FEFE2146FFF7D6FDF1
:102CD0002046FFF7BAFFFFF7D3FF246924B1E36969
:102CE000002BDDD000236361EC6238BD7C0B00203B
:102CF000806B203070470000074B596951B10B6B56
:102D00008A6B934203D21A68044B9A4202D0012084
:102D1000FFF705B8704700BF7C0B0020A52E5AE2D4
:102D200008B502234370024B9861FFF7E5FF08BD29
:102D30007C0B002010B5144B04461A7A5969A0B9CF
:102D4000022A1FD15C6AECB194F9202091F920305D
:102D50009A4217DD2046FFF778FF0846FFF7BAFED4
:102D60002046BDE81040FFF7DBBF022A05D190F9ED
:102D7000202091F920309A42EFDC2046BDE8104037
:102D8000FFF77EBF10BD00BF7C0B0020836B10B52A
:102D900014461962FFF7ECFE1CB1BDE81040FFF7C6
:102DA000C9BFBDE81040FFF76BBF10B54378332BA8
:102DB00004460CD1416A90F82320FFF7F7FE014644
:102DC00028B120460022BDE81040FFF7DFBF10BD4C
:102DD00070B5044648B30378F12B26D1002924DBD3
:102DE0004378042B24D000F1280353E8002F42EA53
:102DF000010543E8005606B1F7E74378332B12D1BB
:102E0000416A90F82320FFF7D1FE014658B194F8AB
:102E100023309B0756BF656A054620EA0505012257
:102E20002046FFF7B3FF284670BD6FF00305FAE7B1
:102E30006FF00205F7E700002DE9F04F85B08146FD
:102E4000029120B90024204605B0BDE8F08F002A89
:102E500044D096689EB1B407F4D1D368432BF1D91E
:102E600002F11004B0CC74B16007EBD1002DE9D0B1
:102E700057B918276907E5D1472D0AD8E2E7D36883
:102E8000002BEDD0DEE73FB37B1E372BDAD8002DC9
:102E9000F0D15368D2F800A0019366BB504BD3F831
:102EA000880008B3FFF721F906460028CAD04FF082
:102EB0000108002C40F08780DFF824B1F5B9494AB9
:102EC000DBF88400556DC8B1FFF70FF90246F0B189
:102ED00048F01008344626E01827D8E792461446F2
:102EE000182715460192D9E7D3F880000122442122
:102EF000FFF787F8D8E74FF00008DAE72246DBF85B
:102F000074002946FFF77DF802460028E2D1B8F1A7
:102F1000000F56D0DBF88820002A49D010463146F1
:102F2000FFF7FDF8002248F00208002C8AD040F29A
:102F3000F1132380019BE3700023A360E36023610E
:102F40006361A361E3616362A362E362A5F140038D
:102F500013447FB2A363FD21234B84F80280C4F89D
:102F600004A084F8207084F8217061842263656372
:102F7000C4F83C9013601B4B1B685B0726D4A36B03
:102F800000201A4603F1340143F8040B9942FBD1A7
:102F9000164B53634FF08073D363029B1362104B45
:102FA000C2F838902046124A1A66FFF7C3FE4AE775
:102FB000DBF8800003923146FFF757F8039A144676
:102FC000B1E74246AFE722463446B0E7AD08113DCF
:102FD0004FF0CC33002DD2D042F8043F013DF9E749
:102FE0007C0B0020B8620100A52E5AE2112B0100D3
:102FF000AB2D010038B51D4C237A022B024633D18C
:10300000606A98B163695A704A1C15D1226B00211D
:103010006AB94FF0FF30D86159611A6151B10B6143
:103020001348FFF709FEFFF77BFE012038BD11466C
:103030001269EDE72363F3E7E26A002012B1D56974
:10304000A9420BD2D96158611A6158B10361002AB3
:10305000E6D0D0695361411AD161E1E71046491BBE
:103060001269EBE7E362F2E70020DFE77C0B002068
:10307000980B0020F8B5114B5E6904460F461546C3
:1030800096B1002813DB0A4601463046FFF78EFD55
:1030900048B97DB1746286F8237029463320FFF762
:1030A000A9FF6FF00100F8BD4FF0FF30FBE76FF0B4
:1030B0000300F8E76FF00200F5E700BF7C0B00208B
:1030C00038B5154D2B7A022B25D16B6A1BB36C6971
:1030D000E06AFFF7B1FBA06918B100221146FFF7C3
:1030E00055FEEFF309830D48A363FFF7A5FDFFF736
:1030F00017FE00236B61E278D20704D42046BDE8B6
:103100003840FFF70BBD04226270E3606B6BA36075
:1031100003B1DC606C6338BD7C0B0020980B002091
:1031200038B50B4C0B48A26D0B4D0021FFF784FE08
:10313000636EA8624BB1E26D08480021FFF77CFE88
:10314000A864003818BF012038BD0120FCE700BF8B
:10315000B86201001D1D01007C0B0020B533010089
:1031600010B50446EFF305830BB1002010BDFFF747
:103170009FFC0028F9D1DFF808C0204600DFF5E702
:10318000392E010008B5EFF3058313B1054B5869DB
:1031900008BDFFF78DFC0028F8D1DFF80CC000DF78
:1031A000F6E700BF7C0B0020052B010038B5024676
:1031B0000D46EFF305831BB162B96FF003041EE007
:1031C000FFF776FC0028F7D1DFF83CC0104600DF9F
:1031D000044614E01378F12BEFD1002DEDDB53788A
:1031E000042B0ED002F1280353E8001F41EA050426
:1031F00043E8004000B1F7E71046FFF727FC204600
:1032000038BD6FF00204FAE7D12D010010B5044675
:10321000EFF3058313B16FF0050010BDFFF748FC15
:103220000028F8D1DFF808C0204600DFF5E700BF2E
:1032300075300100EFF310832BB9EFF311800038E4
:1032400018BF0120704701207047000030B50C4DB9
:103250006B6C002213B11C698C420AD90161826037
:10326000C3601BB11C699860611A19612AB1D060F2
:1032700030BD1A46091BDB68ECE76864F8E700BF5D
:103280007C0B0020C36810B52BB104691A698168F2
:10329000996022441A6182680AB1D36010BD014A64
:1032A0005364FBE77C0B002038B50D460446A8B1FB
:1032B0000378F22B12D189B14378022B07D1FFF7A3
:1032C000E1FF20462946FFF7C1FF002038BD064B2D
:1032D0001B6D33B1022343706161F2E76FF00300AD
:1032E000F4E76FF00200F1E77C0B002070B5134D9E
:1032F0006C6C04B32369013B236101262369D3B9B4
:10330000E3680BB1A2689A606B640023E86C1A460C
:1033100004F11801FFF740F918B121460320FEF728
:10332000FEFCE378012B07D161692046FFF78EFF91
:103330006C6C002CE2D170BD6670F9E77C0B00204C
:10334000F8B50E4617461C46054608B90020F8BDDC
:103350000129FBD8DBB198681A68A0B110F003030B
:10336000F4D1E1681F29F1D914464FF4F972837042
:1033700000230280C67044608360C36003614361C0
:103380008561C761E3E7DB68002BDFD11446084B9A
:10339000D3F88C0028B1FEF7A8FE0028D6D0012370
:1033A000E3E7D3F8800001222021FEF72AFEF4E7AC
:1033B0007C0B00200B4B0C4C07B51A6E586E082185
:1033C000FFF7D8F8094BE0642365E06C4FF0FF335A
:1033D00000226946FFF71CF90028F6D1DDE900302C
:1033E0009847F2E7B86201007C0B0020ED32010043
:1033F00038B505461C46EFF305830BB1002038BDF8
:10340000FFF718FF0028F9D1DFF808C02846234647
:1034100000DFF4E74133010008B50246EFF305830E
:1034200013B16FF0050008BDFFF704FF0028F8D1C5
:10343000DFF808C0104600DFF5E700BFA932010041
:10344000A8B10C4B1B68B3FBF0F00138B0F1807FE2
:103450000DD2094BFF2283F823204FF0E0230622F0
:103460001A61586100209861044B187070474FF042
:10347000FF307047E409002000ED00E0C84900205B
:10348000074B1A782AB100221A70064B4FF080625F
:103490005A604FF0E022136943F001031361704753
:1034A000C849002000ED00E04FF0E0231B697047A1
:1034B0004FF0FF3070474FF0E023586901307047FC
:1034C0004FF0E02358699B69C01A70474FF0E02322
:1034D0001869C0F30040704780B400AF154B1B69FA
:1034E000002B22D0134B1B6993F89C2193F89D115C
:1034F00009020A4393F89E1109040A4393F89F3185
:103500001B061343002B10D00A4B1B6993F89C2118
:1035100093F89D1109020A4393F89E1109040A4386
:1035200093F89F311B06134300E0034B1846BD463A
:1035300080BC7047A0630100A463010080B400AFA9
:103540000F4B1B69002B14D00D4B1B6993F8A02166
:1035500093F8A1311B0213439BB2002B09D0084BF7
:103560001B6993F8A02193F8A1311B0213439BB26E
:1035700001E0034B5B881846BD4680BC704700BF26
:10358000A063010080B400AF054B1B69002B14BF82
:1035900001230023DBB21846BD4680BC704700BF44
:1035A000A063010038B50C4D2C6894B9FFF7C6FF35
:1035B0000A492346DAB251F82220541C04D12B6860
:1035C0003BB9074B2B6004E022B11488844201D13F
:1035D0002A6038BD0133EDE7CC490020200C0020E3
:1035E000687C010070B5144D6B6F044603B19847B9
:1035F000124B1B68E3B19A691AB12046BDE87040CE
:1036000010479A78012A04D12046BDE87040FBF7A4
:1036100061BC022A0ED1A86F10B1FBF705F902E0D8
:1036200058680028F9D12046BDE87040FBF70ABD74
:10363000184670BD0120FCE7A0630100CC490020C2
:10364000034B1B6813B1DB6903B11847704700BF18
:10365000CC490020024B186800B1806A704700BF57
:10366000CC49002008B5064B064A1A60064B0748AD
:1036700000221A80F7F7B6F9054B01221A7008BD2F
:10368000F44B002016410020F04B0020D0490020D0
:10369000F24B002007B500230A48009301AA6946AF
:1036A000F7F7ABF950B1084B1878DDE9001240F09C
:1036B0008000FEF74DFA03B05DF804FB034B0122D6
:1036C0001A70F8E7D04900209F7B0100F24B0020E0
:1036D00073B5194B194D1E88194C1A4B2A8821684D
:1036E0001878B21AFEF7C2F92A88236812FA80F213
:1036F00092B213FA80F3964281B223602A8006D9EF
:10370000114B1878114B33F810308B4211D91049F6
:10371000104801ABF7F78FF938B10F4E337823B16A
:103720000020FFF7B7FF0023337000232B80084BE6
:10373000236002B070BD00BF047A0100F04B00208E
:10374000F44B0020A07B0100004F0020A27B010071
:1037500016410020D0490020F24B0020420710B54E
:10376000044602D50020FFF7B3FF230704D5BDE8C8
:1037700010400020FFF78EBF10BD000010B5144CA4
:1037800014482168144B0288CB1AD21A134B1878AC
:10379000134B33F810309A420FDB124B1878FEF7B8
:1037A00065F92368104A03442360136823B10F4965
:1037B000096809B9013B136010BD0D4B01221A6065
:1037C0000A4B1B68002BF7D0074A13680133F2E756
:1037D0002C4C0020AC7B010056410020004F002003
:1037E000A87B0100A77B0100084C0020044C0020AE
:1037F000FC4B0020F8B5244E244F33683A68244C23
:103800009A1A04D12368C3B9224A1360F8BD224B27
:103810001968224B1B68994207D3214B21481B880A
:1038200003448818834298BF5A1A1F4B19781F4BBC
:1038300033F811309A42A8BF1A46002323601C4B6C
:10384000154D1878296840F08000FEF781F93B6833
:103850002968144A03443B60114F3F8801441744D0
:10386000B94218BF0A462A603268934209D10E4B0A
:103870001A780E4B33F81230984202D1012323609C
:10388000C4E70023FBE700BF1C4C0020184C0020BD
:10389000144C0020104C0020304C0020344C0020F0
:1038A000AE7B010096410020004F0020A87B010064
:1038B000A67B010000207047002070470020704761
:1038C000002070470020704700207047174A1849B1
:1038D00008B500231360174A1360174A1360174A8C
:1038E0001360174A1360174A0A6017490A60174A9B
:1038F00017491360174A1360174A1360174A136079
:10390000174A0A6017490A60174A1380174A6FF06E
:103910003D0113705170D37001211371537108234D
:1039200091709371FCF79EF908BD00BF0C4C00200C
:10393000344C0020104C0020144C00201C4C002063
:10394000184C002096410020304C0020004C0020F4
:103950002C4C0020044C0020084C0020FC4B002084
:1039600056410020284C0020F84B0020204C00201D
:10397000184B194A10B500241C60184B1C60184BDA
:103980001C60184B1C60184B1C60184B1360184AC5
:103990001360184B184A1C60184B1C60184B1C60B5
:1039A000184B1C60184B1360184A1360184B1C808E
:1039B000FCF75FF917486FF03D03437001238370F4
:1039C00008230470C470047144718371FCF756F9C4
:1039D00010BD00BF0C4C0020344C0020104C0020C7
:1039E000144C00201C4C0020184C00209641002054
:1039F000304C0020004C00202C4C0020044C0020B7
:103A0000084C0020FC4B002056410020284C002090
:103A1000F84B0020204C002008B50D4A0D48517885
:103A2000137843EA0123917843EA01430370C3F317
:103A300007211B0C41708370D378C3701379037115
:103A40005379437193798371FCF718F908BD00BF6E
:103A50009F420020204C002010B50F4C2046FCF760
:103A600027F9C0B16278237843EA0223A27843EAB7
:103A70000243E27843EA0263084A190A137051705C
:103A8000190C1B0E9170D3702379137163795371E4
:103A9000A3799371012010BD204C00209F4200208B
:103AA00008B5024B1880FCF739F908BDF84B002027
:103AB000044B054A1888054B12681B689B1AC01AEC
:103AC000704700BFAE7B0100184C00201C4C00204A
:103AD0002DE9F8431D4A1E4B1E4F1C8815683B6894
:103AE0005B1BE51A002D06462DDDDFF86C801B4BB5
:103AF000D8F800001B688D42A8BF0D46984220D31D
:103B0000DFF85C9043194C449C421AD8241A224690
:103B1000314602F0FBFA2644C8F800902C1B54B141
:103B20002246D8F80000314602F0F0FAD8F800201A
:103B30002244C8F800203B682B443B602846BDE87F
:103B4000F8832C46EBE70025F8E700BF184C00206F
:103B5000AE7B01001C4C0020344C0020304C002077
:103B60009641002038B50A4A0A4D14680B46296868
:103B70008C420BD9641A9C42A8BF1C46224602F014
:103B8000C5FA2B6823442B60204638BD0024FBE790
:103B90002C4C0020284C002008B5FFF7E9FE08BD9A
:103BA00038B51E4B1B78002B37D01D4C226862B9EC
:103BB0001C481D4905680B689D4206D11B4B9D4260
:103BC0001FBF03600B601A4B1A601A4B1B6893B13E
:103BD000174A236815681D430DD101232360FFF7A1
:103BE000CDFD104B256018680F4B1B68984202D022
:103BF000C01AFFF75FFE104D104A2B6814681C4373
:103C00000BD10F4B19680F4B1B68994205D001234C
:103C10002B601360FFF7EEFD2C6038BDE84E0020EE
:103C2000004C00202C4C0020284C00205641002045
:103C3000FC4B0020084C00200C4C0020104C0020B5
:103C40001C4C0020184C00207047000070B50D4C33
:103C5000256825B10C4A13680133136070BD0B4E03
:103C6000012323603360FFF789FD094B3560186835
:103C7000084B25601B689842F0D0C01AFFF71AFE67
:103C8000ECE700BF004C0020084C0020044C002052
:103C90002C4C0020284C002010B5064C236843B95A
:103CA00001232360044B1B680BB1FFF7A3FD002326
:103CB000236010BD0C4C0020104C0020420710B5B2
:103CC000044601D5FFF7C2FF230704D52046BDE80F
:103CD0001040FFF7E1BF10BD08B52949294B09780D
:103CE0001A79914205D028490978914201D00020E3
:103CF00017E05A78042A09D9203AD1B20329F6D814
:103D0000032AF4D8DFE802F0092A2D34013A032A05
:103D100003D8DFE802F0070211181C4B1C4A1A6096
:103D2000012008BDFFF7CAFD0028E0D0174B184A54
:103D30001A6001F057FDF3E79A78D87842EA00203C
:103D4000FFF7C0FDF0E79A78D87842EA0020FFF745
:103D5000BBFD0028CBD001F071FDE1E7FFF77CFE51
:103D6000E2E79A78D87842EA0020FFF799FEF0E778
:103D70009A78D87842EA0020FBF7AEFFE9E700BF67
:103D8000A9430020024F0020AA430020EC4E00204F
:103D90009F42002008B51249124B09781A799142C6
:103DA00005D011490978914201D000200DE05A78E0
:103DB000022A0BD0202A10D0002AF6D1FFF77CFD72
:103DC0000028F2D001F03AFD012008BD9A78D87899
:103DD00042EA0020FFF774FDF2E7FFF71DFEEFE770
:103DE000A9430020024F0020AA4300201B4B02469B
:103DF000D878212810B503D0222820D000201DE03B
:103E000017481B790078984203D0164800789842EA
:103E1000F4D1154B1C78154B187808B9012C0DD02E
:103E2000134B1448002C18BF03461360124A128823
:103E30001344124A136009230B60012010BD084A85
:103E40001B7912789A4203D0064A12789A42D5D149
:103E50000A4B0B4A1A600B4B1B88EDE7024F002000
:103E6000AB430020AD430020004F0020C17B010088
:103E7000D64100209E420020E8090020EC4E0020A0
:103E80001A7A01003C7A010010B52E4A2E4C1278A5
:103E900023799A4205D02D4A12789A4201D0002007
:103EA00010BD6378013B0A2BF9D801A252F823F028
:103EB000DD3E01001B3F0100373F01009F3E010036
:103EC0009F3E01009F3E01009F3E01009F3E01007A
:103ED000033F0100293F01003D3F010000F064F86D
:103EE0000028DCD0E378012B06D1194B194A1A605F
:103EF00001F078FC0120D3E7032BF9D1144B164ACB
:103F0000F5E7E378022B03D1114B144A1A60F1E76D
:103F1000032BEFD10E4B104AF8E700F083F800288E
:103F2000BDD00B4B0E4AE2E700F08AF80028B6D06D
:103F300001F084FCDEE700F09DF8F0E700F0A4F863
:103F4000F4E700BFAB430020024F0020AD43002048
:103F5000EC4E0020E5420020E042002026430020F5
:103F60009F42002008B50B490B4B09781A79914202
:103F700005D00A490978914201D0002008BD5B783C
:103F8000092BFAD100F02CF80028F6D001F056FCED
:103F90000120F3E7AB430020024F0020AD43002097
:103FA00000207047704700000A49C878022808B509
:103FB0000DD0032809D00128074A18BF00228978AC
:103FC000002300F0FDFA012008BD044AF7E70020B5
:103FD000FAE700BF024F0020E5420020E042002047
:103FE00037B50D49C878022810D0032810D0012811
:103FF00010D000228B79CC7900250095897843EA8E
:10400000042300F007FB012003B030BD034AF1E7B1
:10401000034AEFE70020F7E7024F00202643002085
:10402000E0420020034B044A9B78D25C034B012002
:104030001A707047024F0020E34200209F42002088
:10404000094A9378D178094A10B543B908480478E9
:10405000D8B2844206D902F8011B0133F8E71344B1
:1040600003F8011C012010BD024F0020E342002094
:10407000B47B010008B5FFF793FF024B18700120D5
:1040800008BD00BF9F42002008B5034B9878FFF79A
:1040900089FF012008BD00BF024F00202DE9F84331
:1040A000534C544E238832889BB29A4220D3524BB1
:1040B0001B68EBB9514F524D3B60338001231846CA
:1040C00015F8011C2A4600F07BFA80B22080238874
:1040D0009BB205F1FF385BB14A4BC7F800801B78F3
:1040E000012B89BF23883D6001339BB288BF2380A9
:1040F00023889BB223B9444A1168002937D0136042
:1041000023883D4D9BB20BB92B6873B3228833884B
:10411000DFF8F8803E4FDFF8E490D21A98F80030CC
:1041200037F813403B4B92B21878944228BF14469C
:1041300030B1D9F80010224640F08000FDF708FDAC
:10414000D9F80030344A2344C9F800303388128843
:1041500023449BB29A42338048D998F8003037F80C
:104160001330A34242D101232B60BDE8F8832B4FCB
:104170003B68002BC4D0234A294D1278012A11D85C
:1041800005F8011B02232A460120318000F018FAAD
:1041900080B2208023889BB20BB1184B1D60002396
:1041A0003B60ADE729780122202928BF002102FACF
:1041B00001F818EA030F01F10101C9B2F4D000239C
:1041C00029700F4A33800120022300F0F9F980B2F0
:1041D000208023889BB22BB1084B1D6023880133BC
:1041E0009BB223803B6823EA0803D9E70023BBE79F
:1041F0004A4C0020484C0020444C00205C4C0020DD
:10420000E5420020B47B0100404C0020004F00201C
:10421000BA7B0100B07B0100B27B01004C4C002056
:10422000E442002037B51F4C1F4D22881F4B2AB98E
:104230001F4929601F492280098819801A8823880C
:104240002968D21A1C4B1878FDF710FC2B6813FA5A
:1042500080F32B60238813FA80F39BB282B2238011
:1042600052B114490988994206D914490878144969
:1042700031F81010914213D9124A1278012A4FF0E6
:104280000102009289BF104A094A12F8011C03F189
:10429000FF3398BF0021022000F0BCF900232380E7
:1042A00003B030BD3A4C0020584C00203C4C00205C
:1042B00025430020BE7B0100B17B0100004F0020A0
:1042C000BA7B0100C07B0100264300200C4A00237A
:1042D00013700C4A13600C4A13600C4A13600C4AAA
:1042E00013800C4A13800C4A13600C4A13600C4A6A
:1042F00013800C4A13800C4A13600C4A13807047D9
:10430000504C0020404C00204C4C00205C4C0020C5
:104310004A4C0020484C0020444C0020584C0020BF
:104320003C4C00203A4C0020544C0020384C0020DB
:10433000020710B5044601D5FFF7B0FE630704D5A8
:104340002046BDE81040FFF76DBF10BD2DE9F04FCE
:10435000554B1B7887B0002B00F0A280534908789A
:10436000431C0B70524B1D78042205EB45039A4009
:10437000013A90424F48A4BF0122029202884FF0B6
:104380000004ACBF0C700294FE2A9CBF0132028074
:10439000494A91F800B032F815E002880192474A84
:1043A000474912780592022202FA03F30493454B1F
:1043B000454D1A68454B03930023984618464FF025
:1043C0000109059CDEB2A6421BD33E4B00B11A6028
:1043D000B8F1000F02D0354A82F800B0019A1B688C
:1043E000964502BF334A00211180002B58D0384B2C
:1043F000188880B2002853D107B0BDE8F04FFFF70E
:104400004DBE029C002C36D14FF0000C2E78049C3F
:1044100006FA04F7BE453FDD019C371E18BF012791
:10442000A64506D1002E39D009FA03F00243012037
:104430000746039C14F801AB039456450CD00E7844
:10444000564507D309FA03F04FF0010802434FF035
:10445000000B404685F800A0BCF1000F07D01FB943
:1044600009FA03F0024301204FF000040C700133FD
:1044700001310135A5E70E78FF2E1CBF01360E7005
:104480002E78002EC0D091F800C0B44534BF4FF054
:10449000000C4FF0010CB9E70027CAE73746C8E720
:1044A00007B0BDE8F08F00BFE84E0020514C00205F
:1044B000004F002066430020B67B0100B47B010062
:1044C000E14200204C4C0020E2420020E342002068
:1044D0004A4C00202DE9F8431D4B1B8893420546AA
:1044E000144633DB1B4B187800282DD01A4B1B4E7B
:1044F00001221A60B6F800801FFA88F8B8F1000FA0
:10450000F8D1DFF85C904F46224607F8015B384649
:1045100001F0FCFD134A144BA2F80080134AC3F8C3
:1045200000901278A4B2012A348089BF33881F60BA
:1045300001339BB24FF0000088BF3380FFF7AEFD20
:104540000B4B00225A550120BDE8F8830020FBE701
:10455000B27B0100E84E0020404C00204A4C002075
:10456000E4420020484C00205C4C0020B47B010059
:10457000E142002007B50B4801AA6946F6F73DFA6B
:1045800038B1019B402B07DD074933220020FBF7A0
:1045900091FC03B05DF804FB009940220020FFF776
:1045A00099FFF6E7604C0020FC7E0100024B0348B7
:1045B00001221A70F6F716BA804E0020604C0020D7
:1045C000012837B515461C4602D0002003B030BD87
:1045D000012BFAD80C4801AA6946F6F70EFA70B119
:1045E000019A402A05DD094950220020FBF762FCB0
:1045F000EBE70099284601F089FD4020E6E7012C11
:10460000E3D1034B1C70E1E7604C0020FC7E01000D
:10461000804E0020022837B511461A4606D12BB12C
:104620000B78072B04D1104B01221A7003B030BD58
:104630000E4801ABF6F7FFF980B101980C4DF4F785
:104640009AFC2B78441E18BF01241BB1FFF792FF80
:1046500000232B702046FAF707F8E7E70549862282
:10466000FBF728FC0124F5E768150020604C0020CA
:10467000804E0020FC7E010000F054B810B51A4BAB
:104680001A4A19791278914201D0002015E05A781F
:10469000FE2A13D0FF2AF8D1DA78997841EA02216C
:1046A0009A79DB7942EA03230B43EED100F070F8EC
:1046B0000028EAD001F0C2F8012010BD9A78D9781C
:1046C00052EA0122E1D19879DC7940EA0424012CF4
:1046D000DBD100F071F80028D7D0054B054A1A60ED
:1046E00001F080F8E8E700BF024F0020AC43002053
:1046F000EC4E00209F4200207047000010B5044699
:10470000FDF78AF92306064B4ABF4FF4803001209B
:1047100004F00F0400FA04F4186804431C6010BD90
:10472000F44E0020154B1B791A0603F08F0042BF90
:1047300003F00F024FF480339340114A127858BFB0
:10474000012342F0800258BF8340824214D10D4AB7
:104750001268134210D00C494A780B7843EA0223BE
:104760008A7843EA0243CA7843EA0263074A9342DB
:1047700002D10D22FDF7ECB9704700BF024F0020B7
:10478000C37B0100F44E0020CB4E00205553425312
:10479000064A00231360064A137053709370D37057
:1047A000044B07221A700120704700BFFC4E002006
:1047B000CB4E00208C4E0020024B00221A700120AC
:1047C000704700BF9F42002010B51A4A1A4C517A18
:1047D000137A43EA0123917AD27A43EA014343EA06
:1047E0000263226815499342154A96BF2360042349
:1047F00003231370134B2268187840F08000FDF7F4
:10480000A7F9114A517A137A43EA0123917A43EACC
:104810000143D17A43EA016321685B1AC3F307219C
:1048200013725172C3F307411B0ED372002313732B
:10483000917210BDAC4E0020884E002068430020CD
:104840008C4E0020C37B0100CB4E0020094908B5E7
:1048500055230B7053234B70CB70074B18784222B3
:104860008A7040F080000D22FDF772F9034B05229B
:104870001A7008BDCB4E0020C37B01008C4E002077
:1048800038B51A4B1D681A4B1D606DBB194B1A4C7D
:10489000597A1A7A42EA0122997A42EA0142D97A8D
:1048A00052EA016209D093F90C30002B0BDA134B5A
:1048B000187840F08000FFF721FF01232373FFF7F2
:1048C000C5FF284638BD627A237A43EA0223A27ADA
:1048D00043EA0243E27A43EA0263094A12689342D6
:1048E000EBD0084B1878E6E70125EAE7D84E002020
:1048F000DC4E0020AC4E0020CB4E0020C37B0100DC
:10490000884E0020C47B01002DE9F8433E4F3F4B09
:104910003A681B683E4D9A423DD33E4B18780024BE
:1049200040F08000FFF7EAFE2C73FFF78FFFFFF7E0
:10493000A7FF394EDFF8E4803368DFF8E490002801
:1049400008BF0024002B31D1002C31D0354BD8F8D2
:1049500000201B6838681344013BB3FBF2F3D9F81D
:1049600000209A4228BF1A462F4B1968F8F7A4FA7C
:104970002D4B31681868274B01441878224640F0C7
:104980008000FDF7E5F83368264A23443360136856
:104990001B1B13600CE0254B1A78254B33F8124093
:1049A000204B1B689C4228BF1C46C0E7002CDFD16F
:1049B000D9F80010D8F8002033684A439A4204D14D
:1049C000002333603B680B443B606A7A2B7A43EAEE
:1049D0000223AA7A43EA0243EA7A43EA02631B1BF0
:1049E000C3F307222B726A72C3F307421B0EAA722B
:1049F000EB7234B10B4B1B681BB90E4A2B730321AE
:104A00001170BDE8F88300BF844E0020A04E002046
:104A1000CB4E0020C37B0100984E0020A84E002002
:104A2000A44E0020904E00209C4E0020004F0020FD
:104A3000C67B01008C4E00202DE9F047484B494EC3
:104A40001B683268484F9A4209D3484B00241878B3
:104A50003C60FFF753FE464B1C73FFF7F7FEFFF772
:104A60000FFF00B93860DFF80C813A68D8F80030E1
:104A7000414813440268934250D8404C404D0021B5
:104A80003A68D8F800308A424FD83E4DD1182B688A
:104A9000C8F80010A3EB0209C5F80090DAB1DFF8FE
:104AA000E8A00468DAF80020B9F1000F45D1002928
:104AB00043D0631E0B44B3FBF4F4314B30681968E8
:104AC000944228BF14462246F8F70CFA3268C8F818
:104AD000009022443260264A3968507A137A43EAB9
:104AE0000023907A43EA0043D07A43EA00635B1ADA
:104AF000C3F3072013725072C3F307401B0E90726A
:104B0000D37259B32B681BB1204B1B78052B25D1D1
:104B100000231373BDE8F047FFF798BEBDE8F047E8
:104B20001B49FE220020FBF7C5B92A6814F801CB07
:104B30000A44013102F803C0A2E75443A142CAD19A
:104B40000F4B30681968F8F7CDF90023DAF8002028
:104B5000C8F80030336813443360BCE7BDE8F08721
:104B6000A04E0020844E0020884E0020C47B01000F
:104B7000CB4E0020984E0020A84E00206843002015
:104B80009C4E0020904E0020A44E00208C4E002011
:104B9000247F0100F8B53E4E3E4B32681B683E4D07
:104BA0009A4209D33D4B002418782C60FFF7A6FDEC
:104BB0003B4B1C73FFF74AFEFFF762FE394C00289F
:104BC0003AD12860384A286811682368091A1160A8
:104BD000364A1568364A126803446A439342236092
:104BE00004D10023236033682B4433602C4A547A69
:104BF000137A43EA0423947A43EA0443D47A43EAD7
:104C000004631B1AC3F3072413725472C3F30744DB
:104C10001B0E9472D372002838D019B1254B1B7823
:104C2000052B33D1244B1B68B3FA83F35B09137351
:104C3000BDE8F840FFF70ABE2A682368002AC1D001
:104C40001E4F83B91A4B39681A68174B30681B68B6
:104C50001344013BB3FBF2F3144A12689A4228BF93
:104C60001A46F8F729F93B6822682F681448991802
:104C70003A4413448B42A5D011F8017B10F8012B64
:104C80009742F7D00C4B00221A609BE7F8BD00BF9B
:104C9000844E0020A04E0020884E0020C47B0100DE
:104CA000CB4E0020984E0020904E0020A44E0020B5
:104CB000A84E00208C4E0020944E00209C4E0020D8
:104CC0006843002010B5304CA27C637C43EA022389
:104CD000E27C43EA0243227D43EA02632B4A1BBA89
:104CE00013602B4A00211160E27BA82A21D01BD837
:104CF0002A2A2AD02F2A28D0282A2BD0254A1268DF
:104D00005343254A1360617A227A42EA0122A17A4A
:104D100042EA0142E17A52EA016222D11F4B0122AA
:104D20001A73FFF793FD13E0AA2AE7D1FFF7A8FD56
:104D300070B1A27D637D43EA0223E27D43EA024330
:104D4000227E43EA02631BBAD8E7FFF799FD08B950
:104D5000002010BDA37DE27D43EA02235BBA9BB233
:104D6000CCE793420DD094F90C30002BB5BF0C4B1F
:104D70000C4B18781878B8BF40F08000FFF7BEFCE5
:104D8000CCE70120E5E700BFAC4E0020844E0020B8
:104D9000984E0020A84E0020904E0020CB4E0020C0
:104DA000C37B0100C47B010010B5124B587A1C7AFA
:104DB00044EA0024987A44EA0044D87A54EA006429
:104DC00006D10D4B02221A73FFF740FD204610BD9D
:104DD00093F90C30002B0ADB084B1878FFF78EFC98
:104DE000054B02221A730024FFF730FDEEE7012481
:104DF000ECE700BFAC4E0020CB4E0020C47B01008E
:104E000010B5FFF7D1FF00283AD01E4B1E48702284
:104E10001A7000241D4A5C701268016832EA0101B0
:104E20001BD006219970282119735C73026000223F
:104E30000A21DA701A715A719A711A725A729A7238
:104E4000DA729A73DA731A745A74D971104B122287
:104E5000BDE810401A60FFF7B7BC2AB9022199706B
:104E60003A2119735A73E2E70A4A127B12B99A700F
:104E70001A73F7E705229A7020221A735973D6E73E
:104E800010BD00BF68430020DC4E0020D84E00203B
:104E9000884E0020CB4E002010B5FFF785FF18B3D9
:104EA000124B002280211A7059705A7102219A7196
:104EB000DA7120200E4A9970D97018711168083380
:104EC0001C220C7874B101311C70013A12F0FF02FF
:104ED00003F10103F5D1074B2422BDE810401A600D
:104EE000FFF772BC1870F0E710BD00BF68430020E8
:104EF000780B0020884E002010B5FFF755FF48B30F
:104F0000FFF7BEFC30B3144B144903221A70002281
:104F10005A700968DA70C9019970114B0420186041
:104F2000104B5C7A197A41EA04219C7A41EA0441E7
:104F3000DC7A41EA0461814208D90B49187208728F
:104F40004A728A72CA725A729A72DA72BDE8104054
:104F5000FFF73ABC10BD00BF68430020E44E0020BC
:104F6000884E0020CB4E0020AC4E002010B5FFF73D
:104F70001BFF68B3FFF784FC50B3164A06210023D9
:104F8000517015491370937009681371C901D1707C
:104F900053719371D371114A08201060104A547AEA
:104FA000117A41EA0421947A41EA0441D47A41EA2F
:104FB0000461814208D90B49107208724B728B72DE
:104FC000CB7253729372D372BDE81040FFF7FCBBF3
:104FD00010BD00BF68430020E44E0020884E002032
:104FE000CB4E0020AC4E002008B5FFF7DDFEE8B147
:104FF000FFF746FCD0B10E4B1A680E4B013A110E6A
:105000001970110C5970DA70110A0B4A99701268F4
:10501000DA71110E1971110C5971110A9971074B3E
:1050200008221A60BDE80840FFF7CEBB08BD00BFEC
:10503000A04E002068430020A84E0020884E00208B
:1050400010B5FFF7B1FE002839D0FFF719FC002892
:1050500035D01B4B0821D97000221A491A705A709A
:105060009A700968D971080E1871080C5871080AED
:1050700002211972144998710968D972080C587282
:10508000080A9872114B0C201860114B5C7A197A3F
:1050900041EA04219C7A41EA0441DC7A41EA046154
:1050A000814208D90B49187208724A728A72CA7210
:1050B0005A729A72DA72BDE81040FFF785BB10BDD4
:1050C00068430020A04E0020A84E0020884E0020FB
:1050D000CB4E0020AC4E002038B5FFF765FE00280F
:1050E0003ED0204B204C214D02221A705A70204B8A
:1050F0002A6003211970617A237A43EA0123A17A95
:1051000043EA0143E17A43EA0163934209D9194929
:10511000227200230A724B728B72CB726372A3727B
:10512000E372154B0F491878022240F08000FCF71B
:105130000FFD627A237A43EA0223A27A43EA02430A
:10514000E27A43EA02632A689B1AC3F307222372B6
:105150006272C3F307421B0EE3720123A272237330
:1051600038BD00BF68430020CB4E0020884E002091
:105170008C4E0020AC4E0020C37B010010B5FFF721
:1051800013FE40B31449154C00234B70CB77144BDE
:10519000202203200A701870124B2260187840F009
:1051A0008000FCF7D5FC104A517A137A43EA0123B8
:1051B000917A43EA0143D17A43EA016321685B1A99
:1051C000C3F3072113725172C3F307411B0ED3724D
:1051D00001239172137310BD68430020884E002094
:1051E0008C4E0020C37B0100CB4E002010B5134A2B
:1051F000517A137AD47A43EA0123917A43EA01433C
:1052000053EA046413D092F90C30002BB5BF0C4B59
:105210000C4B18781878B8BF40F08000FFF76EFA92
:10522000094B01221A73BDE81040FFF70FBBFFF7CF
:1052300027FB10B1044B1C73F5E710BDAC4E0020EA
:10524000C37B0100C47B0100CB4E002038B5094B65
:10525000094C9D7C5DB9D87C084B00F001001860BA
:10526000FFF74AFA2573BDE83840FFF7EFBA01238C
:105270002373F8E7AC4E0020CB4E0020D84E002020
:10528000034B044ADB7C03F001031373FFF7DEBA20
:10529000AC4E0020CB4E0020024B00221A73FFF7C9
:1052A000D5BA00BFCB4E0020A04BA14A1968A14837
:1052B0001F2970B54FF000030D46144628BF1F2567
:1052C000AB423BD11F2940F014816278237843EA36
:1052D0000223A27843EA0243E27843EA0263964A51
:1052E000934240F0068162792379944D43EA022388
:1052F000A27943EA02432B71C3F307221B0C6A71A4
:10530000AB71E379EB71627A237A43EA0223A27AE2
:1053100043EA02432B72C3F307221B0C6A72AB727F
:10532000E37AEB72637B1BB9A37B013B0F2B0BD999
:1053300001232B73BDE87040FFF788BA10F8016BAA
:1053400002F8016B0133BBE7E37B2F2B5ED8192BEF
:105350002AD8032B68D0122B6AD0002BE8D1BDE8E5
:105360007040FFF743BF9E3B0C2BE1D801A252F8DF
:1053700023F000BF7154010031530100315301008B
:105380006954010031530100E5540100315301001B
:1053900031530100315301003153010079540100B0
:1053A00031530100A15401001A3B152BC0D801A2B2
:1053B00052F823F0495401003954010031530100DF
:1053C00031530100415401003153010031530100B8
:1053D0003153010031530100595401003153010090
:1053E000615401003153010031530100795401002F
:1053F00031530100A1540100315301003153010028
:105400003153010031530100B7540100AA2B8FD84A
:105410009D2BA8D85A2B1BD0912B01D0352B87D18F
:10542000BDE87040FFF738BFBDE87040FFF7E8BC4B
:10543000BDE87040FFF730BDBDE87040FFF706BF24
:10544000BDE87040FFF71CBFBDE87040FFF754BDDA
:10545000BDE87040FFF78ABDBDE87040FFF7F0BDC2
:10546000BDE87040FFF7C0BDBDE87040FFF734BE37
:10547000BDE87040FFF782BEFFF724FC60B394F9EB
:105480000C30002B06DA2E4B02221A70BDE8704059
:10549000FFF73ABA2B4B1878FFF730F9022348E7A9
:1054A000FFF710FCC0B194F90C30002B15DB244B36
:1054B00001221A7010E0237C13F002033FF439AF8D
:1054C000FFF700FC40B194F90C30002B05DB1C4ABF
:1054D000012313701C4A136070BD1C4B187840F0F8
:1054E0008000D9E7194B187840F08000FFF706F9E3
:1054F0001EE7164B164C1D7845F08000FFF7FEF8AE
:1055000005F00F0522684FF48033AB40134323604E
:105510000C4B1D782846FFF7F1F820680123AB40BB
:10552000034323600622064BC3E700BF884E0020DA
:10553000AC4E00206843002055534243CB4E002020
:105540008C4E0020C47B0100944E0020C37B0100E0
:10555000FC4E002008B5104A1378023B032B19D8E3
:10556000DFE803F002120C160C4BDB7B03F07F0329
:10557000282B0FD1BDE80840FFF7C6B9084B1878B3
:1055800040F08000FFF7BAF8BDE80840FFF75EB9C9
:105590000023137008BD00BF8C4E0020AC4E0020CD
:1055A000C37B010008B5214B1A78072A31D8DFE800
:1055B00002F02C043030301430261D4BDB7B2F2BB7
:1055C00007D003F07F032A2B2ED1BDE80840FFF758
:1055D00033BABDE80840FFF7DDBA164B16491A7812
:1055E00001239340154A1268134218BF0120BDE8F9
:1055F000084040F23F4208BF0020FAF75BBC00229F
:105600001A700F4B1B681F2B0ED1BDE80840FFF727
:105610004BBE084B1878FFF771F80A4B02221A7339
:10562000BDE80840FFF712B908BD00BF8C4E00204E
:10563000AC4E0020C47B0100247F0100F44E00200A
:10564000884E0020CB4E0020FFF7A2B808B5064BCD
:1056500006491A88064B1878FCF708FA054B1860BB
:10566000BDE80840FFF79EBF3E7A01006843002076
:10567000C47B0100884E0020420710B5044602D5C5
:105680000020FFF7E3FF230703D5BDE81040FFF735
:1056900061BF10BD2D4A137813F01F0370B5054686
:1056A00003D0022B1BD000230FE09478D27844EA79
:1056B0000224012C09D1264E48B12046FCF728F9D6
:1056C000338843F0020333802B46184670BDFCF745
:1056D0001FF9338823F0020333800123F5E71179A2
:1056E0000B0642BF01F00F034FF480349C40194B6E
:1056F0001B7801F08F065CBF0124B440002BE4D07E
:1057000011F00F03E1D0144B1B682340DDD09378D8
:10571000D27853EA0223C6D138B13046FCF77CF97F
:105720000E4A136823431360CEE70D4B1B681C42DF
:10573000D3D13046FCF786F93046FEF79DFF074A85
:10574000136823EA04031360C7E700BF024F002079
:10575000EA4E0020E84E0020F84E0020F44E0020D3
:10576000FC4E002008B5054B00221A70FBF744FFE1
:10577000FBF741FFBDE80840FCF77EB8004F002072
:10578000FCF796B8084B1A78084B1A80084A002391
:105790001370084A1370084A4FF001111160074A4C
:1057A0001360074A13607047CA7B0100EA4E00206D
:1057B000E94E0020E84E0020F84E0020F44E002074
:1057C000FC4E0020024B1878003818BF01207047AB
:1057D000E84E0020024908220020FCF747B900BF2C
:1057E000024F002010B50A490A4C0A78A388934258
:1057F00098BF1A460AB9084B1A7021688020FCF736
:10580000A7F9236803442360A388181AA08010BD59
:10581000C27B0100EC4E00200A4F002010B5064C60
:105820000020A2882168FCF721F923680344236043
:10583000A388181AA08010BDEC4E0020002211464B
:105840008020FCF785B90000024B03491A7800203C
:10585000FCF70CB9C27B01009F4200202DE9F04FFC
:10586000034687B09B07019040F18980914C924D8F
:10587000FFF7B0FF2078C009FCF76AF8E279A37956
:1058800043EA0223AB802378C3F34112012A00F0DC
:105890003D83022A00F04F83002A40F0B3806378F2
:1058A0000B2B00F2AF80DFE813F00C004D00AD00D1
:1058B0005900AD005B00A600AD00A101A7018A025E
:1058C0009E02237803F01F03012B07D0022B15D073
:1058D000002B40F09780794B2B6030E0784B1B78A1
:1058E000002B00F08F80774B22791B789A4280F052
:1058F0008980754B00221A705A70EDE794F90430D4
:105900002279002BB5BF02F00F0102F08F014FF496
:10591000803301238B406A49097809B9170771D18F
:105920006A4A126813426DD06949674A09680B4296
:1059300014BF012300231370002353702A60FFF764
:1059400051FF1CE00020FFF7A5FE00285AD0FFF70A
:1059500075FF604B1B6893B1984710E00120F2E798
:105960002378DE064ED1A0785B4B60F07F020121E8
:1059700000F07F001A70FBF7CCFFFFF75FFF019B81
:10598000580717D54B4D95F90030002BC0F2F08227
:10599000494CA38873B1FFF741FFA38853B92B7813
:1059A000C3F34112012A00F0D3828020FCF734F8BF
:1059B0000023A380019B19070DD53E4B93F90030BE
:1059C000002B80F2D8823C4B9B8813B9434B1B7849
:1059D0000BB1FFF707FF019B5A0602D50020FCF729
:1059E00031F8019B1B0640F1D482802007B0BDE84E
:1059F000F04FFCF727B8237813F01F0313D0012BC7
:105A000000F0EC8094F90030002BC0F29F82A37963
:105A1000E27953EA022300F099820020FBF7FCFFB1
:105A20000023AB80ABE7E378013B0E2BEAD801A261
:105A300052F823F0715A0100F95A01008D5B010000
:105A4000055A0100055A0100995A0100515B0100F5
:105A5000055A0100055A0100055A0100055A0100C6
:105A6000055A0100055A0100055A0100C75B0100F3
:105A70001B4B2B6012230593059BAA889A427FF645
:105A80005EAF184AAB801278013A1A427FF457AFE2
:105A9000124B01221A7052E7134B1B78002BB1D026
:105AA000124B134A1978134B002918BF13462B6069
:105AB0000A23E0E7024F0020EC4E0020EA4E0020CF
:105AC000E84E0020014F00209F420020F84E0020A9
:105AD000F44E0020847A0100E94E00200A4F002095
:105AE000067A0100C27B0100C17B0100004F00204B
:105AF000197A0100187A01008E4A8F4B12781B78B0
:105B000012B9012B3FF47EAF0222ABB98B4B049349
:105B10005A70A078049B0022114681420ED102B136
:105B20000493049B1A78002A3FF46CAF2B609A7898
:105B3000DB7842EA03239EE7814BE8E71E782EB12B
:105B40009A78DE7842EA0622134401220131E4E722
:105B5000784B1B78002B3FF455AF774B1B7807220F
:105B600093B9774B04935A70A078049B0022114696
:105B70008142D4D01E782EB19A78DE7842EA06228D
:105B8000134401220131F3E76C4BEBE7A0786D4B36
:105B90000493032814D1F8F7C5FA286003786AE75C
:105BA0001E780EB13344012201318142F8D102B195
:105BB0000493049A1378002B3FF424AF2A605AE729
:105BC00000221146F1E7604B1B78002B3FF41AAF1F
:105BD0005E4B2B601A78002AA9D113E705A904A807
:105BE000FEF704F900287FF447AF0BE72378D806C7
:105BF0007FF408AF564B6FE62378D9067FF402AFE7
:105C0000A378002B00F0B6804A4A4B4B12781B78E1
:105C100012B9012B3FF4F6AE484E494ADFF834B1D1
:105C2000DFF82C91002B18BF16464FF00008337890
:105C30004BB9474BA2781B789A427FF4E3AEFFF74B
:105C4000FDFD454B86E67378023B052B44D8DFE823
:105C500003F003434F524303A2787379934241D137
:105C600089F800303D4B32791A703D4B3D4A198816
:105C7000002318468B4231D30127BA46DBF80030A7
:105C80000AFA07F21A4202D03846FBF785FEDBF823
:105C900000304FF48032BA401A4203D047F08000FF
:105CA000FBF77AFE0137102FE8D12F4A4FF001138E
:105CB000CBF80030002313602C4A01201360FBF75F
:105CC00029FEF37913F0400F294B1A8814BF42F0D4
:105CD000010222F001021A80337807E002F8010B7A
:105CE0000133C7E7B378F27843EA02231E449EE704
:105CF00096F80380F0E7B8F1000FEDD1B3781A06FB
:105D000003F08F0743BF03F00F024FF4803393403B
:105D10000123DBF8002058BFBB4013433046CBF8CB
:105D20000030FBF7F9FD3846FBF71AFE3846FBF763
:105D30004DFED1E7C17B0100004F0020D64100207D
:105D40009E4200209C7A01009E7B0100CB790100DD
:105D5000E84E0020F84E0020407A0100014F00205C
:105D6000740B002010410020F44E0020FC4E002057
:105D7000EA4E0020884A894F13700126B0463A68DF
:105D800008FA06F3134202D03046FBF705FE3A68E4
:105D90004FF48033B340134203D046F08000FBF74A
:105DA000FBFD0136102EEAD14FF001133B607C4B16
:105DB000002018607B4B1860FBF7ACFD39E72378B7
:105DC00003F01F03012B7FF41DAE734B1B78002BD8
:105DD0003FF418AE744A237912789A427FF612AED5
:105DE000724A134478E5237803F01F03012B7FF4F4
:105DF00009AE694B1B78002B3FF404AE6C4A6D4B27
:105E000012781B7812B9012B3FF4FCAD6A4A6B4E35
:105E10004FF00008002B18BF1646604B604ACDF8C3
:105E20000880C146C346C246317839B9B8F1000F7F
:105E30003FF4E8ADFFF702FD614B8BE57178023965
:105E400005294FD8DFE801F0034E0E234E035249D7
:105E500070790978884245D0B178F07841EA00211C
:105E60000E44E1E796F802A0217996F803B0514577
:105E70000AD1A178594507D14C4911F80A0002907E
:105E800001F80AB04FF001084FF000092AE021792B
:105E9000514527D1B778380607F08F0142BF4FF43C
:105EA000803007F00F0700FA07F7A0785CBF0127E2
:105EB0008F40584518D1186803913843186010680E
:105EC00020EA070010603046FBF726FD03990846DC
:105ED000FBF746FD03990846FBF778FD49EA0709F9
:105EE0002F4A2E4B3178BBE702988345FAD117EA47
:105EF000090FF7D1186820EA07001860106820EA37
:105F0000070010600846FBF747FDE9E703F01F03B1
:105F1000012B7FF477ADFDF7B7FF00287FF42FAD9D
:105F2000FEF7ACFB00287FF42AADFDF7D5FE002874
:105F30007FF425AD66E5DE067FF464AD00F044F83D
:105F400000287FF41CAD00F085F8F0E7802065E5BF
:105F500003F01F03012B7FF428ADFEF703F80028A0
:105F60007FF428ADFDF716FF00287FF423AD1CE574
:105F7000FFF76AFC1EE5134B93F900201878002AFE
:105F8000BFF629AD00F07F0000211870FBF7C1FCBF
:105F900021E507B0BDE8F08FE84E0020F84E002064
:105FA000F44E0020FC4E0020014F00201041002044
:105FB000C17B0100004F00209E420020D6410020FE
:105FC000887A0100E94E002038B51C4D1C4B6A78D8
:105FD0001B789A422ED12B796A7943EA0223022B4D
:105FE00028D1AB7843B3174C002201329A42207873
:105FF0001CD3D0B1F8F77EF80146E01C00F0B6F8EB
:10600000114A20781460AB79E97943EA012383428D
:106010000ED90E4B90801B78013B034202D10C4BF2
:1060200001221A70FFF7DEFB012038BD0444DCE7D3
:106030009380F7E70020F8E71846F6E7024F0020C4
:10604000CB7B0100EA090020EC4E0020C27B01005E
:106050000A4F002008B5154A154B51781B78994214
:1060600021D11379517943EA0123072B1BD111491F
:1060700011480B7A0160497A43EA01239179D27978
:1060800041EA022293420CD20C4A83801278013AF0
:106090001A4202D10A4B01221A70FFF7A3FB01201A
:1060A00008BD8280F9E70020FAE700BF024F002018
:1060B000CC7B0100290A0020EC4E0020C27B0100AD
:1060C0000A4F002008B5074B044613B10021AFF377
:1060D0000080054B1868836A03B19847204600F09A
:1060E00069F800BF00000000487F010010B50139C9
:1060F0000244904201D1002005E0037811F8014FDD
:10610000A34201D0181B10BD0130F2E70A449142AE
:1061100000F1FF3300D1704710B511F8014B03F8BF
:10612000014F9142F9D110BD884210B501EB020434
:1061300002D98442234607D8431EA14208D011F851
:10614000012B03F8012FF8E7024401468A4200D1EF
:1061500010BD13F8014D02F8014DF7E70244034664
:10616000934200D1704703F8011BF9E710B50246CE
:10617000147813460132002CFAD1013B11F8012B9F
:1061800003F8012F002AF9D110BD10B5034672B1F2
:106190000139841813F8010B11F8012F904201D135
:1061A000A34201D1801A10BD0028F3D1FAE71046AE
:1061B000F9E70000FEE700BF3464010084660100D7
:1061C000246401006C6601002864010000000000E6
:1061D000000000000D0A000000000D0A0902A200E4
:1061E00006010080FA0904000002080650080705AD
:1061F000820240000007050202400000080B000276
:106200000202010409040000010202010405240045
:1062100010010524010302042402060524060000DF
:106220000705830310002009040000020A0000058E
:10623000070504024000000705840240000009042D
:1062400000000203000006092100010001222100D4
:10625000070581034000010705010340000109040F
:10626000000000FF0300070904000002FF0000090E
:1062700007050502400000070585024000000000F8
:10628000000000000000000000000000000000000E
:1062900000000000000000000000000000000000FE
:1062A00000000000000000000000000000000000EE
:1062B0000000000000000000030000006400000077
:1062C00000000000E0470020040000000000000083
:1062D00000000000000000000000000000000000BE
:1062E00000000000000000000000000000000000AE
:1062F000000000000000000000000000000000009E
:106300000000000000000000000000004800000045
:10631000DC7B0100187C0100007C0100040000000F
:1063200039393034003939303500393930360039AF
:106330003930330045524153452020204143540019
:106340002E2E2F2E2E2F2E2E2F736F757263652FEC
:10635000626F6172642F6D6963726F626974763205
:106360002F6D6963726F62697476322E63004D69B6
:1063700063726F3A62697420456475636174696F12
:106380006E616C20466F756E646174696F6E004259
:106390004243206D6963726F3A626974205632001D
:1063A00001000236000000000000000000000000B4
:1063B000380800204D4943524F42495448544D4DEE
:1063C0004943524F42495400000068747470733A54
:1063D0002F2F6D6963726F6269742E6F72672F64FD
:1063E00065766963652F3F69643D404226763D408E
:1063F0005600000000000000000000000000000047
:106400000000000000000000000000005D8A0000A5
:1064100000000000B5890000000000006E6301006C
:106420008F63010043535600574156004441544185
:106430002020202042494E002E2E2F2E2E2F2E2E91
:106440002F736F757263652F6461706C696E6B2F4B
:10645000486172644661756C745F48616E646C6516
:10646000722E63002E2E2F2E2E2F2E2E2F736F7531
:106470007263652F6461706C696E6B2F6369726300
:106480005F6275662E63004441504C696E6B00324A
:106490002E312E30002E2E2F2E2E2F2E2E2F736FBC
:1064A000757263652F6461706C696E6B2F647261C5
:1064B000672D6E2D64726F702F66696C655F7374E3
:1064C0007265616D2E6300484558002E2E2F2E2ECA
:1064D0002F2E2E2F736F757263652F6461706C6938
:1064E0006E6B2F647261672D6E2D64726F702F66F4
:1064F0006C6173685F6465636F6465722E63002E00
:106500002E2F2E2E2F2E2E2F736F757263652F64F4
:1065100061706C696E6B2F647261672D6E2D647291
:106520006F702F666C6173685F6D616E6167657215
:106530002E63002E2E2F2E2E2F2E2E2F736F757260
:1065400063652F6461706C696E6B2F647261672D77
:106550006E2D64726F702F6961705F666C61736815
:106560005F696E74662E63005DC3000019C300008E
:1065700015C50000EDC30000B5C40000FDC2000059
:1065800003C3000009C300000000000068650100AB
:106590002E2E2F2E2E2F2E2E2F736F757263652F9A
:1065A0006461706C696E6B2F647261672D6E2D640F
:1065B000726F702F7666735F6D616E616765722EA4
:1065C0006300000000000000FFFFFFFFFFFFFFFF70
:1065D000FFFFFFFFFFFFFFFF0000000000000000C3
:1065E0000000000000000000000000034120626F76
:1065F0006F746C6F6164657220757064617465207E
:10660000776173207374617274656420627574209D
:10661000756E61626C6520746F20636F6D706C6560
:1066200074652E0D0A52656C6F6164207468652074
:10663000626F6F746C6F6164657220746F2066693D
:10664000782074686973206572726F72206D65734B
:10665000736167652E0D0A004441504C494E4B2032
:10666000202020004D4245442020202048544D0049
:1066700044455441494C5320545854004641494CD8
:1066800020202020545854004E4545445F424C2061
:10669000545854002E2E2F2E2E2F2E2E2F736F7502
:1066A0007263652F6461706C696E6B2F64726167D1
:1066B0002D6E2D64726F702F7666735F75736572C1
:1066C0002E63004552524F520068747470733A2F13
:1066D0002F6D6265642E6F72672F646576696365DE
:1066E0002F3F636F64653D40553F76657273696FF8
:1066F0006E3D40563F7461726765745F69643D40EA
:1067000054003C21646F63747970652068746D6C0B
:106710003E0D0A3C212D2D206D62656420506C6178
:1067200074666F726D205765627369746520616E5F
:10673000642041757468656E7469636174696F6E15
:106740002053686F7274637574202D2D3E0D0A3CC2
:1067500068746D6C3E0D0A3C686561643E0D0A3CD0
:106760006D65746120636861727365743D22757430
:10677000662D38223E0D0A3C7469746C653E6D626C
:10678000656420576562736974652053686F72741D
:106790006375743C2F7469746C653E0D0A3C2F68F8
:1067A0006561643E0D0A3C626F64793E0D0A3C737C
:1067B00063726970743E0D0A77696E646F772E6C30
:1067C0006F636174696F6E2E7265706C61636528AA
:1067D000220040520022293B0D0A3C2F736372694C
:1067E00070743E0D0A3C2F626F64793E0D0A3C2F97
:1067F00068746D6C3E0D0A006572726F7200747978
:1068000070653A20002C20003000426F6F746C6F6E
:1068100061646572004170706C69636174696F6E68
:10682000004173736572740D0A0046696C65004C13
:10683000696E6500536F75726365004865786475AD
:106840006D70730D0A0023204441504C696E6B201B
:106850004669726D77617265202D207365652068C9
:10686000747470733A2F2F6461706C696E6B2E694B
:106870006F0D0A4275696C642049443A20763032C3
:1068800035372D6763373832613562612028676399
:1068900063290D0A00556E697175652049443A20D7
:1068A00040550D0A004849432049443A2040440DD0
:1068B0000A004175746F20526573657400417574E8
:1068C0006F6D6174696F6E20616C6C6F77656400C9
:1068D0004F766572666C6F77206465746563746962
:1068E0006F6E00496E636F6D70617469626C6520D4
:1068F000696D61676520646574656374696F6E00B6
:10690000506167652065726173696E6700446170EC
:106910006C696E6B204D6F64653A20496E746572C8
:10692000666163650D0A00496E7465726661636530
:106930002056657273696F6E3A2040560D0A004208
:106940006F6F746C6F616465722056657273696FE6
:106950006E3A2000476974205348413A2063373823
:1069600032613562613930373337373635386263F3
:1069700032386161386431333261306661343435C4
:1069800034333638370D0A4C6F63616C204D6F64B9
:10699000733A20300D0A55534220496E7465726671
:1069A000616365733A204D53442C204344432C20AB
:1069B0004849442C205765625553420D0A00426FE6
:1069C0006F746C6F616465722043524300496E744A
:1069D000657266616365204352430052656D6F7551
:1069E0006E7420636F756E740055524C3A2040529D
:1069F0000D0A00696E7465726E616C007472616E6E
:106A00007369656E74007573657200746172676591
:106A10007400696E74657266616365004153534525
:106A20005254202041435400524546524553482079
:106A3000414354004155544F5F525354434647001D
:106A4000484152445F525354434647004155544FC6
:106A50005F4F4E20434647004155544F5F4F4646D7
:106A6000434647004F56464C5F4F4E204346470033
:106A70004F56464C5F4F4646434647004D53445F92
:106A80004F4E2020434647004D53445F4F4646201B
:106A900043464700434F4D505F4F4E20434647000B
:106AA000434F4D505F4F4646434647005041474590
:106AB0005F4F4E2041435400504147455F4F46468B
:106AC00041435400415353455254202054585400DC
:106AD000F3690100FC690100066A01000B6A01000C
:106AE000126A010074760100000000001C6A0100B7
:106AF00001000000286A0100020000003463010068
:106B000003000000346A010004000000406A010034
:106B1000050000004C6A010006000000586A0100F0
:106B200007000000646A010008000000706A0100AC
:106B3000090000007C6A01000A000000886A010068
:106B40000B000000946A01000C000000A06A010024
:106B50000D000000AC6A01000E000000B86A0100E0
:106B60000F0000002E2E2F2E2E2F2E2E2F736F751E
:106B70007263652F6461706C696E6B2F64726167FC
:106B80002D6E2D64726F702F7669727475616C5FF3
:106B900066732E6300222A2B2C2E2F3A3B3C3D3E5F
:106BA0003F5B5C5D7C000000000000000000000016
:106BB000000100000000764876480000DC8376483B
:106BC000000000000000EB3C904D53443053342E45
:106BD000310002080100022000501FF801000100EE
:106BE00001000000000000000000000029741902EC
:106BF000274441504C494E4B2D444E44464154315C
:106C000036202020FAB8C0070520018ED0BC001025
:106C1000B8C0078ED8BE6D00E80B00EBFEB40EB70F
:106C200000B307CD10C38A044608C07405E8EDFF21
:106C3000EBF4C3504C454153452052454D4F56450A
:106C4000205448452041524D204D42454420444166
:106C5000504C494E4B2055534220444556494345DC
:106C600020414E44205245424F4F54205448452025
:106C700053595354454D2E2E0000000000000000D3
:106C80000000000000000000000000000000000004
:106C900000000000000000000000000000000000F4
:106CA00000000000000000000000000000000000E4
:106CB00000000000000000000000000000000000D4
:106CC00000000000000000000000000000000000C4
:106CD00000000000000000000000000000000000B4
:106CE00000000000000000000000000000000000A4
:106CF0000000000000000000000000000000000094
:106D00000000000000000000000000000000000083
:106D10000000000000000000000000000000000073
:106D20000000000000000000000000000000000063
:106D30000000000000000000000000000000000053
:106D40000000000000000000000000000000000043
:106D50000000000000000000000000000000000033
:106D60000000000000000000000000000000000023
:106D70000000000000000000000000000000000013
:106D80000000000000000000000000000000000003
:106D900000000000000000000000000000000000F3
:106DA00000000000000000000000000000000000E3
:106DB00000000000000000000000000000000000D3
:106DC0000000000055AA00000000000000000000C4
:106DD000002800000000000000000000418EBB32CF
:106DE0000000000000000000FDD90000C5D900002F
:106DF00000020000DDD90000C5D90000000000003D
:106E0000DDD90000C5D90000000000001DDA000037
:106E10005DDE0000000400002E2E2F2E2E2F2E2EC1
:106E20002F736F757263652F6461706C696E6B2F61
:106E30006572726F722E63004F7065726174696F54
:106E40006E20776173207375636365737366756C09
:106E500000416E206572726F7220686173206F63EB
:106E600063757272656400416E20696E7465726E3E
:106E7000616C206572726F7220686173206F63634A
:106E8000757272656400416E206572726F72206F58
:106E90006363757272656420647572696E672074CD
:106EA0006865207472616E7366657200546865204F
:106EB0007472616E736665722074696D6564206FAB
:106EC00075742E00506F737369626C65206D697301
:106ED0006D61746368206265747765656E206669AC
:106EE0006C652073697A6520616E642073697A65C8
:106EF0002070726F6772616D6D65640046696C65C4
:106F00002073656E74206F7574206F66206F7264D5
:106F100065722062792050432E2054617267657437
:106F2000206D69676874206E6F74206265207072CE
:106F30006F6772616D6D656420636F7272656374F3
:106F40006C792E004661696C656420746F207265EF
:106F50007365742F68616C74207468652074617245
:106F6000676574204D4355004661696C6564207403
:106F70006F20646F776E6C6F616420666C617368FC
:106F800020616C676F726974686D20746F20746122
:106F900072676574204D435500466C6173682061CB
:106FA0006C676F726974686D206D697373696E6761
:106FB00020666F72206120726567696F6E0046619E
:106FC000696C656420746F20646F776E6C6F6164A8
:106FD0002074686520666C61736820646174612048
:106FE000636F6E74656E747320746F2062652070B9
:106FF000726F6772616D6D6564004661696C65648E
:1070000020746F20696E697469616C697A65207497
:10701000686520746172676574204D435500466150
:10702000696C656420746F20756E696E697469613E
:107030006C697A6520746865207461726765742074
:107040004D43550050726F6772616D6D696E6720B8
:1070500061626F727465643A20696D61676520775B
:107060006F756C64206C6F636B20746172676574FC
:10707000204D4355004661696C656420746F20752E
:107080006E6C6F636B20746172676574204D43553D
:1070900020666F722070726F6772616D6D696E67C6
:1070A00000466C61736820616C676F726974686D0B
:1070B00020657261736520736563746F7220636FFE
:1070C0006D6D616E64204641494C55524500466CD9
:1070D00061736820616C676F726974686D20657296
:1070E00061736520616C6C20636F6D6D616E6420EF
:1070F0004641494C55524500466C61736820616CAD
:10710000676F726974686D20777269746520636F48
:107110006D6D616E64204641494C55524500466C88
:1071200061736820616C676F726974686D20777233
:107130006974652076657269667920636F6D6D612B
:107140006E64204641494C55524500456E64206F9F
:10715000662073747265616D206861732062656575
:107160006E207265616368656400456E64206F66B9
:107170002073747265616D20697320756E6B6E6F1C
:10718000776E00546865206865782066696C6520B4
:1071900063616E6E6F74206265206465636F646501
:1071A000642E20436865636B73756D2063616C6347
:1071B000756C6174696F6E206661696C75726520AB
:1071C0006F636375727265642E005468652068652C
:1071D000782066696C652063616E6E6F74206265ED
:1071E000206465636F6465642E20506172736572FC
:1071F000206C6F676963206661696C757265206FCA
:10720000636375727265642E0054686520686578E2
:107210002066696C652063616E6E6F742062652004
:1072200070726F6772616D6D65642E204C6F676957
:1072300063206661696C757265206F636375727235
:1072400065642E00546865206865782066696C6501
:1072500020796F752064726F707065642069736E39
:10726000277420636F6D70617469626C6520776943
:1072700074682074686973206D6F6465206F722074
:107280006465766963652E2041726520796F75208B
:10729000696E204D41494E54454E414E4345206D47
:1072A0006F64653F205365652048454C502046413A
:1072B000512E48544D0054686520686578206669F1
:1072C0006C65206F6666736574206C6F6164206105
:1072D000646472657373206973206E6F7420636FCA
:1072E00072726563742E00546865207374617274E1
:1072F000696E67206164647265737320666F7220C3
:1073000074686520626F6F746C6F6164657220755C
:1073100070646174652069732077726F6E672E00E8
:10732000546865207374617274696E672061646467
:107330007265737320666F722074686520696E745D
:107340006572666163652075706461746520697338
:107350002077726F6E672E00546865206170706CC4
:1073600069636174696F6E2066696C6520666F720F
:107370006D617420697320756E6B6E6F776E20611E
:107380006E642063616E6E6F74206265207061723E
:1073900073656420616E642F6F722070726F636515
:1073A000737365642E00546865206170706C696346
:1073B0006174696F6E20696D616765206973206E05
:1073C0006F7420636F6D70617469626C652077699A
:1073D000746820746865207461726765742E004952
:1073E0006E206170706C69636174696F6E20707279
:1073F0006F6772616D6D696E6720696E697469612E
:107400006C697A6174696F6E206661696C65642E5F
:1074100000496E206170706C69636174696F6E20E1
:1074200070726F6772616D6D696E6720756E696EDF
:107430006974206661696C65642E00496E20617014
:10744000706C69636174696F6E2070726F677261CE
:107450006D6D696E67207772697465206661696C0D
:1074600065642E00496E206170706C696361746997
:107470006F6E2070726F6772616D6D696E672073D9
:107480006563746F72206572617365206661696CF3
:1074900065642E00496E206170706C696361746967
:1074A0006F6E2070726F6772616D6D696E67206DAF
:1074B000617373206572617365206661696C6564D0
:1074C0002E00496E206170706C69636174696F6E23
:1074D0002070726F6772616D6D696E672061626F97
:1074E000727465642064756520746F20616E206F0E
:1074F0007574206F6620626F756E647320616464BA
:10750000726573732E00496E206170706C696361DF
:1075100074696F6E2070726F6772616D6D696E67EE
:10752000206E6F7420737570706F72746564206F55
:107530006E2074686973206465766963652E0049FE
:107540006E206170706C69636174696F6E20707217
:107550006F6772616D6D696E67206661696C6564E5
:107560002062656361757365207468652075706459
:107570006174652073656E742077617320696E6332
:107580006F6D706C6574652E0054686520626F6F56
:10759000746C6F6164657220435243206469642097
:1075A0006E6F7420706173732E000000386E0100DE
:1075B000516E0100676E0100866E0100AC6E010025
:1075C000C46E0100FC6E0100446F0100686F010091
:1075D000996F0100BE6F0100FA6F01001E7001007B
:1075E0004470010075700100A1700100CE700100AF
:1075F000F87001001E7101004B7101006A710100F9
:1076000083710100CA710100097201004472010016
:10761000B6720100E7720100207301005873010087
:10762000A6730100DF730100117401003B740100B7
:107630006474010094740100C274010006750100B5
:107640003F75010094680100897501000001010285
:1076500006020208080808080804080808080801C3
:10766000010606060404040404041010101010108F
:107670001010101053544152545F424C4143542E49
:107680002E2F2E2E2F2E2E2F736F757263652F6463
:1076900061706C696E6B2F696E746572666163658B
:1076A0002F6D61696E5F696E746572666163652EC8
:1076B000630033306D73006D61696E00B776010051
:1076C00000000000283B002044000000C8370020D4
:1076D000600300001800000000000000000000002F
:1076E000B2760100000000006C3B0020200000008A
:1076F0002E2E2F2E2E2F2E2E2F736F757263652F29
:107700006461706C696E6B2F696E7465726661631B
:10771000652F7461726765745F666C6173682E6350
:10772000000000009DF400003DF80000E1F20000C0
:10773000A1F7000055F6000011F8000019F700004D
:1077400035F20000C9F500002477010000000000B8
:107750000000010101003031323334353637383919
:10776000616263646566004E6F7264696353656D40
:1077700069636F6E647563746F72006E5246353262
:107780003834305F78784141006E524635323833B4
:10779000335F78784141006E524635323833325F7C
:1077A00078784141006E524635323833325F78780E
:1077B0004142002100002025000020290000204D2A
:1077C0000000207B0000200000000001000020706D
:1077D00001002000100020000200200000002050C6
:1077E000010000F07701000002000000000000002E
:1077F00000BE0AE00D782D0668400824400000D342
:107800005840641EFAD1491C521E002AF2D170471A
:10781000002070470020704770B52B4C022020607C
:107820002949012008310860284D2868C00702D086
:107830000020206070BD00F033F8F6E770B5224CF0
:1078400002212160B0F1102F03D31F490120103114
:1078500001E01D49091D08601C4D00F021F8286851
:10786000C007FAD00020206070BD2DE9F041DFF89C
:1078700058808E08012114460546C8F80010134FA1
:1078800001CC01C53868C00707D0761EF8D10021A9
:10789000C8F800100846BDE8F08100F001F8F1E7F3
:1078A0000B48006810F0FF000CD00A490968002955
:1078B00008D00849084AFC31C30700D00A60091DF6
:1078C0004008F9D17047000004E5014000E40140A0
:1078D00004040140040501403546526E00000000DA
:1078E000000000000010000002360200040000004A
:1078F0000000000000000000000000000000000088
:10790000000000001900010000000000000000005D
:10791000000000000402000191000100BD00010010
:10792000250201007503010021030100C1000100CF
:10793000C7000100E10101009D0101007D0101007E
:1079400025010100CD0001000030004000000000D2
:107950008D020100503C0020A9030100D503010065
:10796000DD0301006109010055080100CD07010098
:10797000F9030100350401003D0401004904010040
:107980006104010091070100390801009D07010011
:1079900003020001000001000000013C4441504C82
:1079A000696E6B3A4F766572666C6F773E0A004D72
:1079B00042454420202020564653202020202020CD
:1079C00020202020202020302E3100050F390002F9
:1079D0001810050038B60834A909A0478BFDA07619
:1079E0008815B665000121001C100500DF60DDD898
:1079F0008945C74C9CD2659D9E648A9F0000030602
:107A00004A012000400012011002EF020140280D3F
:107A1000040200100102030100000600FF0901A199
:107A200001150026FF007508954009018102954067
:107A30000901910295010901B102C0002100400035
:107A4000D51501005D580100314301007956010050
:107A5000493C0100BD3C01005D3701000000000011
:107A60000000000000000000000000000000000016
:107A70000000000000000000000000000000000006
:107A8000000000000000000000000000D915010007
:107A900000000000E71501000000000004030904D5
:107AA0000803410072006D003003420042004300B1
:107AB00020006D006900630072006F003A006200F0
:107AC00069007400200043004D005300490053003A
:107AD0002D004400410050001A03300030003000F7
:107AE0003100410030003000300030003000300004
:107AF000300022036D006200650064002000530026
:107B000065007200690061006C00200050006F0089
:107B10007200740022036D006200650064002000A2
:107B2000530065007200690061006C002000500085
:107B30006F00720074001A0343004D0053004900A7
:107B400053002D0044004100500020007600310019
:107B500024035700650062005500530042003A00BC
:107B6000200043004D005300490053002D00440005
:107B70004100500010035500530042005F004D00CB
:107B8000530043001A0343004D00530049005300C3
:107B90002D00440041005000200076003200010515
:107BA0000500400000020404400040004000400086
:107BB00001014000010001000200400040004000BF
:107BC00001004002020040000002002120525458EF
:107BD0002056352E352E3200000000000000000037
:107BE00000000000B8480020440000008049002048
:107BF000480000000100000000000000000000003C
:107C00000000000000000000F047002034000000E9
:107C10002448002050000000000000000000000088
:107C2000744800204400000000490020800000004B
:107C3000280000000000000000000000000000001C
:107C40000000000000000000000000000000000034
:107C50000000000000000000000000000000000024
:107C60000000000000000000010001000000000012
:107C70000000000000000000000000000000000004
:107C800000000000000000000000000000000000F4
:107C900000000000000000000000000000000000E4
:107CA00000000000000000000000000000000000D4
:107CB00000000000000000000000000000000000C4
:107CC00000000000000000000000000000000000B4
:107CD00000000000000000000000000000000000A4
:107CE0000000000000000000000000000000000094
:107CF0000000000000000000000000000000000084
:107D00000000000000000000000000000000000073
:107D10000000000000000000000000000000000063
:107D20000000000000000000000000000000000053
:107D30000000000000000000000000000000000043
:107D40000000000000000000000000000000000033
:107D50000000000000000000000000000000000023
:107D60000000000000000000000000000000000013
:107D70000000000000000000000000000000000003
:107D800000000000000000000000000000000000F3
:107D900000000000000000000000000000000000E3
:107DA00000000000000000000000000000000000D3
:107DB00000000000000000000000000000000000C3
:107DC00000000000000000000000000000000000B3
:107DD00000000000000000000000000000000000A3
:107DE0000000000000000000000000000000000093
:107DF0000000000000000000000000000000000083
:107E00000000000000000000000000000000000072
:107E10000000000000000000000000000000000062
:107E20000000000000000000000000000000000052
:107E30000000000000000000000000000000000042
:107E40000000000000000000000000000000000032
:107E50000000000000000000000000000000000022
:107E60000000000000000000000000000000000012
:107E700000000000000000000300020004000000F9
:107E800000000000000000000000000000000000F2
:107E900000000000000000000000000000000000E2
:107EA00000000000020002000100000000000000CD
:107EB00000000000000000000000000000000000C2
:107EC00000000000000000000000000000000000B2
:107ED00000000000000000000000000000000000A2
:107EE0000000000000000000000000000000000092
:107EF0000000000000000000000000002E2E2F2EC9
:107F00002E2F2E2E2F736F757263652F7573622F50
:107F10006869642F757362645F757365725F686901
:107F2000642E63002E2E2F2E2E2F2E2E2F736F7564
:107F30007263652F7573622F6D73632F757362643F
:107F40005F6D73632E630000680C0020F8B500BFFE
:107F5000F8BC08BC9E467047F8B500BFF8BC08BC2A
:107F60009E467047DC04FF7F01000000258400006E
:107F7000018400007407000000000220B502000028
:107F8000DD020000DF020000E1020000E302000069
:107F9000E5020000000000000000000000000000FA
:107FA00000000000E7020000E902000000000000FD
:107FB000EB020000ED020000EF020000EF02000003
:107FC000EF020000EF020000EF020000EF020000ED
:107FD000EF020000EF020000EF020000EF020000DD
:107FE000EF020000EF020000EF020000EF020000CD
:107FF000EF020000EF020000EF020000EF020000BD
:10800000EF020000EF020000EF020000EF020000AC
:10801000EF020000EF020000EF020000EF0200009C
:10802000EF020000EF020000EF020000EF0200008C
:108030000000000000000000EF020000EF0200005E
:10804000EF020000EF020000EF020000EF0200006C
:10805000EF020000EF020000EF020000000000004D
:10806000000000000000000000000000EF0200001F
:1080700000000000EF02000000000000000000000F
:1080800000000000000000000000000000000000F0
:1080900000000000000000000000000000000000E0
:1080A00000000000000000000000000000000000D0
:1080B00000000000000000000000000000000000C0
:1080C00000000000000000000000000000000000B0
:1080D00000000000000000000000000000000000A0
:1080E0000000000000000000000000000000000090
:1080F0000000000000000000000000000000000080
:10810000000000000000000000000000000000006F
:10811000000000000000000000000000000000005F
:10812000000000000000000000000000000000004F
:10813000000000000000000000000000000000003F
:10814000000000000000000000000000000000002F
:10815000000000000000000000000000000000001F
:10816000000000000000000000000000000000000F
:10817000000000000000000010B5054C237833B962
:10818000044B13B10448AFF300800123237010BDEA
:1081900074000020000000006007000008B5034BD9
:1081A0001BB103490348AFF3008008BD0000000085
:1081B0007800002060070000154B002B08BF134B10
:1081C0009D46A3F5803A00218B460F461348144A7A
:1081D000121A00F047FA0F4B002B00D098470E4BB5
:1081E000002B00D098470020002104000D000D480E
:1081F000002802D00C48AFF3008000F00FFA2000F6
:10820000290000F0EDF900F0F5F900BF00000800CA
:1082100000000220000000000000000074000020A8
:108220009000002000000000000000000649074AFE
:10823000074B9B1A03DD043BC858D050FBDC00F011
:108240002FF8FFF7B9FF00006C07000000000020C6
:1082500074000020FEE7FEE7FEE7FEE7FEE7FEE72C
:10826000FEE7FEE7FEE7FEE7BFF34F8F0549064B4B
:10827000CA6802F4E0621343CB60BFF34F8F00BFC4
:10828000FDE700BF00ED00E00400FA05034B1868AD
:10829000A0F10D0358425841704700BF3001001053
:1082A00008B5FFF7F3FF40B14FF080430022C3F859
:1082B0000C21C3F81021C3F83825FFF7E7FF002889
:1082C00046D04FF08052594BD2F80414C3F8201511
:1082D000D2F80814C3F82415D2F80C14C3F82815E2
:1082E000D2F81014C3F82C15D2F81414C3F83015B2
:1082F000D2F81814C3F83415D2F81C14C3F840157A
:10830000D2F82014C3F84415D2F82414C3F8481541
:10831000D2F82814C3F84C15D2F82C14C3F8501511
:10832000D2F83014C3F85415D2F83414C3F86015D9
:10833000D2F83814C3F86415D2F83C14C3F86815A1
:10834000D2F84014C3F86C15D2F84424C3F8702551
:10835000FFF79CFF48B14FF08043D3F80024D107CA
:1083600044BF6FF00102C3F80024314AD2F88830CC
:1083700043F47003C2F88830BFF34F8FBFF36F8FA1
:108380004FF01023D3F80C22D2071ED5294B01221F
:10839000C3F80425D3F80024002AFBD04FF01022A4
:1083A000D2F80C3223F00103C2F80C32214B1A46EA
:1083B000D3F800140029FBD00021C3F80415D2F82B
:1083C0000034002BFBD0FFF74FFFD3F80022002A28
:1083D00003DBD3F80432002B23DA164B0122C3F857
:1083E0000425D3F80024002AFBD04FF010221221DC
:1083F000C2F80012D3F80024002AFBD04FF010235B
:108400001222C3F804220B4B1A46D3F80014002999
:10841000FBD00021C3F80415D2F80034002BFBD0A8
:10842000D1E7054B054A1A6008BD00BF00C00040F7
:1084300000ED00E000E00140000000200090D003CB
:108440001F2886BF00F01F00044A4FF0A0420123FE
:1084500003FA00F0C2F80805704700BF000300509F
:10846000805CC1F104010841C04300F00100704785
:1084700000234FF0A042834200DB7047D2F804157E
:108480000133F8E738B51C20FFF7DAFF0B20FFF7C0
:10849000D7FF1F20FFF7D4FF2520FFF7D1FF0B4C9C
:1084A0000B4D1E20FFF7CCFF00220120135D1F2B78
:1084B00086BF03F01F0329464FF0A041013200FAA6
:1084C00003F3052AC1F80C35F0D138BD540700007C
:1084D000000300502DE9F84F80463B483B4D0022F9
:1084E00082460324135C1F2B86BF03F01F0329461B
:1084F0004FF0A04103F5E0730132052A41F8234013
:10850000F0D13348314D00220324135C1F2B86BF6A
:1085100003F01F0329464FF0A04103F5E073013239
:10852000052A41F82340F0D1FFF7ACFF4FF00109D5
:10853000284C002632270025254B585DFFF780FF89
:108540004FF0000B2A46594620461AF80B30FFF729
:1085500087FFA0BB1F2B86BF03F01F031B4A4FF0F2
:10856000A04209FA03F3C2F80C350BF1010BBBF181
:10857000050FE7D144F620600135FFF779FFFFF7DB
:1085800081FF052DD8D1013FD5D113480136FFF722
:108590006FFF042ECCD0314664230A2202E0013959
:1085A00093FBF2F30129FAD198FBF3F393FBF2F476
:1085B00002FB1434094B04EB84041C44BAE718464C
:1085C000FFF73EFFD1E700BF4A070000000300505D
:1085D000540700004F07000040420F00180700003A
:1085E00008B5034B9888FFF775FF002008BD00BF52
:1085F0000400002008B5074B044613B10021AFF377
:108600000080054B1868836A03B19847204600F044
:1086100031F800BF000000005C07000070B50D4E8F
:108620000D4CA41BA4100025A54209D10B4E0C4CE7
:1086300000F022F8A41BA4100025A54205D170BDAE
:1086400056F8253098470135EEE756F8253098471B
:108650000135F2E76C0000206C0000206C00002067
:108660007000002002440346934200D1704703F893
:10867000011BF9E7FEE700BFF8B500BFF8BC08BC76
:108680009E467047F8B500BFF8BC08BC9E467047D0
:108690000C9252524C048C84848E1C824C901E1E70
:1086A000C244924C06CA525FE21FF01EC13E024411
:1086B0008ED12E1FE24488100ED12ED12E0ED12E37
:1086C000C4881C0B1F251E1B1B000E1115160F182E
:1086D000130000000C00002000000000DCFAFF7F07
:1086E000010000000090D003DEC0CEFA460000007A
:1086F000000000000000000000000000000000007A
:108700000000000000000000000000000000000069
:108710000000000000000000000000000000000059
:108720000000000000000000000000000000000049
:108730000000000000000000000000000000000039
:108740000000000000000000000000000000000029
:108750002502000001020000E0070000010003996B
:10876000039908FF01FF01006766637344415441A8
:108770002020202042494E0000E0010000000000BF
:108780000000000029B8000017B800003BB8000046
:1087900059B700001BB80000F9B700005DB7000032
:1087A000EDB800000101010004000000010000001C
:1087B000E078010001000000000000000000080057
:1087C0000100000000000000B3770100000000007D
:1087D0000000000000000000000000000000000099
:1087E0000000000000000000000000000000000089
:1087F0000000000000000000000000000000000079
:108800000000000000000000000000000000000068
:108810000000000000000000000000000000000058
:108820000000000000000000000000000000000048
:108830000000000000000000000000000000000038
:108840000000000000000000000000000000000028
:108850000000000000000000000000000000000018
:108860000000000000000000000000000000000008
:1088700000000000000000000000000000000000F8
:1088800000000020000002200000000000000000A6
:1088900000000000000000000000000000000000D8
:1088A00000000000000000000000000000000000C8
:1088B00000000000000000000000000000000000B8
:1088C00000000000000000000000000000000000A8
:1088D0000000000000000000000000000000000098
:1088E0000000000000000000000000000000000088
:1088F0000000000000000000000000000000000078
:108900000000000000000000000000000000000067
:108910000000000000000000000000000000000057
:108920000000000000000000000000000000000047
:108930000000000000000000000000000000000037
:108940000000000000000000000000000000010026
:1089500067770100897701000090D0036B002C033A
:10896000016F732E6D6265642E636F6D2F77656284
:108970007573622F6C616E64696E672D70616765D7
:108980002F3F6269643D000000001303016F732EE6
:108990006D6265642E636F6D2F000000000A000099
:1089A00000000003064A01080002000000A00014B5
:1089B00000030057494E55534200000000000000DC
:1089C0000000008400040007002A004400650076CF
:1089D0000069006300650049006E00740065007264
:1089E00000660061006300650047005500490044CF
:1089F000007300000050007B003900320043004546
:108A00000036003400360032002D003900430037B4
:108A10000037002D0034003600460045002D003997
:108A2000003300330042002D003300310043004288
:108A30000039004300350041004100330042003955
:108A4000007D0000000000080002000000A00014EB
:108A500000030057494E555342000000000000003B
:108A60000000008400040007002A0044006500762E
:108A70000069006300650049006E007400650072C3
:108A8000006600610063006500470055004900442E
:108A9000007300000050007B00430044004200339C
:108AA0000042003500410044002D003200390033FF
:108AB0000042002D0034003600360033002D004106
:108AC000004100330036002D0031004100410045D7
:108AD00000340036003400360033003700370036EB
:108AE000007D00000000000006000000AF790100DA
:108AF000CD7B0100D2B3FB020000000000000000AB
:108B00000000000000000000000000000000000065
:108B10000000000000000000000000000000000055
:108B20000000000000000000000000000000000045
:108B30000000000000000000000000000000000035
:108B40000000000000000000000000000000000025
:108B50000000000000000000000000000000000015
:108B60000000000000000000000000000000000005
:108B700000000000000000000000000000000000F5
:108B800000000000000000000000000000000000E5
:108B900000000000687C0100A47E0100787E0100D6
:108BA000447D0100707D0100187D01009C7D010065
:108BB000C87D0100F47D0100EC7C0100E878010033
:108BC000207E01004C7E0100D07E01003C7C010033
:108BD000947C0100C07C0100FFFFFFFF000000004B
:108BE0000000000000000000000000000000000085
:108BF0000000000000000000000000000000000075
:108C00000000000000000000000000000000000064
:108C10000000000000000000000000000000000054
:108C20000000000000000000000000000000000044
:108C3000000000000000000000000000FFFFFFFF38
:108C4000FFFFFFFFFFFFFFFFFFFFFFFFFFFFFFFF34
:108C5000FFFFFFFFFFFFFFFFFFFFFFFFFFFFFFFF24
:108C6000FFFFFFFFFFFFFFFFFFFFFFFFFFFFFFFF14
:108C7000FFFFFFFFFFFFFFFFFFFFFFFFFFFFFFFF04
:10EFF000FFFFFFFFFFFFFFFFFFFFFFFFDEF161E508
:00000001FF
